:100000000C94D2030C94EF030C946B2E0C94EF031E
:100010000C94EF030C94EF030C94EF030C94EF0398
:100020000C94EF030C94F2450C94EF030C94EF0343
:100030000C94EF030C94EF030C94EF030C94EF0378
:100040000C94EF030C94EF030C94EF030C94EF0368
:100050000C94EF030C949F540C94EF030C94EF0357
:100060000C94EF030C94EF030C94EF030C94EF0348
:100070000C94EF030C94EF030C94EF030C94EF0338
:100080000C94EF030C94EF030C94EF030C94EF0328
:100090000C94EF037747C2478148A7481F4943495B
:1000A00068496C497C490752075207520752075268
:1000B0000752075207520752075207520752075278
:1000C0000752075207520752075207520752075268
:1000D00007520F4A8C49A8492E4A3E4AB24BFC4B64
:1000E000894CCB4C074D7A4D0752075207520752A5
:1000F0000752075207520752075207520752075238
:100100000752075207520752075207520752075227
:1001100007526D4AB24AE84D014E314E484E0752E1
:100120000752075207520752075207520752075207
:100130000752E24A3A4B554ED54E544F964F4951CD
:1001400058510D502150675179518C5107529D5192
:100150001F4B474B6F4BD151EC51D74FF24F35509E
:1001600069508C50D850F3501E51CE03C103B303D5
:10017000A30390037A036103470329030803E602FC
:10018000C2029E0276024F02280203026C01B801ED
:1001900096017501560139011F010601EF00DA00D1
:1001A000B5008200A5009600000043414E203100BA
:1001B00000000000000000000043414E203200001B
:1001C000000000000000000043414E20330000000A
:1001D0000000000000000043414E203400000000F9
:1001E00000000000000043414E20350000000000E8
:1001F000000000000043414E2036000000000000D7
:100200000000000043414E203700000000000000C5
:1002100000000043414E20380000000000000000B4
:10022000000043414E2039000000000000000000A3
:100230000043414E2031300000000000000000006B
:1002400043414E2031310000000000000000004317
:10025000414E203132000000000000000000434108
:100260004E20313300000000000000000043414EEA
:1002700020313400000000000000000043414E2007
:10028000313500000000000000000043414E2031E5
:100290003600000000000000000043414E203137CE
:1002A00000000000000000000043414E20313800F3
:1002B000000000000000000043414E2031390000E2
:1002C0000000000000000043414E203230000000DA
:1002D00000000000000043414E20323100000000C9
:1002E000000000000043414E2032320000000000B8
:1002F0000000000043414E203233000000000000A7
:1003000000000043414E2032340000000000000095
:10031000000043414E203235000000000000000084
:100320000043414E20323600000000000000000073
:1003300043414E203237000000000000000000431F
:10034000414E203238000000000000000000434110
:100350004E20323900000000000000000043414EF2
:1003600020333000000000000000000043414E2018
:10037000333100000000000000000043414E2033F4
:1003800032000000000000000000466C617368202D
:10039000310000000000000000466C6173682032EC
:1003A0000000000000000000466C6173682033000C
:1003B00000000000000000466C61736820340000FB
:1003C000000000000000466C6173682035000000EA
:1003D00000000000005357495443482031000000FA
:1003E00000000000535749544348203200000000E9
:1003F00000000053574954434820330000000000D8
:1004000000005357495443482034000000000000C6
:1004100000535749544348203500000000000000B5
:100420005357495443482036000000000000005351
:10043000574954434820370000000000000053573C
:100440004954434820380000000000000053574939
:10045000544348203900000000000000535749541D
:1004600043482031300000000000005357495443F6
:10047000482031310000000000004348414E4E4505
:100480004C20310000000000004348414E4E454CD6
:1004900020320000000000004348414E4E454C20F1
:1004A000330000000000004348414E4E454C2034CC
:1004B0000000000000004348414E4E454C203500EE
:1004C00000000000004348414E4E454C20360000DD
:1004D000000000004348414E4E454C2037000000CC
:1004E0000000004348414E4E454C203800000000BB
:1004F00000004348414E4E454C20390000000000AA
:10050000004348414E4E454C203130000000000071
:100510004348414E4E454C2031310000000000431D
:1005200048414E4E454C2031320000000000434807
:10053000414E4E454C2031330000000000434841FD
:100540004E4E454C20313400000000004348414EDF
:100550004E454C20313500000000004348414E4ECE
:10056000454C20313600000000004348414E4E45C6
:100570004C20313700000000004348414E4E454CAE
:1005800020313800000000004348414E4E454C20C9
:10059000313900000000004348414E4E454C2032A6
:1005A0003000000000004348414E4E454C2032319F
:1005B00000000000004348414E4E454C20323200BE
:1005C000000000004348414E4E454C2032330000AD
:1005D0000000004348414E4E454C2032340000009C
:1005E00000004348414E4E454C203235000000008B
:1005F000004348414E4E454C20323600000000007A
:100600004348414E4E454C20323700000000004325
:1006100048414E4E454C203238000000000043480F
:10062000414E4E454C203239000000000043484105
:100630004E4E454C20333000000000004348414EF0
:100640004E454C20333100000000004348414E4EDF
:10065000454C20333200000000004348414E4E45D7
:100660004C20333300000000004348414E4E454CBF
:1006700020333400000000005649525455414C20AC
:10068000310000000000005649525455414C2032C0
:100690000000000000005649525455414C203300E0
:1006A00000000000005649525455414C20340000CF
:1006B000000000005649525455414C2035000000BE
:1006C0000000005649525455414C203600000000AD
:1006D00000005649525455414C203700000000009C
:1006E000005649525455414C20380000000000008B
:1006F0005649525455414C20390000000000005624
:1007000049525455414C20313000000000005649F8
:10071000525455414C2031310000000000564952DE
:100720005455414C203132000000000056495254CB
:1007300055414C20313300000000005649525455B9
:10074000414C2031340000000000564952545541BC
:100750004C20313500000000005649525455414CA0
:1007600020313600000000005649525455414C20BB
:10077000313700000000005649525455414C203199
:100780003800000000005649525455414C20313980
:1007900000000000005649525455414C20323000B0
:1007A0000000000011241FBECFEFD0E1DEBFCDBF9F
:1007B00011E0A0E0B1E0EAE8FDEC00E00BBF02C010
:1007C00007900D92AA3AB107D9F71EE0AAEAB1E064
:1007D00001C01D92A63FB107E1F70C945F380C945D
:1007E0000000282F277099279695879596958795CD
:1007F0009695879533272330310529F1243031052B
:100800004CF421303105B9F022303105C4F4232BEA
:1008100071F02CC025303105F1F025303105BCF0E8
:1008200026303105E1F027303105E9F01FC0A098EE
:10083000A198A2981BC0A09AA198A29817C0A098AE
:10084000A19AA29813C0A09AA19AA2980FC0A098AA
:10085000A198A29A0BC0A09AA198A29A07C0A098AA
:10086000A19AA29A03C0A09AA19AA29A80628093A8
:100870007C0020E02F5F2A3FE8F380917A008061BE
:1008800080937A0080917A00806480937A008091CE
:100890007A0084FFFCCF209178008091790099271D
:1008A000880F991F880F991F2295269526952370EA
:1008B000820F911D0895282F277099279695879567
:1008C000969587959695879533272330310529F19D
:1008D000243031054CF421303105B9F02230310596
:1008E000C4F4232B71F02CC025303105F1F02530F4
:1008F0003105BCF026303105E1F027303105E9F053
:100900001FC0A098A198A2981BC0A09AA198A298D5
:1009100017C0A098A19AA29813C0A09AA19AA298D1
:100920000FC0A098A198A29A0BC0A09AA198A29AD1
:1009300007C0A098A19AA29A03C0A09AA19AA29ACD
:10094000806280937C0080917A00806480937A003A
:1009500080917A0084FFFCCF80917A00806180933F
:100960007A00809179009927089540E050E0FC01D9
:100970000296259134916217730760F44B5F5F4FC5
:10098000FC010296259134916217730718F44639D9
:100990005105A4F3CA010895FC0180910001813042
:1009A000B1F410920001F093B301E093B201F0931F
:1009B000B101E093B001F093AF01E093AE01F09389
:1009C000AD01E093AC01F093AB01E093AA0160911B
:1009D000B0017091B1017093B3016093B201409185
:1009E000AE015091AF015093B1014093B0012091FD
:1009F000AC013091AD013093AF012093AE018091F5
:100A0000AA019091AB019093AD018093AC01F0935A
:100A1000AB01E093AA01E80FF91FE20FF31FE40F07
:100A2000F51FCF01860F971F65E070E00E940C66EE
:100A3000CB01089580E10E94F1030E94CC04BC0127
:100A40008AE691E00E94B5049927089583E10E9407
:100A50005B042091720E3327829FA001839F500D6B
:100A6000929F500D11249A01220F232F221F330B26
:100A700031952F3F310519F010F04FEF01C0422F93
:100A80008091B401882339F44093B6014093B501B5
:100A90004093B40118C08091B601280F311D909188
:100AA000B501290F311D8091B401280F311D90939C
:100AB000B6018093B5014093B401C901969587951D
:100AC00096958795482F842F9927089580E28093E3
:100AD0007C0087E880937A00989A999A9A9AA098CD
:100AE000A198A298089590E0892F8295807F8093A5
:100AF000ED001092EE001092EF001092F0001092B4
:100B0000F1001092F2001092F3001092F400109293
:100B1000F5001092F6001092F70080E01092FA00B3
:100B20008F5F8830D8F39F5F9F30F0F20895309147
:100B3000ED0090E020EC892F8295807F8093ED007E
:100B40008091EF00822329F43093ED00892F9927BB
:100B500008959F5F9F3078F33093ED008FEF90E022
:100B600008958091EE0086FF03C080E090E0089534
:100B70008091EE0085FF03C081E090E008958091B0
:100B8000EF00807C19F48FEF90E0089582E090E010
:100B90000895BC0140E08091EF0099278F7090701C
:100BA000892B89F0FB01E40FF11D8091FA0080830D
:100BB0004F5F242F33278091EF0099278F7090701B
:100BC000281739077CF3089589E79DE00E94AC352A
:100BD0006FE17EE080E00E94E93567ED7DE081E035
:100BE0000E94E93561E97DE082E00E94E93581E01B
:100BF0008093B7018091790D813061F480917A0DF5
:100C000090917B0D6AE070E00E940C667093770D06
:100C10006093760D8091200E813061F48091210ED9
:100C20009091220E6AE070E00E940C667093720D43
:100C30006093710D8091D80D813061F48091D90D50
:100C40009091DA0D6AE070E00E940C667093750D69
:100C50006093740D8091920D813061F48091930DB9
:100C60009091940D6AE070E00E940C6670931E0EE5
:100C700060931D0E0895CF93DF93CDB7DEB7CE55A9
:100C8000D0400FB6F894DEBF0FBECDBF19828CE006
:100C9000888F84E690E09B838A831D821C821E825B
:100CA0001F82188619861A861B8689819E01245FF9
:100CB0003F4FF901E80FF11D10828F5F8C30C8F3B0
:100CC000CE0101960E949C35A895198E1A8E84E655
:100CD00090E09C8F8B8F1E8E1D8E898D9E012F5FC5
:100CE0003F4FF901E80FF11D168E8F5F8232C8F376
:100CF000CE0149960E94BC35A89581E0898F1A8E55
:100D000084E690E09C8F8B8F1E8E1D8E8A8D9E01B7
:100D10002F5F3F4FF901E80FF11D168E8F5F823272
:100D2000C8F3CE0149960E94BC35A89582E0898F10
:100D30001A8E84E690E09C8F8B8F1E8E1D8E8A8D7E
:100D40009E012F5F3F4FF901E80FF11D168E8F5F57
:100D50008034C8F3CE0149960E94BC35C25ADF4F99
:100D60000FB6F894DEBF0FBECDBFDF91CF910895CF
:100D700099278832910509F440C08932910594F48D
:100D80008532910559F18632910534F4833291050B
:100D9000D9F08497F1F04FC08632910521F1879701
:100DA00039F149C08B329105B9F18C32910534F497
:100DB0008932910539F18A9751F13DC08C32910504
:100DC00081F18D9799F137C080EC0E94BC4499273E
:100DD000089581EC0E94BC449927089582EC0E94FA
:100DE000BC449927089581ED0E94BC449927089539
:100DF00084EC0E94BC449927089585EC0E94BC4471
:100E00009927089586EC0E94BC449927089587ECA1
:100E10000E94BC449927089583EC0E94BC44992702
:100E2000089582ED0E94BC449927089583ED0E94A5
:100E3000BC449927089580E090E00895EF92FF92D6
:100E40000F931F93CF93DF93CDB7DEB765970FB6A0
:100E5000F894DEBF0FBECDBF80916F0E9091700EE3
:100E600001978F5F974008F029C490916E0E9923E7
:100E700009F424C48091730D8F5F8093730D8917DB
:100E800008F41CC41092730D88E08D8300E0CE013D
:100E90000696FC01E00FF11D10820F5F0830C8F3C9
:100EA0008091780D99278530910509F4BDC286306F
:100EB00091059CF48230910509F408C283309105B4
:100EC00024F4019709F4C8C11EC08330910509F4C8
:100ED00037C2049709F46EC216C08830910509F430
:100EE00060C38930910544F48630910509F4D1C27C
:100EF000079709F403C307C08930910509F481C33A
:100F00000A9709F4B7C380916F0E9091700EAA27CB
:100F1000BB2789839A83AB83BC8301E00093780D60
:100F200010E080EC0E94BC448111102F81EC0E94E3
:100F3000BC448111126082EC0E94BC448111146097
:100F400081ED0E94BC448111186084EC0E94BC4475
:100F50008111106185EC0E94BC448111106286EC05
:100F60000E94BC448111106487EC0E94BC44811132
:100F700010681E8310E083EC0E94BC44811111E0D4
:100F800082ED0E94BC448111126083ED0E94BC443A
:100F9000811114601F8310E081E090E00E94D5571A
:100FA000892B09F011E082E090E00E94D557892B4F
:100FB00009F0126083E090E00E94D557892B09F078
:100FC000146084E090E00E94D557892B09F01860E6
:100FD00085E090E00E94D557892B09F0106186E0EA
:100FE00090E00E94D557892B09F0106287E090E0CD
:100FF0000E94D557892B09F0106488E090E00E9488
:10100000D557892B09F01068188710E089E090E027
:101010000E94D557892B09F011E08AE090E00E94E8
:10102000D557892B09F012608BE090E00E94D557CC
:10103000892B09F014608CE090E00E94D557892B31
:1010400009F018608DE090E00E94D557892B09F0D7
:1010500010618EE090E00E94D557892B09F0106254
:101060008FE090E00E94D557892B09F0106480E151
:1010700090E00E94D557892B09F01068198710E07D
:1010800081E090E00E944B11892B09F011E082E091
:1010900090E00E944B11892B09F0126083E090E0F0
:1010A0000E944B11892B09F0146084E090E00E94AB
:1010B0004B11892B09F0186085E090E00E944B11DC
:1010C000892B09F0106186E090E00E944B11892B7A
:1010D00009F0106287E090E00E944B11892B09F023
:1010E000106488E090E00E944B11892B09F0106891
:1010F0001A8710E089E090E00E944B11892B09F0DB
:1011000011E08AE090E00E944B11892B09F01260F7
:101110008BE090E00E944B11892B09F014608CE069
:1011200090E00E944B11892B09F018608DE090E04F
:101130000E944B11892B09F010618EE090E00E9413
:101140004B11892B09F010628FE090E00E944B1147
:10115000892B09F0106480E190E00E944B11892BEB
:1011600009F010681B8710E081E190E00E944B11AC
:10117000892B09F011E082E190E00E944B11892B4C
:1011800009F0126083E190E00E944B11892B09F075
:10119000146084E190E00E944B11892B09F01860E3
:1011A00085E190E00E944B11892B09F0106186E1E6
:1011B00090E00E944B11892B09F0106287E190E0CA
:1011C0000E944B11892B09F0106488E190E00E9485
:1011D0004B11892B09F010681C8710E089E190E021
:1011E0000E944B11892B09F011E08AE190E00E94E6
:1011F0004B11892B09F012608BE190E00E944B119A
:10120000892B09F014608CE190E00E944B11892B2E
:1012100009F018608DE190E00E944B11892B09F0D4
:1012200010618EE190E00E944B11892B09F0106251
:101230008FE190E00E944B11892B09F0106480E24D
:1012400090E00E944B11892B09F010681D87CE0198
:1012500001960E944B4232C280916F0E9091700EA7
:101260000196AA27BB2789839A83AB83BC8382E03C
:101270008093780D00E00F2EF6E0EF2EFF24F02D86
:10128000EC0EFD1E802F8F5F0E94752CDC01FC018F
:10129000878580FF02C014E60DC0FD01878583FFAE
:1012A00002C015E607C0FD018181803F11F411E005
:1012B00001C010E0F701E00FF11D10830F5F08304F
:1012C00008F3CE0101960E944B42F8C180916F0E47
:1012D0009091700E0296AA27BB2789839A83AB83CD
:1012E000BC8383E08093780D00E00F2EF6E0EF2EB4
:1012F000FF24F02DEC0EFD1E802F875F0E94752CC1
:10130000DC01FC01878580FF02C014E60DC0FD01F1
:10131000878583FF02C015E607C0FD018181803FFC
:1013200011F411E001C010E0F701E00FF11D10838E
:101330000F5F083008F3CE0101960E944B42BEC1F8
:1013400080916F0E9091700E0396AA27BB27898318
:101350009A83AB83BC8384E08093780D00E00F2EEA
:10136000F6E0EF2EFF24F02DEC0EFD1E802F8F5E99
:101370000E94752CDC01FC01878580FF02C014E609
:101380000DC0FD01878583FF02C015E607C0FD0182
:101390008181803F11F411E001C010E0F701E00FFE
:1013A000F11D10830F5F083008F3CE0101960E94F3
:1013B0004B4284C180916F0E9091700E0496AA27C3
:1013C000BB2789839A83AB83BC8385E08093780DA8
:1013D00000E00F2EF6E0EF2EFF24F02DEC0EFD1EA8
:1013E000802F875E0E94752CDC01FC01878580FFC1
:1013F00002C014E60DC0FD01878583FF02C015E61B
:1014000007C0FD018181803F11F411E001C010E0AF
:10141000F701E00FF11D10830F5F083008F3CE01D4
:1014200001960E944B424AC180916F0E9091700EBE
:101430000596AA27BB2789839A83AB83BC8386E062
:101440008093780D00E00F2EF6E0EF2EFF24F02DB4
:10145000EC0EFD1E802F8F5F0E94752CFC01818198
:10146000803F59F49701200F311D808991890196A1
:1014700096958795F901808304C0F701E00FF11D6F
:1014800010820F5F083030F3CE0101960E944B426C
:1014900015C180916F0E9091700E0696AA27BB27FA
:1014A00089839A83AB83BC8387E08093780D00E0C7
:1014B0000F2EF6E0EF2EFF24F02DEC0EFD1E802FF8
:1014C000875F0E94752CFC018181803F59F4970150
:1014D000200F311D80899189019696958795F90194
:1014E000808304C0F701E00FF11D10820F5F083008
:1014F00030F3CE0101960E944B42E0C080916F0E06
:101500009091700E0796AA27BB2789839A83AB8395
:10151000BC8388E08093780D00E00F2EF6E0EF2E7C
:10152000FF24F02DEC0EFD1E802F8F5E0E94752C87
:10153000FC018181803F59F49701200F311D808982
:101540009189019696958795F901808304C0F701EA
:10155000E00FF11D10820F5F023030F30830E0F42D
:101560000F2EF6E0EF2EFF24F02DEC0EFD1E1FE0F7
:10157000802F8F5E0E94752CFC018181803F29F4B1
:10158000F701E00FF11D108304C0F701E00FF11D1A
:1015900010820F5F083060F3CE0101960E944B422B
:1015A0008DC080916F0E9091700E0896AA27BB2770
:1015B00089839A83AB83BC8389E08093780D00E0B4
:1015C0000F2EF6E0EF2EFF24F02DEC0EFD1E1FE097
:1015D000802F875E0E94752CFC018181803F29F459
:1015E000F701E00FF11D108304C0F701E00FF11DBA
:1015F00010820F5F083060F3CE0101960E944B42CB
:101600005DC080916F0E9091700E0996AA27BB273E
:1016100089839A83AB83BC838AE08093780DCE0163
:101620000E960E945B2C8889282F3327C901880FCA
:10163000991F880F991F880F991F820F931F280FDA
:10164000391F832F99278E832F838989282F33274A
:1016500084E690E0289FA001299F500D389F500DEF
:101660001124852F992788874987CE0101960E94EA
:101670004B4224C080916F0E9091700E0A96AA275B
:10168000BB2789839A83AB83BC831092780DCE01EC
:101690000E960E945B2C1E821F82188619868E85EC
:1016A0009F859C012F5F3F4F36952795832F992764
:1016B0008A872B87CE0101960E944B428091760D3E
:1016C0009091770D009709F479C001979093770D69
:1016D0008093760D892B09F071C080917A0D9091DD
:1016E0007B0D6AE070E00E940C667093770D60934A
:1016F000760D80917C0D90917D0DAA27BB27898363
:101700009A83AB83BC8388E08D838091B7018E83FD
:1017100080917E0D0E94FF2C9695879596958795D2
:101720008F8380917F0D0E94FF2C969587959695CB
:10173000879588878091800D0E94FF2C96958795CC
:101740009695879589878091810D0E94FF2C9695AB
:101750008795969587958A878091820D0E94FF2CA8
:1017600096958795969587958B878091830D0E9496
:10177000FF2C96958795969587958C872091B70134
:1017800089E79DE0FC01E20FF11D82850E94FF2C9C
:1017900096958795969587958D878091B701982F17
:1017A0009F5F9093B7018091900D891718F481E0A5
:1017B0008093B701CE0101960E944B428091710D3A
:1017C0009091720D009709F405C101979093720DE5
:1017D0008093710D892B09F0FDC0CE010E960E94F9
:1017E0005B2C8091210E9091220E6AE070E00E94A5
:1017F0000C667093720D6093710D8091230E909121
:10180000240EAA27BB2789839A83AB83BC8388E0F5
:101810008D83EE240F2EF0E8FF2EF02D0E2D802F5D
:101820009927FC01E15EF14F1681133238F4812FC4
:101830000E94152C882379F0EF280DC01E3238F451
:10184000812F0E94B806882331F0EF2804C01E3291
:1018500011F4A499EF28F6940F5F083000F3EE829C
:10186000EE240F2EF0E8FF2EF02D0E2D802F99275D
:10187000FC01E15EF14F1685133238F4812F0E948E
:10188000152C882379F0EF280DC01E3238F4812FF3
:101890000E94B806882331F0EF2804C01E3211F4EC
:1018A000A499EF28F6940F5F083000F3EF82EE243E
:1018B0000F2EF0E8FF2EF02D0E2D802F9927FC0122
:1018C000E15EF14F1689133238F4812F0E94152CF6
:1018D000882379F0EF280DC01E3238F4812F0E9442
:1018E000B806882331F0EF2804C01E3211F4A49901
:1018F000EF28F6940F5F083000F3E886EE240F2EF1
:10190000F0E8FF2EF02D0E2D802F9927FC01E15ECF
:10191000F14F168D133238F4812F0E94152C882335
:1019200079F0EF280DC01E3238F4812F0E94B806DE
:10193000882331F0EF2804C01E3211F4A499EF2857
:10194000F6940F5F083000F3E986EE241091450EFF
:10195000133250F4812F0E94152C882399F00F2EFA
:10196000F0E8EF2EF02D0EC01E3240F4812F0E94C1
:10197000B806882339F050E8E52A04C01E3211F475
:10198000A499EF281091460E133240F4812F0E9443
:10199000152C882389F080E4E82A0EC01E3240F41A
:1019A000812F0E94B806882339F0E0E4EE2A04C0B3
:1019B0001E3211F4A499EF28EA868E859F856AE08D
:1019C00070E00E940C666B871C861D86CE01019616
:1019D0000E944B428091740D9091750D009709F40F
:1019E000FCC001979093750D8093740D892B09F0BD
:1019F000F4C08091D90D9091DA0D6AE070E00E94F8
:101A00000C667093750D6093740D8091DB0D909151
:101A1000DC0DAA27BB2789839A83AB83BC8388E02C
:101A20008D83EE240F2EF0E8FF2EF02D0E2D802F4B
:101A30009927FC01E952F24F1681133238F4812FB5
:101A40000E943B2C882379F0EF280DC01E3238F419
:101A5000812F0E94B806882331F0EF2804C01E327F
:101A600011F4A499EF28F6940F5F083000F3EE828A
:101A7000EE240F2EF0E8FF2EF02D0E2D802F99274B
:101A8000FC01E952F24F1685133238F4812F0E947F
:101A90003B2C882379F0EF280DC01E3238F4812FBB
:101AA0000E94B806882331F0EF2804C01E3211F4DA
:101AB000A499EF28F6940F5F083000F3EF82EE242C
:101AC0000F2EF0E8FF2EF02D0E2D802F9927FC0110
:101AD000E952F24F1689133238F4812F0E943B2CC1
:101AE000882379F0EF280DC01E3238F4812F0E9430
:101AF000B806882331F0EF2804C01E3211F4A499EF
:101B0000EF28F6940F5F083000F3E886EE240F2EDE
:101B1000F0E8FF2EF02D0E2D802F9927FC01E952C1
:101B2000F24F168D133238F4812F0E943B2C8823FC
:101B300079F0EF280DC01E3238F4812F0E94B806CC
:101B4000882331F0EF2804C01E3211F4A499EF2845
:101B5000F6940F5F083000F3E986EE241091FD0D36
:101B6000133250F4812F0E943B2C882399F00F2EC2
:101B7000F0E8EF2EF02D0EC01E3240F4812F0E94AF
:101B8000B806882339F0F0E8EF2A04C01E3211F4B9
:101B9000A499EF281091FE0D133240F4812F0E947A
:101BA0003B2C882389F020E4E22A0EC01E3240F448
:101BB000812F0E94B806882339F040E4E42A04C04B
:101BC0001E3211F4A499EF28EA8688898B871C8637
:101BD0001D86CE0101960E944B4280911D0E909170
:101BE0001E0E009709F45CC1019790931E0E80931E
:101BF0001D0E892B09F054C18091930D9091940D85
:101C00006AE070E00E940C6670931E0E60931D0ED9
:101C10008091950D9091960DAA27BB2789839A8371
:101C2000AB83BC8388E08D83EE240F2EF0E8FF2E7B
:101C3000F02D0E2D802F9927FC01EF56F24F1681C3
:101C4000133238F4812F0E94152C882379F0EF2865
:101C50000DC01E3238F4812F0E94B806882331F05F
:101C6000EF2804C01E3211F4A499EF28F6940F5FF8
:101C7000083000F3EE82EE240F2EF0E8FF2EF02D58
:101C80000E2D802F9927FC01EF56F24F1685133247
:101C900038F4812F0E94152C882379F0EF280DC08D
:101CA0001E3238F4812F0E94B806882331F0EF28C5
:101CB00004C01E3211F4A499EF28F6940F5F083087
:101CC00000F3EF82EE240F2EF0E8FF2EF02D0E2D04
:101CD000802F9927FC01EF56F24F1689133238F402
:101CE000812F0E94152C882379F0EF280DC01E3219
:101CF00038F4812F0E94B806882331F0EF2804C001
:101D00001E3211F4A499EF28F6940F5F083000F307
:101D1000E886EE240F2EF0E8FF2EF02D0E2D802FFA
:101D20009927FC01EF56F24F168D133238F4812FAC
:101D30000E94152C882379F0EF280DC01E3238F44C
:101D4000812F0E94B806882331F0EF2804C01E328C
:101D500011F4A499EF28F6940F5F083000F3E98698
:101D6000EE240F2EF0E8FF2EF02D0E2D802F992758
:101D7000FC01EF56F24F16A1133238F4812F0E9466
:101D80003B2C882379F0EF280DC01E3238F4812FC8
:101D90000E94B806882331F0EF2804C01E3211F4E7
:101DA000A499EF28F6940F5F083000F3EA86EE243A
:101DB0000F2EF0E8FF2EF02D0E2D802F9927FC011D
:101DC000EF56F24F16A5133238F4812F0E943B2CA8
:101DD000882379F0EF280DC01E3238F4812F0E943D
:101DE000B806882331F0EF2804C01E3211F4A499FC
:101DF000EF28F6940F5F083000F3EB86EE240F2EE9
:101E0000F0E8FF2EF02D0E2D802F9927FC01EF56C4
:101E1000F24F16A9133238F4812F0E943B2C8823ED
:101E200079F0EF280DC01E3238F4812F0E94B806D9
:101E3000882331F0EF2804C01E3211F4A499EF2852
:101E4000F6940F5F083000F3EC86EE240F2EF0E8D6
:101E5000FF2EF02D0E2D802F9927FC01E153F24F1C
:101E60001081133238F4812F0E943B2C882379F0A3
:101E7000EF280DC01E3238F4812F0E94B806882347
:101E800031F0EF2804C01E3211F4A499EF28F69423
:101E90000F5F083000F3ED86CE0101960E944B42A1
:101EA00065960FB6F894DEBF0FBECDBFDF91CF9120
:101EB0001F910F91FF90EF9008958091650E909182
:101EC000660E885E934031F084EF91E09093660E49
:101ED0008093650E2FE030E03093680E2093670EFC
:101EE00089E999E090936A0E8093690E10926B0EC7
:101EF00010926C0E10926D0E10926E0E1092700E6B
:101F000010926F0EE5E6FEE0A0E7B0E02115310586
:101F100051F081E02030380719F40E94C06608951E
:101F2000122E0E94C0660895BF92CF92DF92EF9268
:101F3000FF920F931F93CF93DF93CDB7DEB7AE978A
:101F40000FB6F894DEBF0FBECDBFBB24BE016F5FDE
:101F50007F4F8B2D0E94D2338B2D99279C01229588
:101F60003295307F3227207F3227B90169537E4F67
:101F70009981492F4170DB018C91887F9670842B69
:101F8000892B8C930F2EF8EBCF2EF1E0DF2EF02D66
:101F9000C20ED31E8A819B81F601918380838C813E
:101FA0009D81938382834E815F815583448388859D
:101FB000998597838683D901A054BE4F2A858B8546
:101FC000982F9295907F822F8F70892B8C938C8580
:101FD00081878D8582878E8583878F8584878F8D86
:101FE0008170982F990F990F990FFB018081877F3E
:101FF000892B808388A1F601858789A186878AA19C
:102000008170982F9295907FFB0180818F7E892B24
:1020100080838C918F70833090F5CA01AA2797FD39
:10202000A095BA2FBC01CD010E942463DC01CB0135
:1020300028A539A54AA55BA5BC01CD010E943E6239
:102040007B018C018CA5992787FD9095A92FB92F2D
:10205000BC01CD010E942463DC01CB019C01AD01D8
:10206000C801B7010E940962DC01CB01BC01CD01AE
:102070000E948A60DC01CB01F601958384838B2D5D
:1020800099279C0122953295307F3227207F322775
:10209000F901E054FE4F808182958F708330D8F52E
:1020A0000F2EF8EBCF2EF1E0DF2EF02DC20ED31E57
:1020B00088859985AA2797FDA095BA2FBC01CD01E7
:1020C0000E942463DC01CB0128A539A54AA55BA5A4
:1020D000BC01CD010E943E627B018C018CA5992739
:1020E00087FD9095A92FB92FBC01CD010E942463D3
:1020F000DC01CB019C01AD01C801B7010E9409625E
:10210000DC01CB01BC01CD010E948A60DC01CB0166
:10211000F601978386832B2D3327C90182959295EB
:10212000907F9827807F9827FC01E953FE4F80819C
:1021300086958370813029F4F901E854FC4F80833F
:1021400006C08B2D9927FC01E854FC4F10828B2D83
:102150009927880F991FFC01E951FC4F11821082C9
:10216000B394FFE1FB1508F0F1CEFE01BD96AAEE97
:10217000B8E082E090E021E08030920719F40E94FC
:10218000AF6603C0182E0E94AF668DA58093E5034D
:102190008EA58093E6031092D9031092D803AE96D1
:1021A0000FB6F894DEBF0FBECDBFDF91CF911F9168
:1021B0000F91FF90EF90DF90CF90BF9008951F9305
:1021C000CF93DF93CDB7DEB7AE970FB6F894DEBFEF
:1021D0000FBECDBF10E0A8958981887F89831B82BF
:1021E0001A821D821C821F821E82198618861A86F8
:1021F0001B861C8681E08D871E868F871F8E18A206
:1022000019A21AA280E090E0A0E8BFE388A799A7EE
:10221000AAA7BBA71CA685E0FE01B39611928A95DA
:10222000E9F78FE0FE017096DF01282F1D922A95B5
:10223000E9F7189FC001112486559E4FBC01CF01BC
:102240000E94AF65BE016F5F7F4F812F0E949A335E
:102250001F5F103208F4BFCF1EA61DA6FE01BD965B
:10226000AAEEB8E082E090E021E08030920719F415
:102270000E94C06603C0182E0E94C066AE960FB6BC
:10228000F894DEBF0FBECDBFDF91CF911F910895AF
:102290008093D80308950F93CF93DF93CDB7DEB724
:1022A00021970FB6F894DEBF0FBECDBF8983815052
:1022B000803270F000E021E0AE014F5F5F4F69E0D7
:1022C00071E081E091E00E949D2F80E090E007C0E6
:1022D00089819927FC01E954FC4F80819927219637
:1022E0000FB6F894DEBF0FBECDBFDF91CF910F9137
:1022F00008958091E503882381F08091E6030E9490
:10230000BC44882351F4482F88EB93E0FC01E40F90
:10231000F11D10824F5F4032C8F340E067EE73E07A
:10232000A8EBB3E051E0242F3327C901820F931F9C
:10233000FC01E60FF71F80819181009709F1019759
:1023400091838083892BE1F4C90182959295907FD6
:102350009827807F9827FC01E953FE4F808186955E
:10236000837099278130910539F0029749F0F9017E
:10237000EA0FFB1F108204C0FD01E40FF11D508322
:102380004F5F403280F208958091D803882399F0FE
:102390008091D903882379F089ED93E0AC014C5FFB
:1023A0005F4F6091DC038091DA039091DB030E9420
:1023B0004D521092D90308958F929F92AF92BF927F
:1023C000CF92DF92EF92FF920F931F93CF93DF9301
:1023D0008C01EE24FF2499248091E503882339F0B1
:1023E0008091E6030E94BC44882309F432C28091A4
:1023F000690E90916A0E9C0144275527F80180814F
:102400009181A281B38182179307A407B50799F43C
:1024100080916B0EE80FF11D858190916C0E8923E0
:10242000891749F40E94E6530E947B2110928B0E7B
:1024300082E28093110160E07091D8030F2EF8EBD7
:10244000AF2EF3E0BF2EF02D88248394C090670E4A
:10245000D090680E862F992782959295907F982725
:10246000807F9827EC01C854DE4F88819981AA2784
:1024700097FDA095BA2FF8012081318142815381C7
:1024800082179307A407B50759F08A819B81AA2771
:1024900097FDA095BA2F82179307A407B507C1F43B
:1024A000462F5527CA01840F951FFC01E951FC4FA7
:1024B000D182C082872F733048F099279C012F73F7
:1024C0003070CA0103962817390711F499249394A0
:1024D0008F8583FF09C08D85F801E80FF11D9E856A
:1024E0008581981709F062C128813981211531054C
:1024F00009F45CC1442737FD4095542FF8018081D1
:102500009181A281B381281739074A075B0709F037
:102510009DC091E08985882379F0E80FF11D8481C1
:10252000E82EFF24FE2CEE248A85F801E80FF11D29
:102530008481E80EF11C14C08A85882381F0F8019B
:10254000E80FF11D8481E82EFF248F8584FF08C0E9
:10255000EE2034F420E03FEFE22AF32A01C090E0BD
:10256000992309F473C088858F709927823091056B
:10257000B9F1833091052CF4009779F00197C1F0FF
:1025800065C08430910509F44DC0843091050CF488
:102590003EC0059709F451C059C08C819D818E15AC
:1025A0009F0509F053C0F501E60FF11D80824EC072
:1025B0008F8584FF0BC08C819D818E159F050CF04B
:1025C00045C0F501E60FF11D808240C08C819D81E0
:1025D0008E159F05D8F5F501E60FF11D808236C0F6
:1025E0008F8584FF0AC08C819D81E816F90674F5F9
:1025F000F501E60FF11D808229C08C819D81E816CE
:10260000F90620F5F501E60FF11D80821FC08C81CF
:102610009D818E219F21892BC9F0F501E60FF11DC7
:10262000808214C08C819D818E219F21892B71F421
:10263000F501E60FF11D808209C08C819D818E1508
:102640009F0521F0F501E60FF11D80828A819B81B3
:102650009C01442737FD4095542FF80180819181DA
:10266000A281B381281739074A075B0709F09EC08A
:1026700091E08B85882379F0E80FF11D8481E82EA5
:10268000FF24FE2CEE248C85F801E80FF11D8481D7
:10269000E80EF11C14C08C85882381F0F801E80F46
:1026A000F11D8481E82EFF248F8584FF08C0EE2071
:1026B00034F420E03FEFE22AF32A01C090E09923AE
:1026C00009F474C0888582958F70992782309105AE
:1026D000B9F1833091052CF4009779F00197C1F09E
:1026E00065C08430910509F44DC0843091050CF427
:1026F0003EC0059709F451C059C08E819F818E1547
:102700009F0509F053C0F501E60FF11D10824EC080
:102710008F8584FF0BC08E819F818E159F050CF0E5
:1027200045C0F501E60FF11D108240C08E819F81EA
:102730008E159F05D8F5F501E60FF11D108236C004
:102740008F8584FF0AC08E819F81E816F90674F593
:10275000F501E60FF11D108229C08E819F81E816D8
:10276000F90620F5F501E60FF11D10821FC08E81DC
:102770009F818E219F21892BC9F0F501E60FF11D64
:10278000108214C08E819F818E219F21892B71F42C
:10279000F501E60FF11D108209C08E819F818E1513
:1027A0009F0521F0F501E60FF11D10826F5F603289
:1027B00008F450CE8091D803882309F44AC09920A8
:1027C00019F4823009F045C08091D903823009F4B0
:1027D00040C08091DA039091DB039C014427552788
:1027E000F80180819181A281B381281739074A07B6
:1027F0005B0799F49091DC038481981771F4892F19
:10280000992798012B5F3F4FAC01B90189ED93E007
:1028100004960E94B665892BC9F082E08093D903A3
:10282000F80124812093DC03808191819093DB0364
:102830008093DA03822F992798012B5F3F4FAC01D9
:10284000B9018DED93E00E94C36503C081E08093E0
:10285000D903DF91CF911F910F91FF90EF90DF90FF
:10286000CF90BF90AF909F908F9008950E94730576
:102870008091D80082608093D8000895CF93DF9331
:10288000EC018981833089F48985882309F403C1A7
:1028900088818295807F8093ED008091EF008F7317
:1028A0008093EF0018821986F6C00E949705982F32
:1028B00081E089879F3F09F4EBC09883892F829537
:1028C000807F8093ED001092EE001092EF00109246
:1028D000F7001092F6001092F5001092F40010929A
:1028E000F000898199278130910509F46BC082300D
:1028F00091051CF4892B29F0C9C0029709F4BBC0CB
:10290000C5C08A8581FF30C08D81982F990F990F9E
:10291000990F8C81829586958770890F8093F3003B
:102920008C81982F990F990F990F8B81829586959D
:102930008770890F8093F2008B81982F990F990FE0
:10294000990F8A81829586958770890F8093F1000F
:102950008A81880F880F880F8093F0008091EF00A4
:1029600080618093EF0012C08B81982F9295990F10
:10297000907E8A81869586958695890F8093F3004F
:102980008A818295880F807E8093F20020E08E817C
:10299000181660F48F819885FC01E20FF11D80818B
:1029A0008093FA002F5F8E812817A0F39091EF009B
:1029B0008E81892B8093EF008091EF00806480935B
:1029C000EF0069C08A8581FF35C08D81982F990FEE
:1029D000990F990F8C81829586958770890F8093C6
:1029E000F3008C81982F990F990F990F8B81829505
:1029F00086958770890F8093F2008B81982F990FAD
:102A0000990F990F8A81829586958770890F809397
:102A1000F1008A81880F880F880F8093F0008091E1
:102A2000EF0080618093EF008091F00084608093DC
:102A3000F00015C08B81982F9295990F907E8A8116
:102A4000869586958695890F8093F3008A81829575
:102A5000880F807E8093F20084E08093F000909154
:102A6000EF008E81892B8093EF008091EF008064CE
:102A70008093EF0010C08091EF008F738093EF0080
:102A80008091EF0080688093EF0005C0198603C035
:102A90008FEF90E002C080E090E0DF91CF91089549
:102AA000CF93DF93EC018985882319F482E090E0CD
:102AB00082C088818295807F8093ED000E94B1055D
:102AC000813009F06CC019868091EF008F708E8381
:102AD0008F8198850E94C9058091F00099278470A4
:102AE00090709595879595958795982F91708A8583
:102AF000282F2E7F292B2A878091EF0084FF31C059
:102B0000822F82608A878091F300869586958695CC
:102B10008D838091F200982F969596959695809149
:102B2000F3008295880F807E890F8C838091F1005D
:102B3000982F9695969596958091F2008295880F9C
:102B4000807E890F8B838091F000982F96959695C3
:102B500096958091F1008295880F807E890F8A83F7
:102B600016C08A858D7F8A878091F300829586952D
:102B700087708B838091F200982F9295969597702D
:102B80008091F300880F880F880F890F8A838091C6
:102B9000EF008F738093EF0080E090E00CC08823FB
:102BA00049F489878091EF008F738093EF0080E074
:102BB00090E001C09927DF91CF910895982F8F3F22
:102BC00019F481E090E00895805C843128F4892F25
:102BD0000E94BC4499270895892F8150803228F49F
:102BE000892F0E944B1199270895892F8152843192
:102BF00028F4892F0E942E589927089580E090E0AC
:102C00000895982F8F3F19F481E090E00895805C3B
:102C1000843128F4892F0E949B4399270895892F96
:102C20008150803228F4892F0E944B1199270895F2
:102C3000892F8152843128F4892F0E942E58992798
:102C4000089580E090E008958091810E9091820E29
:102C500001969093820E8093810E8091760E9091D2
:102C6000770E01969093770E8093760E8091750E75
:102C7000833008F46DC08F5F8093750E843031F41B
:102C800040E061E486E00E949F3C62C08091810E3A
:102C90009091820E8035910598F48091750E853063
:102CA00031F440E061E486E00E94EA3C51C080914A
:102CB000750E883009F04CC083E08093750E48C0D3
:102CC0008091810E9091820E803A910590F48091CE
:102CD000750E853031F440E061E486E00E94EA3C04
:102CE00037C08091750E873098F183E08093750E20
:102CF0002FC08091810E9091820E8856914088F469
:102D00008091750E863029F440E061E40E94EA3C2F
:102D10001FC08091750E8730D8F083E08093750EC8
:102D200017C08091810E9091820E8E5F914068F461
:102D30008091750E873060F040E061E486E00E948B
:102D4000EA3C83E08093750E03C081E08093750EAA
:102D50008091780E833008F46DC08F5F8093780E79
:102D6000843031F441E061E486E00E949F3C0895A4
:102D70008091760E9091770E8035910598F4809130
:102D8000780E853031F441E061E486E00E94EA3C4F
:102D900008958091780E883009F04CC083E08093CC
:102DA000780E08958091760E9091770E803A910575
:102DB00090F48091780E853031F441E061E486E052
:102DC0000E94EA3C08958091780E873098F183E064
:102DD0008093780E08958091760E9091770E8856A4
:102DE000914088F48091780E863029F441E061E4C6
:102DF0000E94EA3C08958091780E8730D8F083E0F5
:102E00008093780E08958091760E9091770E8E5F64
:102E1000914068F48091780E873060F041E061E481
:102E200086E00E94EA3C83E08093780E089581E07A
:102E30008093780E089580917A0E0E94DE15882383
:102E400021F085E08093E00946C080917F0E0E94CA
:102E5000DE15882341F08091800E8093E30983E0A2
:102E60008093E00938C08091790E0E94DE15882396
:102E700021F084E08093E0092EC080917B0E0E94B7
:102E8000DE15882369F08091E009873049F08630AB
:102E900039F086E08093E0098AE08093E2091BC064
:102EA0008091E009853021F482E08093E00913C02D
:102EB0008091E009833041F48091E309882321F473
:102EC00081E08093E00907C08091E009843019F423
:102ED00081E08093E0098091E0098150823058F4CC
:102EE00080917C0E0E94011690917D0E981719F426
:102EF0001092E00917C08091E209882399F480912B
:102F0000E009863079F480917C0E0E940116909140
:102F10007D0E981739F487E08093E00980917E0E4A
:102F20008093E1098BE599E00E94F52D0E945519E7
:102F300008951F93CF93DF9310E0812F9927EC0121
:102F4000C80FD91FFE01ED57F14F8081882309F486
:102F5000B4C00E94DE15882309F4AFC0FE01EC570F
:102F6000F14F808183FDB3C088608083877099278B
:102F70008230910539F1833091051CF4019729F0D5
:102F8000A6C0039709F452C0A2C0812F9927880FC9
:102F9000991FFC01EC57F14F9081892F82958F701A
:102FA000877021F0892F8F78808391C0812F992796
:102FB000880F991FFC01EC57F14F80818F78806159
:102FC000808385C0812F9927880F991FFC01EC57BA
:102FD000F14F808182958F7087709927009719F043
:102FE000019769F018C0812F9927880F991FFC015C
:102FF000EC57F14F80818F788061808368C0812F8A
:103000009927880F991FFC01EC57F14F80818F7829
:10301000806280835CC0812F9927880F991FFC01F3
:10302000EC57F14F80818F78808351C0812F992791
:10303000880F991FFC01EC57F14F808182958F70AA
:103040008770992781309105A9F0823091051CF491
:10305000892B21F027C00297C9F024C0812F99271E
:10306000880F991FFC01EC57F14F80818F788061A8
:1030700080832DC0812F9927880F991FFC01EC5761
:10308000F14F80818F788062808321C0812F9927C2
:10309000880F991FFC01EC57F14F80818F78806376
:1030A000808315C0812F9927880F991FFC01EC5749
:1030B000F14F80818F7880830AC0812F9927880FF4
:1030C000991FFC01EC57F14F8081877F80831F5F40
:1030D000143008F432CF0E944F220E94E4200E9454
:1030E000CA2310E085E2189FC0011124EC01C25DE3
:1030F000DB4F8C899D89009719F001979D8B8C8BF4
:103100008D859E85009761F001979E878D879985B3
:103110009F3F31F085E0989FC00111249B878A87EB
:103120002A853B852115310561F089858F3F49F05E
:10313000C90101979B878A87892B19F48F85806243
:103140008F878A8D9B8D009779F001979B8F8A8F4F
:10315000892B51F48F8586FD04C0812F8F5F0E94DB
:103160007B328F8580648F878F81882311F0815017
:103170008F831F5F123208F4B5CFDF91CF911F917B
:1031800008958091E209882319F081508093E20923
:103190008091E0098730B9F48091E109882321F01A
:1031A00081508093E1090FC080917B0E0E94DE1553
:1031B000882339F086E08093E0098AE08093E20971
:1031C00002C01092E0098091E309882319F0815030
:1031D0008093E309A49B23C02091DD092F3710F4CD
:1031E000220F01C02FEF80916D0E8A30D0F09091A8
:1031F000740E981710F0921730F48091740E8F5F50
:103200008093740E0EC080918B0E882351F48F5FD3
:1032100080938B0E0E94E6530E947B2102C0109285
:10322000740E90915209809162099817E0F420E0A1
:1032300042E659E065E270E0FA01E20FF11D828199
:10324000823268F49927869FF001879FF00D969F40
:10325000F00D1124EE5CFB4F8081816080832F5F35
:103260002C3050F308959091520980916309891789
:10327000D8F420E042E659E065E270E0FA01E20F9E
:10328000F11D8281823268F49927869FF001879F21
:10329000F00D969FF00D1124EE5CFB4F80818E7F28
:1032A00080832F5F2C3050F30895CF92DF92EF92FE
:1032B000FF920F931F93CF93DF938091280488236D
:1032C00009F004C1F82E0F2EFAE0EF2EF02D8EE05B
:1032D000F89EC0011124EC01C956D64F00E08A8146
:1032E0008F3F11F401E01DC09A81892F805C8431E9
:1032F00028F4892F0E94BC44082F13C09A81892F7B
:103300008150803228F4892F0E944B11082F09C068
:103310009A81892F8152843120F4892F0E942E585E
:10332000082F8981992781309105C9F18230910553
:103330001CF4892B29F0C5C0029709F4BFC0C1C095
:10334000013009F0BEC08F818E9DC00111249C8385
:103350008B8389858E9DC00111249E838D838881F6
:103360008460888310E025E230E0FE01E10FF11D6A
:1033700082858F3F71F09927829FA001839F500D16
:10338000929F500D1124FA01EE5CFB4F8081846006
:1033900080831F5F143048F381E0898392C08B8162
:1033A0009C81009709F48DC001979C838B83892BA6
:1033B00081F5288122FF17C08F818E9DC0011124C5
:1033C0009C838B83822F8B7F888310E0FE01E10F2B
:1033D000F11D82858F3F19F060E00E946F1A1F5F18
:1033E0001430A0F316C088858E9DC00111249C83E3
:1033F0008B8388818460888310E0FE01E10FF11DDA
:1034000082858F3F19F061E00E946F1A1F5F1430B0
:10341000A0F38881282F227081FD28C08D819E8194
:10342000009709F44EC001979E838D83892B09F084
:1034300048C082E08983122F25E230E0FE01E10FCF
:10344000F11D82858F3F71F09927829FA001839F94
:10345000500D929F500D1124FA01EE5CFB4F8081BC
:103460008B7F80831F5F143048F32BC0002349F506
:10347000102F0F2EF5E2CF2EDD24F02DFE01E10FEF
:10348000F11D22852F3F99F0822F99278C9DA00155
:103490008D9D500D9C9D500D1124FA01EE5CFB4F4B
:1034A00080818B7F808361E0822F0E946F1A1C8253
:1034B0001B821F5F143010F3198203C0002309F42C
:1034C0000983F39454E05F1508F001CFDF91CF91A9
:1034D0001F910F91FF90EF90DF90CF900895DF92B2
:1034E000EF92FF920F931F93CF93DF93CDB7DEB789
:1034F00021970FB6F894DEBF0FBECDBF8983162F7C
:10350000DD24833260F00D2D21E0AE014F5F5F4F6F
:1035100065EE72E082E191E00E949D2F4EC099819C
:1035200085E2989F700111248EE294E0E80EF91E66
:10353000F701858D9927807F9070803A910529F455
:103540000F2EF1E4DF2EF02D18C0F701858D99279D
:10355000807F9070803B910529F40F2EF2E4DF2EDE
:10356000F02D0BC000E021E0AE014F5F5F4F61EF37
:1035700072E082E191E00E949D2F112379F483E0B3
:10358000F701878380EF818387858F7B8787858D90
:1035900041A16D2D8F700E949F3C0FC0113069F4C6
:1035A000F70117828FE08183878586798787858DEC
:1035B00041A16D2D8F700E94EA3C21960FB6F894C0
:1035C000DEBF0FBECDBFDF91CF911F910F91FF9056
:1035D000EF90DF90089520E040E759E065E270E069
:1035E0008170382F330FFA01E20FF11D8181823291
:1035F00070F49927869FF001879FF00D969FF00D3C
:103600001124EE5CFB4F80818D7F832B80832F5FA5
:103610002E3048F3089520E040E759E065E270E07D
:103620008170382F330FFA01E20FF11D8189823248
:1036300070F49927869FF001879FF00D969FF00DFB
:103640001124EE5CFB4F80818D7F832B80832F5F65
:103650002E3048F3089580912A0490912B04089508
:103660008091290499270895EF92FF921F93CF9399
:10367000DF937A01809362096093630910E0C12FA0
:10368000DD27F701EC0FFD1F80810E94822A823224
:1036900020F4FE01EE59F64F82831F5F1C3078F351
:1036A000DF91CF911F91FF90EF9008957F928F92BD
:1036B0009F92AF92BF92CF92DF92EF92FF920F93C1
:1036C0001F93CF93C0E00E94832C0E94722D0E9412
:1036D0009D2D8BE599E00E94EA2D109250091092E1
:1036E0004F09C0935109C0935309C0935409C09323
:1036F0005509C093560982E1E8E1F9E011928A95F3
:10370000E9F74AE259E028EB31E08C2F9927880F3E
:10371000991FFC01E40FF51F31832083CF5FC23175
:10372000A0F3C0E047E959E02EE030E08C2F992764
:10373000829FB001839F700D929F700D1124FB0139
:10374000E40FF51F11821482138216821582FB0189
:10375000E956F64F808184608083CF5FC53030F3B7
:103760000E942A36803221F487E68093100103C03C
:103770008EE680931001AEE2B4E041E040932E0467
:1037800028EC30E0309341042093400452EA5093F7
:103790004B0462EB60934C0410924F049FEF9093A4
:1037A0004D0450934E0483E0809350048D010B5DD3
:1037B0001F4F40935304FD0130AF27ABF801558FE5
:1037C000668F41A3978F0F2EF7EAEF2EF02DE0A220
:1037D0000F2EFFE0BF2EF02DB2A2FD01E65BFF4FE2
:1037E00040937804338B228B0F2EF3EADF2EF02DDB
:1037F000D58E83EB868F41A3978F90A389E082A318
:10380000FD01E159FF4F40939D04338B228BE58EE0
:103810000F2EF7EBCF2EF02DC68E41A3978F90A3DE
:103820008BE082A3FD01EC56FF4F4093C204338B23
:10383000228B11EA158F0F2EF1EBFF2EF02DF68E55
:1038400041A3978F90A38EE082A3FD01E754FF4F21
:103850004093E704338B228B55EA558F05EB068F97
:1038600041A3978F90A38DE082A3C6E0FD01E252B1
:10387000FF4F40930C05338B228B60EA658F70EB12
:10388000768F11A2978F50A3C2A3FD01ED5FFE4F6B
:1038900040933105338B228B558F068F11A2978F62
:1038A00090A384E082A3FD01E85DFE4F409356059E
:1038B000338B228B658F768F41A3978F60A38AE02D
:1038C00082A3FD01E35BFE4F40937B05338B228B8C
:1038D000758F54EB568F75E071A3978F90A382E19B
:1038E00082A3FD01EE58FE4F4093A005338B228B3F
:1038F00064EA658F568F41A3978FD0A288E082A398
:10390000FD01E956FE4F4093C505338B228B56EAE5
:10391000558F86EB868F11A2978F60A342A3CCE0D0
:10392000FD01E454FE4F4093EA05338B228B558F03
:10393000868F41A3978F10A3C2A3FD01EF51FE4FC5
:1039400040930F06338B228BE58EC68E11A2978F84
:1039500090A382E082A3FD01EA5FFD4F409334060D
:10396000338B228B158FF68E11A2978F90A387E051
:1039700082A3FD01E55DFD4F40935906338B228BF9
:10398000F58E068F71A3978F2B2D3327AD0185E21E
:1039900090E0289FB001299F700D389F700D112471
:1039A000FB01EA0FFB1F9FEF90A381E182A3FD01C2
:1039B000E05BFD4F61E060937E0628EC30E0338BE6
:1039C000228BB4EAB58F0F2EF4EBFF2EF02DF68E7E
:1039D00011A2978F0F2EF6EAEF2EF02DE0A285E0D0
:1039E00082A3FA01EB58FD4F6093A306338B228B21
:1039F0008D2CD58E03EB068F11A2978F90A312A268
:103A0000FA01E656FD4F70E47093C8062FEF3FEFC2
:103A1000338B228B0F2EF7EADF2EF02DD58EF68E0C
:103A200063E061A3E78E90A392A3FA01E154FD4FF6
:103A30007093ED06338B228BE58E15EB168F61A309
:103A4000E78E90A392A3FA01EC51FD4F70931207F9
:103A5000338B228BA5EAA58F0F2EF6EB7F2EF02D50
:103A6000768E61A3D78E90A392A3FA01E75FFC4FF5
:103A700070933707338B228BB58FC68E61A3D78E99
:103A800090A392A3FA01E25DFC4F70935C07338B25
:103A9000228B80EA858F068F61A3A78F90A392A3C4
:103AA000FA01ED5AFC4F70938107338B228B0F2E56
:103AB000F1EABF2EF02DB58E0F2EF2EBAF2EF02DCA
:103AC000A68E61A3A78F90A392A3FA01E858FC4F9A
:103AD0007093A607338B228B0F2EF2EA9F2EF02DC8
:103AE000958EA1EBA68F61A3B78F90A392A3FA0145
:103AF000E356FC4F7093CB07338B228B858E0F2EB2
:103B0000F0EBCF2EF02DC68E61A3B78F90A392A3BA
:103B1000FA01EE53FC4F7093F007338B228B858FA5
:103B2000068F82E081A3178F90A392A3FA01E95137
:103B3000FC4F70931508338B228BB58EA68E81A314
:103B4000178F90A392A3FA01E45FFB4F70933A089A
:103B5000338B228B958EA68F81A3F78E90A392A391
:103B6000FA01EF5CFB4F70935F08338B228B858EDD
:103B7000C68E81A3F78E90A392A3FA01EA5AFB4F57
:103B800070938408338B228BD58EF68E81A3778E2B
:103B900090A392A3FA01E558FB4F7093A908338BC9
:103BA000228BE58EFA01E558FB4F168F9A01FA0138
:103BB000E558FB4F52E051A3778E4FEF40A342A34D
:103BC000F901E056FB4FA72F7093CE086FEF7FEF00
:103BD000738B628B85EA858F768E51A397EB978FD7
:103BE00040A342A3F901EB53FB4FA093F308738B5F
:103BF000628BB58F968F51A3978F40A342A3C0E0ED
:103C0000B90145E250E02FE001E21EE130E18C2FE6
:103C10009927849FF001859FF00D949FF00D11244A
:103C2000CF01E60FF71F158A148ADC01AE5CBB4F8B
:103C30008C918C7D8C931786168A218314A213A2F3
:103C40001686158614861386128611868C918B7FB4
:103C50008C93178A17820087168335832283118EEF
:103C6000108E138E128E148ECF5FC23280F2CF91DF
:103C70001F910F91FF90EF90DF90CF90BF90AF908A
:103C80009F908F907F900895E8E1F9E082E1DF0155
:103C90001D928A95E9F7CF010E945C3520E06AE227
:103CA00079E048EB51E0822F9927880F991FFC019A
:103CB000E60FF71F518340832F5F2231A0F38AE282
:103CC00099E00E947C350895AF92BF92CF92DF9227
:103CD000EF92FF920F931F93CF93DF93CDB7DEB791
:103CE000C35CD0400FB6F894DEBF0FBECDBF10E06E
:103CF0000F2EF5E6EF2EFF24F02DEC0EFD1E212FEA
:103D0000332785E290E0289FA001299F500D389F1E
:103D1000500D11249A01225D3B4FF901828993894C
:103D2000892F9927D7018C938289F7018183F90123
:103D30008681F7018283158214821682F9018581BA
:103D4000F7018383F9018085F70187838FE0189F4E
:103D5000C001112486589B4FBC01C70108960E94E0
:103D6000AF65F701178A108E1F5F612FC7010E9490
:103D70007A34A895123218F28E0102581F4F84E649
:103D8000D8018C9388E7F80181834CE050E06FEF15
:103D900070E0C80102960E94D065C8010E94BA3244
:103DA0008E0104571F4FF80181EC81934EE050E0E3
:103DB0006FEF70E0CF010E94D065F80117868AE0AE
:103DC000808B4EE050E06FEF70E0C80141960E949A
:103DD000D065C8010E94E832A89510E00F2EF4E1EA
:103DE000DF2EF02D7E010894E11CF11C0FE0D701BD
:103DF000ED2D1D92EA95E9F7109FC00111248B5219
:103E00009C4FBC01C7010E94AF65188A1F5FB701B4
:103E1000812F0E9411351B3050F3A89510E00F2E12
:103E2000F5EBAF2EBB24F02DAC0EBD1E0F2EFFE028
:103E3000CF2EF02D0F2EFBEAEF2EFF24F02DEC0EEF
:103E4000FD1EDD24D3940FEFD501EC2D1D92EA95D4
:103E5000E9F71C9DC001112486579C4FBC01C70186
:103E60000A960E94AF65D7011C92F7011182128257
:103E7000D382D4828AE085838081F701E80FF11D27
:103E800006838F5F8430C8F3BE0165557F4F812F55
:103E90000E9428331F5F1530B8F2EFE8F9E018E010
:103EA000DF01212F1D922A95E9F7CF010E940833E7
:103EB0000E94652DA895E9E7FEE0DF011D921A95A5
:103EC000E9F781E080937D0E8EE180937E0E82E3A0
:103ED0008093800EAEE6BFE088E090E021E0803085
:103EE000920719F40E94C06603C0182E0E94C06693
:103EF0009E012B5E3F4F8CE4D9011D928A95E9F714
:103F00008CE0A0E2B1E0FE017796482F0D9001927F
:103F10004A95E1F7ACE2B1E0FE01BA96582F0D9058
:103F200001925A95E1F7A8E3B1E0FE01FD96982FC2
:103F30000D9001929A95E1F7A4E4B1E0FE01E05BF7
:103F4000FF4F0D9001928A95E1F7F901AEE8BFE0CD
:103F50008CE490E021E08030920719F40E94C06662
:103F600003C0182E0E94C06688E0E3E8FEE01192CC
:103F70008A95E9F7CD53DF4F0FB6F894DEBF0FBE39
:103F8000CDBFDF91CF911F910F91FF90EF90DF9008
:103F9000CF90BF90AF900895CF92DF92EF92FF92B3
:103FA0000F931F93CF93DF93CDB7DEB7E4970FB690
:103FB000F894DEBF0FBECDBF00E0102F1F5F612F52
:103FC000CE0101960E94BF34202F332785E290E076
:103FD000289FA001299F500D389F500D1124FA01F0
:103FE000E25DFB4F89819927982F88272A81820FCC
:103FF000911D938B828B8B818683888580878C81B2
:104000008583888D8487898D81878D819E81918F1D
:10401000808F8F81848F012F123278F282E699E0AF
:104020000E94D83280E799E00E94F83288E199E056
:104030000E946C358AE299E00E948C358FE899E005
:104040000E9418330E94652D00E0BE01665E7F4F1E
:10405000802F0E946133202F33278EE090E0289F2D
:10406000F001299FF00D389FF00D11249F01E956B2
:10407000F64F8A8D582F51708081482F4C7F8B8D41
:104080008170982F990F842F852B892B8083F901BC
:10409000E956F64F8C8D82838D8D87838E8D808738
:1040A0008F8D8187F901EF55F64F88A199A1AAA1BB
:1040B000BBA180839183A283B3830F5F053028F275
:1040C000E9E7FEE0AEE6BFE088E090E021E0803086
:1040D000920719F40E94AF6603C0182E0E94AF66C3
:1040E00000E073E142E050E0642F0F2EF3E8CF2EA2
:1040F000FEE0DF2EF02D0F2EF3E3EF2EFF24F02D48
:10410000EC0EFD1EFE01F396079FC0011124DC0199
:10411000A257B04F4115510551F081E0403058078A
:1041200019F40E94AF6603C0162E0E94AF66802F5E
:1041300099279C01280F391FF901EC0DFD1D8BA952
:104140008083D901AC57B14FF7018181982F9770C7
:104150008C918078892B8C930F5F043098F2E496D1
:104160000FB6F894DEBF0FBECDBFDF91CF911F9188
:104170000F91FF90EF90DF90CF900895CF93DF9352
:10418000EC01862F0E94822A8332D8F4282F33270D
:1041900085E290E0289FA001299F500D389F500D87
:1041A0001124FA01E25DFB4F8F898487888199276A
:1041B000982F88272981820F911D938B828B8A816A
:1041C0008683DF91CF9108951F93CF93C0E01C2F7A
:1041D00090917009892F8150803238F4892F0E9484
:1041E0004B118823B1F011E014C090917009892F10
:1041F0008152843138F4892F0E942E58882349F047
:1042000011E007C0809170090E94BC44813009F41C
:10421000182F90917F09892F8150803220F4892FA7
:104220000E944B110EC090917F09892F81528431D9
:1042300020F4892F0E942E5804C080917F090E948B
:10424000BC448E3FF1F08130B9F48091DE098430B6
:1042500020F48F5F8093DE0909C01092DE098091FF
:10426000DF09882319F081508093DF098091DF09ED
:10427000882359F4C1E009C0809180098093DF0947
:1042800004C0809180098093DF09113021F4812FCF
:104290000E94EB1A0CC0C13021F48C2F0E940B1B22
:1042A00006C080E00E94EB1A80E00E940B1BCF91B9
:1042B0001F910895FC018481982F986080EF82837C
:1042C000878586798787168A892F8F7D8483848561
:1042D00025E0829FC001112496878587892B41F4B0
:1042E00081858F3F29F0829FC001112493878287A7
:1042F00083E0878308951F93CF93C0E015E2C19FA9
:10430000C0011124FC01E25DFB4F8785992783FDE5
:1043100002C080FF03C0CF010E945A21CF5FC2328A
:1043200070F3CF911F91089599278C33910509F46B
:1043300066C08D339105A4F488339105A1F18933CA
:1043400091051CF4C79721F1A7C089339105B1F1FC
:104350008A33910509F43DC0CB9709F445C09CC050
:104360008034910509F477C08134910544F48E338B
:10437000910509F45AC0CF970CF062C04BC081344C
:10438000910509F473C08234910509F47AC084C0A0
:104390008091840E8077803119F481E090E0089557
:1043A00080E090E008958091840E8077803219F447
:1043B00081E090E0089580E090E008958091840E7F
:1043C0008077803319F481E090E0089580E090E0F8
:1043D00008958091860E8077803119F481E090E015
:1043E000089580E090E008958091860E8077803275
:1043F00019F481E090E0089580E090E008958091C4
:10440000860E8077803319F481E090E0089580E093
:1044100090E008958091880E8077803119F481E0D2
:1044200090E0089580E090E008958091880E807774
:10443000803219F481E090E0089580E090E00895E2
:104440008091880E8077803319F481E090E00895A0
:1044500080E090E0089580918A0E8077803119F491
:1044600081E090E0089580E090E0089580918A0EC8
:104470008077803219F481E090E0089580E090E048
:10448000089580918A0E8077803319F481E090E05E
:10449000089580E090E0089580E090E00895FF9214
:1044A0000F931F93CF93DF9310E00F2EFFE0FF2EAB
:1044B000F02D82E00E94624585E2189FC001112420
:1044C000EC01C25DDB4F8885882361F48981803FE0
:1044D00009F0F4C08C8188608C838F85867B8F8700
:1044E000FA82ECC02885822F81508032D0F58F85EA
:1044F000992783FD24C080FD22C0822F0E944B118A
:10450000882341F089818F3009F0D8C0CE010E9404
:104510005A21D4C08981803F09F0D0C089858F3F5E
:1045200009F4CCC08A859B85892B09F0C7C08C8192
:1045300088608C838F85867B8F87FA82BFC0888551
:104540000E944B11882309F0B9C08981803F09F08E
:10455000B5C08C8188608C838F85867B8F87FA823B
:10456000ADC02885822F81528431D0F58F8599275F
:1045700083FD24C080FD22C0822F0E942E588823F4
:1045800041F089818F3009F099C0CE010E945A21F3
:1045900095C08981803F09F091C089858F3F09F4DA
:1045A0008DC08A859B85892B09F088C08C818860A5
:1045B0008C838F85867B8F87FA8280C088850E9456
:1045C0002E58882309F07AC08981803F09F076C08F
:1045D0008C8188608C838F85867B8F87FA826EC002
:1045E00000E08885853371F49091E009892F83502C
:1045F000823020F0913011F0963011F491E01DC01E
:1046000090E01BC08885863351F48091E0098530A5
:1046100011F0823011F491E010C090E00EC0988546
:10462000892F87538C3028F4892F0E949421982F4A
:1046300004C088850E94BC44982F9E3FA9F08885BD
:10464000803C21F49130A1F4092F12C08D8181307A
:1046500021F4913011F4092F0BC08D81803141F488
:10466000992331F401E004C088858F3F09F401E00B
:10467000002369F089818F3009F58F85992783FDA3
:104680001DC080FD1BC0CE010E945A2117C0898128
:10469000803F31F08F85992783FD02C080FF0EC0D7
:1046A00089858F3F59F08A859B85892B39F48C81C8
:1046B00088608C838F85867B8F87FA8289818F3093
:1046C00079F48F85992789709070892B49F48091AE
:1046D0001101811729F482E28093110110928B0E4F
:1046E0001F5F123208F4E5CEDF91CF911F910F9139
:1046F000FF90089560932804623019F48FEF80933F
:104700004E090895CF93DF93EC0188818150823266
:1047100018F080E090E03BC088810E94822A282F18
:10472000898199278F30910521F0803F9105A1F073
:104730002CC0332785E290E0289FA001299F500DCF
:10474000389F500D1124FA01E25DFB4F8FE0818309
:104750008785867F878719C0332785E290E0289F69
:10476000A001299F500D389F500D1124FA01E25DE0
:10477000FB4F80EF81838785867F8787168AFA01C2
:10478000EE5CFB4F80818F7D808381E090E0DF9144
:10479000CF9108956F927F928F929F92AF92BF9226
:1047A000CF92DF92EF92FF920F931F93CF93DF93FD
:1047B000CDB7DEB721970FB6F894DEBF0FBECDBFE1
:1047C000BB24B9829B2CAB2C8B2C109250091092DD
:1047D0004F09B0925309B0925509B09254090E9402
:1047E00026058093520980912804882309F0D1C3BB
:1047F000B9828B2D823208F04EC67724689471F806
:104800000F2EF3E06F2EF02D82E00E946245992476
:10481000998185E2989FC00111240F2EFEE2CF2ED0
:10482000F4E0DF2EF02DC80ED91EF601858D9927F4
:10483000807F9070803A910529F40F2EF1E4AF2E1D
:10484000F02D18C0F601858D9927807F9070803BF0
:10485000910529F40F2EF2E4AF2EF02D0BC000E0ED
:1048600021E0AE014F5F5F4F6FED77E082E191E0B5
:104870000E949D2FF601118A108A248122FD0AC20E
:10488000808199278130910509F403C18034910515
:1048900009F00DC2818199278F30910509F49BC0E1
:1048A000803F910509F003C2822F837019F4878538
:1048B00085FF1BC089818B3031F48091750E882370
:1048C00011F07092750E89818C3031F48091780EE0
:1048D000882311F07092780EF601858D41A16A2D22
:1048E0008F700E94EA3C99244FC0F6018585968519
:1048F000892B09F049C0878580FD46C089818B30AE
:10490000D9F48091750E8823B9F0823048F4858DF2
:1049100041A16A2D8F700E949F3C9924939434C0CA
:104920008091750E813081F56092750E1092820E25
:104930001092810E992428C089818C30E1F48091F5
:10494000780E8823C1F0823050F4F601858D41A1A4
:104950006A2D8F700E949F3C9924939415C080917A
:10496000780E813089F46092780E1092770E109252
:10497000760E992409C0F601858D41A16A2D8F70AC
:104980000E949F3C99249394F601848183FF8FC1F8
:10499000877F848382818F3009F089C189818B3040
:1049A00031F48091750E882311F07092750E898113
:1049B0008C3031F48091780E882311F07092780E4B
:1049C0008FE0F6018183858D41A16A2D8F700E9451
:1049D000EA3C99246CC1F601248123FF68C1822F2F
:1049E000877F84838281803F09F061C181838585CF
:1049F0009685892B09F05BC1822F837009F057C11E
:104A000089818B30E1F48091750E8823C1F082306A
:104A100048F4858D41A16A2D8F700E949F3C992496
:104A2000939445C18091750E823009F040C1609227
:104A3000750E1092820E1092810E992438C18981D0
:104A40008C30E9F48091780E8823C9F0823050F4DC
:104A5000F601858D41A16A2D8F700E949F3C99249B
:104A6000939425C18091780E823009F020C1609224
:104A7000780E1092770E1092760E992418C1F601D6
:104A8000858D41A16A2D8F700E949F3C992493943B
:104A90000EC1F601818199278F30910509F49EC0DE
:104AA000803F910509F003C18481837019F48785E3
:104AB00085FF1BC089818B3031F48091750E88236E
:104AC00011F07092750E89818C3031F48091780EDE
:104AD000882311F07092780EF601858D41A16A2D20
:104AE0008F700E94EA3C992452C0F6018585968514
:104AF000892B09F04CC08785992780FD48C083FD2C
:104B000046C089818B30D9F48091750E8823B9F025
:104B1000823048F4858D41A16A2D8F700E949F3CA0
:104B20009924939434C08091750E823081F56092FF
:104B3000750E1092820E1092810E992428C08981E0
:104B40008C30E1F48091780E8823C1F0823050F4EB
:104B5000F601858D41A16A2D8F700E949F3C99249A
:104B6000939415C08091780E823089F46092780E0B
:104B70001092770E1092760E992409C0F601858D59
:104B800041A16A2D8F700E949F3C99249394F60155
:104B9000848183FF8CC0877F848382818F3009F07A
:104BA00086C089818B3031F48091750E882311F095
:104BB0007092750E89818C3031F48091780E882343
:104BC00011F07092780E8FE0F6018183858D41A1FE
:104BD0006A2D8F700E94EA3C992469C0F6012481F5
:104BE00023FF65C0822F877F84838281803F09F005
:104BF0005EC0818385859685892B09F058C0822FF8
:104C0000837009F054C089818B30D9F48091750E7E
:104C10008823B9F0823048F4858D41A16A2D8F70C8
:104C20000E949F3C9924939442C08091750E8230DB
:104C3000F1F56092750E1092820E1092810E9924F9
:104C400036C089818C30E1F48091780E8823C1F0E0
:104C5000823050F4F601858D41A16A2D8F700E943B
:104C60009F3C9924939423C08091780E8230F9F46C
:104C70006092780E1092770E1092760E992417C0DB
:104C8000F601858D41A16A2D8F700E949F3C992469
:104C900093940DC0F601818199278F30910531F0F1
:104CA000803F910521F49924939401C09924F60141
:104CB0008181803F09F058C082A18F3F09F454C020
:104CC0000E94F1037C0100271127F601F4A2E3A260
:104CD00089819927FC01E85EF64F80819927AA27F0
:104CE000BB278E159F05A007B10724F0EE24FF24F3
:104CF00087010AC089819927FC01E85EF64F80810F
:104D0000E81AF10801091109F3E0EF16F1040105B1
:104D10001105CCF089819927880F991FFC01E65D68
:104D2000F64F808191819C0144275527C801B70126
:104D30000E94E16520EE31E040E050E00E945566BF
:104D400079018A0103C0EE24FF248701F601F18A6C
:104D5000E08A80914F09909150098E0D9F1D90938C
:104D6000500980934F0903C0F601118A108A9920D7
:104D700039F4F601828D938D892B11F0138E128EEA
:104D8000F60187859927AC014870507083FD70C08B
:104D9000208931898289938982179307E0F5828D72
:104DA000938D892B11F0538F428FF601848185FFFB
:104DB00026C084899589892B09F05AC08785886027
:104DC0008787809153098F5F809353098081813059
:104DD00071F4858D41A16A2D8F700E94EA3C99245F
:104DE000898180931101F60186818093DD09898193
:104DF000F601608971898F5F0E94103239C0F60117
:104E0000848180628483968185E0989FC00111240B
:104E1000958B848B2DC0F60184818F7D8483208DBA
:104E2000318D2115310521F19920A1F080899189D9
:104E30008217930778F4828D938D892BC9F4878527
:104E400086FD16C0948D85E0989FC0011124938F34
:104E5000828F0EC0F601828D938D892B49F02089B7
:104E60003189808D918D8217930710F4138E128EE5
:104E7000F601868D9927807F9070803A910529F4FC
:104E80000F2EF1E48F2EF02D18C0F601868D992794
:104E9000807F9070803B910529F40F2EF2E48F2ED5
:104EA000F02D0BC000E021E0AE014F5F5F4F6DE5DC
:104EB00079E082E191E00E949D2FF601868D41A16B
:104EC000682D8F700E946D3D282FF6018181803FF3
:104ED00009F042C08785992783FD3EC080FD3CC014
:104EE00090915209809110018917B0F5F1E09F1659
:104EF00089F5222379F5F6018781882369F5848570
:104F0000882351F587898F3F11F08F5F878BF601DA
:104F10008789863008F186898F5F868B843150F4CB
:104F2000858D41A16A2D8F700E94EA3CF601178A97
:104F3000678212C0F601858D41A16A2D8F700E9493
:104F4000EA3CF60187858160878789818F5F0E94AF
:104F5000483202C0F601178AF601878580FF05C036
:104F6000809155098F5F80935509F601878583FFEE
:104F700005C0809153098F5F80935309F60187859F
:104F80008111B39489818F5F8983823208F43CCC8C
:104F900082C280912804813009F0B0C119828981D0
:104FA000482F823208F077C2242F332785E290E021
:104FB000289FB001299F700D389F700D1124FB01AF
:104FC000E25DFB4F87858F7D878785E2489FC00123
:104FD00011240F2EFEE2CF2EF4E0DF2EF02DC80EAE
:104FE000D91EF601858D9927807F9070803A9105B2
:104FF00029F40F2EF1E4AF2EF02D0CC0F601858DB3
:105000009927807F9070803B910521F40F2EF2E468
:10501000AF2EF02DF601848182FD4FC0808199274B
:105020008130910569F18034910509F046C0818194
:1050300099278F30910561F0803F9105F1F5858DBD
:1050400041A16A2D8F700E949F3C9924939435C092
:105050008981282F332785E290E0289FA001299F8E
:10506000500D389F500D1124FA01E25DFB4F858DE4
:10507000F60141A16A2D8F700E94EA3C99241DC05F
:10508000F601818199278F30910561F0803F91056C
:10509000A1F4858D41A16A2D8F700E949F3C9924B7
:1050A00093940BC0F601858D41A16A2D8F700E94EB
:1050B000EA3C8FE0F60181839924F6018181803FEB
:1050C00009F057C082A18F3F09F453C00E94F10339
:1050D0007C0100271127F601F4A2E3A28981992718
:1050E000FC01E85EF64F80819927AA27BB278E1521
:1050F0009F05A007B10724F0EE24FF2487010AC012
:1051000089819927FC01E85EF64F8081E81AF10851
:1051100001091109F3E0EF16F10401051105CCF0C6
:1051200089819927880F991FFC01E65DF64F8081E0
:1051300091819C0144275527C801B7010E94E16570
:1051400020EE31E040E050E00E94556679018A018E
:1051500003C0EE24FF248701F601F18AE08A8091E2
:105160004F09909150098E0D9F1D90935009809387
:105170004F09F60120893189828993898217930723
:1051800088F5848185FF22C084899589892B81F5E2
:10519000878588608787809153098F5F8093530943
:1051A0008081813059F4858D41A16A2D8F700E94D4
:1051B000EA3C99248FE0F601818382838981F6019C
:1051C000608971898F5F0E94103212C0F60184815C
:1051D00080628483968185E0989FC0011124958B1D
:1051E000848B06C0F60184818F7D8483158A148A9E
:1051F000F601868D9927807F9070803A910529F479
:105200000F2EF1E48F2EF02D0CC0F601868D99271C
:10521000807F9070803B910521F40F2EF2E48F2E59
:10522000F02DF601868D41A1682D8F700E946D3D95
:10523000282FF6018785992783FD42C080FD40C055
:1052400090915209809110018917D0F5F1E09F16D5
:10525000A9F5222399F5F6018781882389F58485AC
:10526000882371F58181803F59F587898F3F11F03F
:105270008F5F878BF6018789863010F186898F5F73
:10528000868B843158F4858D41A16A2D8F700E94E0
:10529000EA3CF601178A83E0878312C0F601858D08
:1052A00041A16A2D8F700E94EA3CF60187858160DA
:1052B000878789818F5F0E94483202C0F601178A72
:1052C000F601878580FF05C0809155098F5F809327
:1052D0005509F601878583FF05C0809153098F5FCB
:1052E00080935309F60187858111B39489818F5F7B
:1052F0008983482F823208F457CECDC0809128048C
:10530000823009F0C8C019828981982F823208F052
:10531000C2C085E2989FC00111240F2EFEE2CF2E5D
:10532000F4E0DF2EF02DC80ED91EF601858D9927E9
:10533000807F9070803A910529F40F2EF1E4AF2E12
:10534000F02D0CC0F601858D9927807F9070803BF1
:10535000910521F40F2EF2E4AF2EF02D40914E096D
:105360004423D1F0898199279C012F5F3F4F842FDF
:1053700099272817390741F4F601858D41A16A2D37
:105380008F700E949F3C0FC0F601858D41A16A2D50
:105390008F700E94EA3C07C0F601858D41A16A2DFD
:1053A0008F700E949F3CF60182A18F3F09F46CC070
:1053B0000E94F1037C0100271127F601F4A2E3A269
:1053C0008091270480FF1CC089819927FC01E85E39
:1053D000F64F80819927AA27BB278E159F05A00726
:1053E000B10724F0EE24FF2487010AC089819927A0
:1053F000FC01E85EF64F8081E81AF1080109110905
:10540000F3E0EF16F1040105110574F18091270412
:1054100081FF19C089819927880F991FFC01E65DDA
:10542000F64F808191819C0144275527C801B7011F
:105430000E94E16520EE31E040E050E00E945566B8
:1054400079018A0114C0C801B70128EB31E040E0BE
:1054500050E00E94E16520EE31E040E050E00E9423
:10546000556679018A0103C0EE24FF248701F60105
:10547000F18AE08A80914F09909150098E0D9F1D0D
:105480009093500980934F0989818F5F8983982F6A
:10549000823208F43ECFBB2031F4B0925409B0926E
:1054A0005509B09256090E941A05982F8093510908
:1054B00080912904891710F49093290420914F09B1
:1054C0003091500980912A0490912B048217930700
:1054D00020F430932B0420932A0421960FB6F894DD
:1054E000DEBF0FBECDBFDF91CF911F910F91FF9017
:1054F000EF90DF90CF90BF90AF909F908F907F9074
:105500006F900895815099270895CF93DF93EC0110
:10551000862F0E94822A833278F4282F332785E24F
:1055200090E0289FA001299F500D389F500D112415
:10553000FA01E25DFB4FC683DF91CF910895EF92B0
:10554000FF921F93CF937C01C0E080EC0E94BC448B
:105550008111C1E081EC0E94BC448111C26082ECE7
:105560000E94BC448111C46081ED0E94BC44811141
:10557000C86084EC0E94BC448111C06185EC0E942B
:10558000BC448111C06286EC0E94BC448111C0649D
:1055900087EC0E94BC448111C06810E083EC0E943B
:1055A000BC44811111E082ED0E94BC448111126063
:1055B00083ED0E94BC4481111460F701C083118304
:1055C000C0E081E00E944B118111C1E082E00E94A5
:1055D0004B118111C26083E00E944B118111C460A4
:1055E00084E00E944B118111C86085E00E944B113C
:1055F0008111C06186E00E944B118111C06287E079
:105600000E944B118111C06488E00E944B118111EE
:10561000C068F701C283C0E089E00E944B1181118C
:10562000C1E08AE00E944B118111C2608BE00E94B0
:105630004B118111C4608CE00E944B118111C86034
:105640008DE00E944B118111C0618EE00E944B11D0
:105650008111C0628FE00E944B118111C06480E112
:105660000E944B118111C068F701C383C0E081E142
:105670000E944B118111C1E082E10E944B11811106
:10568000C26083E10E944B118111C46084E10E94D9
:105690004B118111C86085E10E944B118111C061DD
:1056A00086E10E944B118111C06287E10E944B117B
:1056B0008111C06488E10E944B118111C068F7011B
:1056C000C483C0E089E10E944B118111C1E08AE1ED
:1056D0000E944B118111C2608BE10E944B1181111C
:1056E000C4608CE10E944B118111C8608DE10E9461
:1056F0004B118111C0618EE10E944B118111C0627A
:105700008FE10E944B118111C06480E20E944B1115
:105710008111C068F701C583CF911F91FF90EF9071
:1057200008951F93CF93DF93182FEB010E94822AD5
:10573000482F833218F080E090E073C0992725E26B
:1057400030E0829FB001839F700D929F700D1124F5
:10575000FB01EE5CFB4F208122FD24C0FB01E25DDA
:10576000FB4F8181803F71F485859685892B39F4C3
:1057700021FD05C020FD03C0878585FF03C08FE0A4
:10578000888335C0242F332785E290E0289FF001DD
:10579000299FF00D389FF00D1124E25DFB4F8181B0
:1057A000888325C030E0232F5EE0259FC0011124AF
:1057B000DC01A956B64FFD018181813099F490E05A
:1057C0007FE060EFFD01E90FF11D8285841739F458
:1057D00031E08C9182FF02C0788301C068839F5FB3
:1057E000943080F32F5F253010F43323F1F2242F0F
:1057F000332785E290E0289FA001299F500D389F14
:10580000500D1124FA01E25DFB4F87858983808961
:1058100091899C838B83812F0E9493328A8381E0BC
:1058200090E0DF91CF911F9108950E94822A8332E8
:1058300018F080E090E00895282F332785E290E06B
:10584000289FA001299F500D389F500D1124FA0167
:10585000E25DFB4F8181803F59F4FA01EE5CFB4F22
:10586000208121FD05C020FD03C081E090E0089566
:1058700080E090E008950E94822A833218F080E050
:1058800090E00895282F332785E290E0289FA0011B
:10589000299F500D389F500D1124FA01E25DFB4FF6
:1058A0002785283011F0213019F481E090E0089527
:1058B00080E090E00895FC0180914F09909150099B
:1058C00091838083809151098283809152098383DF
:1058D000809153098483809154098583809155096F
:1058E00086838091560987830895982F815082324C
:1058F00038F485E2989FC0011124875F9B4F08957B
:1059000080E090E008959EEF81B1892381B982B152
:10591000892382B917B818B891EF8AB189238AB957
:105920008BB189238BB908950F930E94822A282F67
:10593000833168F000E0202F40E050E062E07CE03E
:1059400082E191E00E949D2F80E090E007C088E115
:1059500099E0FC01E20FF11D808199270F910895D4
:105960000F930E94822A833168F000E0202F40E0EC
:1059700050E060E17CE082E191E00E949D2F80E6B2
:1059800092E212C09927880F991FFC01E65DF64F3D
:105990002081318184E190E0289FA001299F500D52
:1059A000389F500D1124CA010F9108950F93CF9382
:1059B000DF93EB010E94822A833158F000E0202F10
:1059C00040E050E06FE17CE082E191E00E949D2F99
:1059D00012C099272AE239E0880F991FFC01E20FD3
:1059E000F31FCE0164E170E00E940C667183608356
:1059F000C9010E947C35DF91CF910F9108950E94DB
:105A0000822A833118F080E090E00895282F332710
:105A100085E290E0289FA001299F500D389F500DEE
:105A20001124FA01E25DFB4F8089918908950E945B
:105A3000822A833118F080E090E00895282F3327E0
:105A400085E290E0289FA001299F500D389F500DBE
:105A50001124FA01E25DFB4F83A194A10895809384
:105A6000270460934E0908951F93CF93C0E015E279
:105A7000C19FC0011124FC01E25DFB4F82A18F3F59
:105A800041F00E94F1032C2F3327F901E85EF64F15
:105A90008083CF5FC23160F388E199E00E945C357A
:105AA000CF911F910895CF9380912804833059F0AE
:105AB00083E080932804C0E061E08C2F0E946F1A7D
:105AC000CF5FC232C8F3CF910895809190098823A7
:105AD00041F00E94722D0E949D2D8BE599E00E945D
:105AE000EA2D0895259A2D98269A2E988AEA809371
:105AF000800089E1809381001092850010928400DB
:105B000080E395E09093870080938600109289004F
:105B10001092880010928B0010928A0010928D00D3
:105B200010928C0060E070E081E00E94C82D60E07F
:105B300070E082E00E94C82D08951092900084E0E9
:105B4000809391001092950010929400109297000B
:105B500010929600109299001092980010929B005B
:105B600010929A0010929D0010929C001092580979
:105B70001092570910925A091092590980916900A0
:105B800088608093690010926A00E99AE19A08950A
:105B900099278230910581F0833091051CF401979B
:105BA00021F00895039779F00895872F992780931E
:105BB0008900609388000895872F992780938B0030
:105BC00060938A000895872F992780938D006093B2
:105BD0008C000895FC01118210821382128285E0EC
:105BE00090E09583848316820895EF92FF920F933D
:105BF0001F93CF93DF93EC018E81982F8F5F8E835D
:105C0000963068F060E375E081E00E94C82D60E3A3
:105C100075E082E00E94C82D86E08E8355C08A819F
:105C20009B819C0144275527888199817C0100270D
:105C30001127DA01C901689412F8880F991FAA1F69
:105C4000BB1F1694D1F7820F931FA41FB51F280FF7
:105C5000391F4A1F5B1FCA01B90125E830E040E047
:105C600050E00E94E165A80197010E943366E901B6
:105C7000C901845490408652944010F0C0E3D5E0AE
:105C800080919009882349F08091E804803F29F4AD
:105C9000BE0181E00E94C82D05C060E375E081E08F
:105CA0000E94C82D80919109882349F080911006A7
:105CB000803F29F4BE0182E00E94C82D05C060E348
:105CC00075E082E00E94C82DDF91CF911F910F9166
:105CD000FF90EF9008951F920F920FB60F9211242C
:105CE0002F933F938F939F9380919400282F332776
:105CF000322F2227809195009927282B392B8091CC
:105D0000690099278C7090700C97E1F430935C09CE
:105D100020935B09109294001092950080912C04BE
:105D200090912D0490935E0980935D0910922D044B
:105D300010922C0410926109809169008B7F8093EE
:105D4000690010C08091690099278C709070089745
:105D500049F430932D0420932C04809169008460D1
:105D6000809369009F918F913F912F910F900FBE6B
:105D70000F901F901895CF93DF93CDB7DEB7239781
:105D80000FB6F894DEBF0FBECDBFFE013196A0E87E
:105D9000B1E083E090E021E08030920719F40E94A6
:105DA000AF6603C0182E0E94AF6643E050E060E586
:105DB00071E0CE0101960E94D654882391F00E9492
:105DC000FB2EE0E5F1E0A0E8B1E083E090E021E027
:105DD0008030920719F40E94C06603C0182E0E94FA
:105DE000C066279823960FB6F894DEBF0FBECDBFCE
:105DF000DF91CF910895CF93DF93CDB7DEB76E9744
:105E00000FB6F894DEBF0FBECDBF84E1FE013B9616
:105E100011928A95E9F740E064E124E130E0522FE5
:105E2000FE013B96469FC0011124DC01AC57BE4FDA
:105E30002115310551F081E02030380719F40E9416
:105E4000C06603C0152E0E94C066A8954F5F4830FB
:105E500038F31982FE013196A3E8B1E081E090E0C9
:105E600021E08030920719F40E94C06603C0182E0A
:105E70000E94C0666E960FB6F894DEBF0FBECDBF0F
:105E8000DF91CF910895CF93DF93CDB7DEB7219700
:105E90000FB6F894DEBF0FBECDBFFE013196A3E86A
:105EA000B1E081E090E021E08030920719F40E9497
:105EB000AF6603C0182E0E94AF668981893010F04A
:105EC00088E089838981992721960FB6F894DEBFEF
:105ED0000FBECDBFDF91CF910895CF93DF93CDB7A4
:105EE000DEB764970FB6F894DEBF0FBECDBF9B013F
:105EF000FE01319694E1899FD0011124A059BE4F33
:105F000084E190E041E08030940719F40E94AF668C
:105F100003C0182E0E94AF6684E1FE013196D901BC
:105F200001900D928A95E1F764960FB6F894DEBF62
:105F30000FBECDBFDF91CF9108956F927F928F9268
:105F40009F92AF92BF92CF92DF92EF92FF920F9308
:105F50001F93CF93DF93CDB7DEB7A9970FB6F89411
:105F6000DEBF0FBECDBF6C015B013A01022FFE0107
:105F7000B996A3E8B1E081E090E021E0803092079B
:105F800019F40E94AF6603C0182E0E94AF6689A55F
:105F9000883008F0D4C09924FE01759684E1DF01B1
:105FA0001D928A95E9F7B601CF010E94DA65192D95
:105FB00089A5981608F05EC00F2EF4E18F2EF02D03
:105FC0000F2EF4E1EF2EFF24F02DFE013196189DE7
:105FD000C0011124DC01AC57BE4FE114F10459F0AB
:105FE00020E0E21621E0F20619F40E94AF6603C039
:105FF0001E2C0E94AF668D859E858A159B0599F59E
:1060000046E050E0B601CE0101960E94D6548823A6
:1060100051F5992493948F858A3008F090C0890DAA
:106020008F87053008F004E0198A1A8A1B8A1C8AB7
:10603000802F9927AC01B301CE0141960E94C36520
:10604000FE013196189DD0011124AC57BE4F84E15A
:1060500090E021E08030920719F40E94C06603C0EE
:10606000182E0E94C0661F5F89A5181718F4992082
:1060700009F4ABCF992009F052C089A5883008F007
:106080004EC08F5F89A78CE0FE01319611928A95F0
:10609000E9F7F60101900020E9F731972E2F2C192E
:1060A0002C3008F02BE010E0121780F4AE014F5FA7
:1060B0005F4F812F9927DC01A40FB51FF601E80F70
:1060C000F91F80818C931F5F121798F3BE86AD86EF
:1060D00081E08F87053008F004E0088B198A1A8A5E
:1060E0001B8A1C8A802F9927AC01B301CE014196EF
:1060F0000E94C365FE01319699A584E1989FD00165
:106100001124A059BE4F84E190E021E08030920735
:1061100019F40E94C06603C0182E0E94C066FE01DA
:10612000B996A3E8B1E081E090E021E080309207E9
:1061300019F40E94C06603C0182E0E94C066A9967A
:106140000FB6F894DEBF0FBECDBFDF91CF911F9188
:106150000F91FF90EF90DF90CF90BF90AF909F9006
:106160008F907F906F900895089582E1ECE8FEE0B3
:1061700011928A95E9F780E1EEE9FEE011928A95A5
:10618000E9F7E0ECFEE0A8E8B0E082E190E021E091
:106190008030920719F40E94AF6603C0182E0E9447
:1061A000AF66E2EDFEE0AAE9B0E082E190E021E036
:1061B0008030920719F40E94AF6603C0182E0E9427
:1061C000AF66E4EEFEE0ACEAB0E080E190E021E012
:1061D0008030920719F40E94AF6603C0182E0E9407
:1061E000AF66EEEAFEE0ADEBB0E082E190E021E0E8
:1061F0008030920719F40E94AF6603C0182E0E94E7
:10620000AF66E4EEF9E0A5E8B0E081E090E021E0DF
:106210008030920719F40E94AF6603C0182E0E94C6
:10622000AF66E5EEF9E0A6E8B0E082E090E021E0BC
:106230008030920719F40E94AF660895182E0E94CC
:10624000AF660895CF93DF93CDB7DEB762970FB6F1
:10625000F894DEBF0FBECDBFFE01319682E1DF01B3
:106260001D928A95E9F7A8E8B0E082E190E021E08C
:106270008030920719F40E94C06603C0182E0E9455
:10628000C066FE013196AAE9B0E082E190E021E02B
:106290008030920719F40E94C06603C0182E0E9435
:1062A000C066FE013196ACEAB0E080E190E021E00A
:1062B0008030920719F40E94C06603C0182E0E9415
:1062C000C066FE013196ADEBB0E082E190E021E0E6
:1062D0008030920719F40E94C06603C0182E0E94F5
:1062E000C0660E94B53062960FB6F894DEBF0FBE4E
:1062F000CDBFDF91CF9108950E94301B982F8091E0
:10630000E409891790F49093E409E4EEF9E0A5E834
:10631000B0E081E090E021E08030920719F40E9423
:10632000C06603C0182E0E94C0660E942B1B9C01F1
:106330008091E5099091E60982179307A0F43093C4
:10634000E6092093E509E5EEF9E0A6E8B0E082E091
:1063500090E021E08030920719F40E94C066089511
:10636000182E0E94C06608958091E4099927089527
:106370008091E5099091E609089590E04CE85EE08F
:10638000292F3327F901E40FF51F808180FF17C003
:106390008E7F8083D901A857BF4FF901E054F14F98
:1063A0008081082E0E94B466D901A656BF4FF9011C
:1063B000EE52F14F8081082E0E94B4660895E92FB5
:1063C000FF27DF01A40FB51F8C9181FF0CC08D7FCB
:1063D0008C93DF01A354BF4FE255F14F8081082E0B
:1063E0000E94B46608959F5F923150F290E02EE9CA
:1063F0003EE0E92FFF27DF01A20FB31F8C91813010
:1064000059F41C92DF01A455BF4FEC51F14F80812C
:10641000082E0E94B46608959F5F903150F308954E
:10642000282F2150223198F580EC9EE0FC01E20FEC
:10643000F11D3081832F9927929582958F7089273E
:106440009F7089278F30910514F5482F4F5F942F47
:106450009295907F832F8F70890F8083CB018370FB
:106460009070892B11F041E001C040E03327F90121
:10647000EE52F14FCB019695879596958795840FAF
:106480008083F901E457F14F808181608083089512
:10649000E82FE150E231C0F4FF27DF01A054B14FF3
:1064A0002C91822F99278F7090700F971CF5822F57
:1064B0008F708F5F922F907F890F8C93E457F14FED
:1064C00080818160808308958351803198F4E82F22
:1064D000FF27DF01AC51B14F2C91822F99278F708C
:1064E00090700F973CF4822F8F5F8C93E256F14FA0
:1064F00081E08083089581508231A0F4E82FFF2746
:10650000DF01A255B14F2C91822F99278F70907087
:106510000F9744F4822F8F5F8C93E457F14F808163
:10652000826080830895E82FE150E23188F42E2FB5
:106530003327F901E054F14F8081882331F4F901C8
:10654000E255F14F8081882391F081E090E0089539
:10655000282F2351203158F484EE9EE0FC01E20FF5
:10656000F11D8081882319F081E090E0089580E09A
:1065700090E00895CF93DF93EC01FC0120E532E039
:106580008EE090E041E08030940721F4D9010E9430
:10659000C06604C0D901182E0E94C066CE010296C2
:1065A000AC01698188810E94341BDF91CF910895ED
:1065B000FC01A0E5B2E08EE090E021E0803092079F
:1065C00019F40E94AF660895182E0E94AF660895D0
:1065D000FC01A0E6B2E08FE190E021E0803092077C
:1065E00019F40E94C0660895182E0E94C06608958E
:1065F000FC01A0E6B2E08FE190E021E0803092075C
:1066000019F40E94AF660895182E0E94AF6608958F
:10661000FC01ACE7BBE088E090E021E0803092072D
:1066200019F40E94C0660895182E0E94C06608954D
:10663000FC01ACE7BBE088E090E021E0803092070D
:1066400019F40E94AF660895182E0E94AF6608954F
:106650000F93CF93DF93CDB7DEB721970FB6F894A2
:10666000DEBF0FBECDBF8983853060F000E021E042
:10667000AE014F5F5F4F67E470E084E591E00E94F8
:106680009D2F15C0898199E1899FC0011124FB01CB
:10669000DC01A252B14F89E190E021E08030920705
:1066A00019F40E94C06603C0182E0E94C06621968D
:1066B0000FB6F894DEBF0FBECDBFDF91CF910F9123
:1066C00008950F93CF93DF93CDB7DEB721970FB621
:1066D000F894DEBF0FBECDBF8983853060F000E047
:1066E00021E0AE014F5F5F4F64E570E084E591E02B
:1066F0000E949D2F15C0898199E1899FC0011124B5
:10670000FB01DC01A252B14F89E190E021E0803031
:10671000920719F40E94AF6603C0182E0E94AF665C
:1067200021960FB6F894DEBF0FBECDBFDF91CF919B
:106730000F9108950F93CF93DF93CDB7DEB72197D5
:106740000FB6F894DEBF0FBECDBF8983803260F0F4
:1067500000E021E0AE014F5F5F4F60E670E084E54E
:1067600091E00E949D2F14C0FB0199818CE2989FBB
:10677000D0011124A659BC4F8CE290E021E080307A
:10678000920719F40E94C06603C0182E0E94C066CA
:1067900021960FB6F894DEBF0FBECDBFDF91CF912B
:1067A0000F9108950F93CF93DF93CDB7DEB7219765
:1067B0000FB6F894DEBF0FBECDBF8983803260F084
:1067C00000E021E0AE014F5F5F4F6AE670E084E5D4
:1067D00091E00E949D2F14C0FB0199818CE2989F4B
:1067E000D0011124A659BC4F8CE290E021E080300A
:1067F000920719F40E94AF6603C0182E0E94AF667C
:1068000021960FB6F894DEBF0FBECDBFDF91CF91BA
:106810000F9108950F93CF93DF93CDB7DEB72197F4
:106820000FB6F894DEBF0FBECDBF8983843160F010
:1068300000E021E0AE014F5F5F4F64E770E084E568
:1068400091E00E949D2F14C0FB01998188E1989FDF
:10685000D0011124A451B74F88E190E021E08030AD
:10686000920719F40E94C06603C0182E0E94C066E9
:1068700021960FB6F894DEBF0FBECDBFDF91CF914A
:106880000F9108950F93CF93DF93CDB7DEB7219784
:106890000FB6F894DEBF0FBECDBF8983843160F0A0
:1068A00000E021E0AE014F5F5F4F6EE770E084E5EE
:1068B00091E00E949D2F14C0FB01998188E1989F6F
:1068C000D0011124A451B74F88E190E021E080303D
:1068D000920719F40E94AF6603C0182E0E94AF669B
:1068E00021960FB6F894DEBF0FBECDBFDF91CF91DA
:1068F0000F910895CF93DF93CDB7DEB769970FB6A9
:10690000F894DEBF0FBECDBFFC01862F81508232CE
:1069100018F080E090E02AC06150808189838181F5
:106920008A8382818B8383818C838781888787890F
:10693000888F808D898F848195819E838D838681C8
:106940008F83DF0118968FE0FE0139960D9001923A
:106950008A95E1F789E1689FC00111248457944F1B
:10696000BC01CE0101960E944B35992769960FB65E
:10697000F894DEBF0FBECDBFDF91CF9108950F9386
:106980001F93CF93DF93CDB7DEB769970FB6F89417
:10699000DEBF0FBECDBF8C01962F91509232B0F565
:1069A00089E1989FC00111249E012F5F3F4FDC01B8
:1069B000A457B44F89E190E041E08030940721F47E
:1069C000F9010E94AF6604C0F901182E0E94AF665B
:1069D0008981F80180838A8181838B8182838C8184
:1069E000838388858783888D878B898D808F8D8130
:1069F0009E81958384838F818683D80118968FE04A
:106A0000FE01399601900D928A95E1F769960FB6CD
:106A1000F894DEBF0FBECDBFDF91CF911F910F91D4
:106A2000089581508B30C8F4FB01A82FBB27CD01FE
:106A300082959295907F9827807F9827DC01A453B8
:106A4000B54F80E190E021E08030920719F40E9478
:106A5000C0660895182E0E94C066089581508B303C
:106A6000C8F4FB01A82FBB27CD0182959295907F9A
:106A70009827807F9827DC01A453B54F80E190E0F0
:106A800021E08030920719F40E94AF660895182E15
:106A90000E94AF660895FC01DB0189E190E021E0EE
:106AA0008030920719F40E94C06603C0182E0E941D
:106AB000C06681E090E00895FC01A0E1B0E082E1D1
:106AC00090E021E08030920719F40E94C06608959A
:106AD000182E0E94C0660895FC01A0E1B0E082E19A
:106AE00090E021E08030920719F40E94AF6608958B
:106AF000182E0E94AF660895FC01A0E3B0E084E286
:106B000090E021E08030920719F40E94C066089559
:106B1000182E0E94C0660895FC01A0E3B0E084E254
:106B200090E021E08030920719F40E94AF6608954A
:106B3000182E0E94AF660895FC01A0E8B2E088E13B
:106B400090E021E08030920719F40E94C066089519
:106B5000182E0E94C0660895FC01A0E8B2E088E10A
:106B600090E021E08030920719F40E94AF6608950A
:106B7000182E0E94AF6608950F93FC018081882330
:106B800019F488E992E016C08081813019F48EED05
:106B900092E010C08081823019F484E293E00AC050
:106BA00000E021E0AF0167E471E084E591E00E943C
:106BB0009D2F0DC0DC0186E490E021E0803092073B
:106BC00019F40E94C06603C0182E0E94C0660F917F
:106BD00008950F93CF93DF93CDB7DEB721970FB60C
:106BE000F894DEBF0FBECDBF8983882319F488E9EE
:106BF00092E018C08981813019F48EED92E012C0C4
:106C00008981823019F484E293E00CC000E021E035
:106C1000AE014F5F5F4F60E671E084E591E00E9456
:106C20009D2F0EC0FB01DC0186E490E021E0803066
:106C3000920719F40E94AF6603C0182E0E94AF6637
:106C400021960FB6F894DEBF0FBECDBFDF91CF9176
:106C50000F910895CF93DF93CDB7DEB760970FB64E
:106C6000F894DEBF0FBECDBFFE013196A0E0B0E0CC
:106C700080E190E021E08030920719F40E94AF6635
:106C800003C0182E0E94AF668B858F3119F48FE1F7
:106C900090E008C08B85803219F480E290E002C059
:106CA0008FE190E060960FB6F894DEBF0FBECDBFC7
:106CB000DF91CF9108950F931F93CF93DF93CDB7BB
:106CC000DEB76E970FB6F894DEBF0FBECDBFFE01E4
:106CD0003196A0E0B0E084E090E021E080309207BF
:106CE00019F40E94AF6603C0182E0E94AF6644E0FC
:106CF00050E068E671E0CE0101960E94D6548823E8
:106D000009F44DC08E010F5F1F4F8EE1D8011D9217
:106D10008A95E9F785E0E8E6F1E0D80101900D9267
:106D20008A95E1F71D821E821F82188619861A86AF
:106D30001B860E94441EF801A0E0B0E080E190E0D4
:106D400021E08030920719F40E94C06603C0182E1B
:106D50000E94C066FE013196A0E0B0E084E090E0C1
:106D600021E08030920719F40E94C06603C0182EFB
:106D70000E94C066FE01319684E1DF011D928A9572
:106D8000E9F7AAEDBFE084E190E021E080309207CE
:106D900019F40E94C06603C0182E0E94C066FE014E
:106DA0003196A0E3B2E08AE090E021E080309207E3
:106DB00019F40E94AF6603C0182E0E94AF664AE025
:106DC00050E064E871E0CE0101960E94D654882319
:106DD00079F10E94641E0E94DF100E94A9560E9451
:106DE0003B060E945D0FFE0131968EE1DF011D9290
:106DF0008A95E9F7AEE5BFE080E190E021E08030E0
:106E0000920719F40E94C06603C0182E0E94C06643
:106E1000E4E8F1E0A0E3B2E08AE090E021E0803035
:106E2000920719F40E94C06603C0182E0E94C06623
:106E3000FE013196A0E8B1E083E090E021E08030EF
:106E4000920719F40E94AF6603C0182E0E94AF6625
:106E500043E050E06DE671E0CE0101960E94D65409
:106E6000882391F00E94FB2EEDE6F1E0A0E8B1E06E
:106E700083E090E021E08030920719F40E94C06620
:106E800003C0182E0E94C066FE013196A0E8B0E053
:106E900085E090E021E08030920719F40E94AF660F
:106EA00003C0182E0E94AF6645E050E061E771E034
:106EB000CE0101960E94D654882309F475C0FE01C4
:106EC00031968EE1DF011D928A95E9F7ACEBB0E0D7
:106ED00081E090E021E08030920719F40E94C066C2
:106EE00003C0182E0E94C066FE013196A5E8B0E0EE
:106EF00081E090E021E08030920719F40E94C066A2
:106F000003C0182E0E94C066FE013196A6E8B0E0CC
:106F100082E090E021E08030920719F40E94C06680
:106F200003C0182E0E94C066FE013196A8E8B0E0AA
:106F300082E190E021E08030920719F40E94C0665F
:106F400003C0182E0E94C066FE013196ACEAB0E084
:106F500080E190E021E08030920719F40E94C06641
:106F600003C0182E0E94C066FE013196ADEBB0E062
:106F700082E190E021E08030920719F40E94C0661F
:106F800003C0182E0E94C066E1E7F1E0A0E8B0E07F
:106F900085E090E021E08030920719F40E94C066FD
:106FA00003C0182E0E94C066FE013196AAEDBFE014
:106FB00089E090E021E08030920731F40E94AF66D2
:106FC00006C00E94C06630C0182E0E94AF6690E0D6
:106FD0009E012F5F3F4F8981181634F5AE014F5F38
:106FE0005F4FF901E90FF11D808180538A3090F0E5
:106FF00089E0F90111928A95E9F7F901AAEDBFE05C
:1070000089E090E021E080309207D9F2182E0E94AA
:10701000C0660AC09F5F983038F49A01FA01E90F00
:10702000F11D80811816ECF2FE013196A3EEBFE04F
:1070300089E090E021E08030920731F40E94AF6651
:1070400006C00E94C06630C0182E0E94AF6690E055
:107050009E012F5F3F4F8981181634F5AE014F5FB7
:107060005F4FF901E90FF11D808180538A3090F064
:1070700089E0F90111928A95E9F7F901A3EEBFE0E1
:1070800089E090E021E080309207D9F2182E0E942A
:10709000C0660AC09F5F983038F49A01FA01E90F80
:1070A000F11D80811816ECF26E960FB6F894DEBFD3
:1070B0000FBECDBFDF91CF911F910F910895CFEFFC
:1070C000D0E1DEBFCDBF0E94C9530E94993A0E9411
:1070D000561B0E9466050E94DB530E9408460E94D0
:1070E000BB2E0E945B36E5E6FEE0A0E7B0E08FE055
:1070F00090E021E08030920719F40E94AF6603C04F
:10710000182E0E94AF668091650E9091660E8A3FA0
:10711000910531F18B3F910538F48436910561F08A
:107120008D37910599F039C021E0843F920711F124
:10713000885E934049F131C086E28093E20084E0AA
:107140008093E30083E18093E40027C08EE1809385
:10715000E20084E08093E30083E18093E4001DC0BB
:107160008EE08093E20084E08093E30083E18093EB
:10717000E40013C086E08093E20084E08093E300A3
:1071800083E18093E40009C082E08093E20084E020
:107190008093E30083E18093E4000E94940F809148
:1071A000670E9091680E059738F485E090E0909313
:1071B000680E8093670E0DC08091670E9091680EE7
:1071C000815D974030F080ED97E09093680E80935A
:1071D000670E8091690E90916A0E28E080309207C8
:1071E00038F08959994021F010926A0E1092690E78
:1071F0008091710E80FF04C082E08093750E02C002
:107200001092750E8091710E81FF04C082E0809310
:10721000780E02C01092780E8091720E8A50813FD3
:1072200018F08FE48093720E0E94AB3D0E94585676
:107230000E94CC1F0E944D4587E00E943F607894D9
:107240000E943052A89580E00E9462450E94134639
:10725000FACF1F93162FA398992787709070880FE5
:10726000991F81640E94D453812F0E94D45380E0DF
:107270000E94D453A39A99271F9108950F931F93A7
:10728000162F042FA398992787709070880F991F45
:1072900080640E94D453812F0E94D453802F0E9477
:1072A000D453A39A1F910F9108951F93CF93C09128
:1072B000E709CC2389F511E01093E7094CE16AE076
:1072C0008C2F0E943E394C2F6C2F8C2F0E943E3900
:1072D0004FEF612F8C2F0E943E394C2F62E08C2F94
:1072E0000E943E394C2F63E08C2F0E943E394C2F78
:1072F00064E08C2F0E943E394C2F65E08C2F0E9459
:107300003E394C2F6CE08C2F0E943E394C2F6DE0A3
:107310008C2F0E943E390AC1C091E709C13089F51E
:107320004CE16AE08C2F0E943E3940E0642F8C2FA4
:107330000E943E394FEF6C2F8C2F0E943E3940E067
:1073400062E08C2F0E943E3940E063E08C2F0E9467
:107350003E3940E064E08C2F0E943E3940E065E019
:107360008C2F0E943E3940E06CE08C2F0E943E3909
:1073700040E06DE08C2F0E943E3982E08093E70967
:10738000D5C0C091E709C23089F54CE16AE08C2F85
:107390000E943E3940E0642F8C2F0E943E394FEF0F
:1073A00061E08C2F0E943E3940E06C2F8C2F0E94B0
:1073B0003E3940E063E08C2F0E943E3940E064E0BB
:1073C0008C2F0E943E3940E065E08C2F0E943E39B0
:1073D00040E06CE08C2F0E943E3940E06DE08C2F45
:1073E0000E943E3983E08093E709A0C0C091E7097D
:1073F000C33089F54CE16AE08C2F0E943E3940E0B1
:10740000642F8C2F0E943E394FEF61E08C2F0E9439
:107410003E3940E062E08C2F0E943E3940E06C2F04
:107420008C2F0E943E3940E064E08C2F0E943E3950
:1074300040E065E08C2F0E943E3940E06CE08C2FEC
:107440000E943E3940E06DE08C2F0E943E3984E07E
:107450008093E7096BC0C091E709C43089F54CE11E
:107460006AE08C2F0E943E394CEF60E08C2F0E9426
:107470003E394FEF61E08C2F0E943E3940E062E0E0
:107480008C2F0E943E3940E063E08C2F0E943E39F1
:1074900040E06C2F8C2F0E943E3940E065E08C2F3D
:1074A0000E943E3940E06CE08C2F0E943E3940E063
:1074B0006DE08C2F0E943E3985E08093E70936C04D
:1074C000C091E709C53081F54CE16AE08C2F0E943C
:1074D0003E3940E0642F8C2F0E943E3940EF61E03E
:1074E0008C2F0E943E3940E062E08C2F0E943E3992
:1074F00040E063E08C2F0E943E3940E064E08C2F36
:107500000E943E3940E06C2F8C2F0E943E3940E0B3
:107510006CE08C2F0E943E3940E06DE08C2F0E9481
:107520003E391092E70902C01092E709CF911F91EE
:1075300008959B9AA39A4CE16AE080E00E943E394C
:1075400040E064E1842F0E943E3940E0642F842FA4
:107550000E943E394FEF61E080E00E943E3940E0FA
:1075600062E0842F0E943E3940E063E0842F0E9455
:107570003E3940E064E0842F0E943E3940E065E0FF
:10758000842F0E943E3940E06CE0842F0E943E39F7
:1075900040E06DE0842F0E943E394CE16AE081E0DA
:1075A0000E943E3940E064E181E00E943E3940E0C3
:1075B000642F81E00E943E394FEF61E0862F0E94E8
:1075C0003E3940E062E081E00E943E3940E063E005
:1075D00081E00E943E3940E064E081E00E943E3953
:1075E00040E065E081E00E943E3940E06CE081E0EF
:1075F0000E943E3940E06DE081E00E943E394CE15E
:107600006AE082E00E943E3940E064E182E00E944C
:107610003E3940E0642F82E00E943E394FEF61E046
:1076200082E00E943E3940E062E0862F0E943E39AF
:1076300040E063E082E00E943E3940E064E082E0A6
:107640000E943E3940E065E082E00E943E3940E021
:107650006CE082E00E943E3940E06DE082E00E94F2
:107660003E394CE16AE083E00E943E3940E064E14B
:1076700083E00E943E3940E0642F83E00E943E395F
:107680004FEF61E083E00E943E3940E062E083E03A
:107690000E943E3940E063E0862F0E943E3940E080
:1076A00064E083E00E943E3940E065E083E00E94B0
:1076B0003E3940E06CE083E00E943E3940E06DE0FE
:1076C00083E00E943E394CE16AE084E00E943E394A
:1076D00040E064E184E00E943E394CEF60E084E0E9
:1076E0000E943E394FEF61E084E00E943E3940E065
:1076F00062E084E00E943E3940E063E084E00E9462
:107700003E3940E064E0862F0E943E3940E065E06B
:1077100084E00E943E3940E06CE084E00E943E3903
:1077200040E06DE084E00E943E394CE16AE085E093
:107730000E943E3940E064E185E00E943E3940E02D
:1077400065E185E00E943E3940E0642F85E00E94BB
:107750003E3940EF61E085E00E943E3940E062E062
:1077600085E00E943E3940E063E085E00E943E39BA
:1077700040E064E085E00E943E3940E065E0862F0D
:107780000E943E3940E06CE085E00E943E3940E0D6
:107790006DE085E00E943E3908950F931F93CF93CB
:1077A000082FC62F142F20E030E0613611F421E0BD
:1077B00030E080E090E0C13411F481E090E0822B71
:1077C000932B892B91F060E0812F0E94293921E0D1
:1077D00030E0002E02C0220F331F0A94E2F7482F38
:1077E000422B60E0812F0E943E3920E030E0C2361B
:1077F00011F421E030E080E090E0C23411F481E047
:1078000090E0822B932B892B89F061E0812F0E94DD
:10781000293921E030E002C0220F331F0A95E2F738
:10782000482F422B61E0812F0E943E39CF911F915A
:107830000F9108950F931F93CF93082FC62F142FE6
:1078400020E030E0613611F421E030E080E090E0AB
:10785000C13411F481E090E0822B932B892BA1F0AD
:1078600060E0812F0E94293921E030E0002E02C023
:10787000220F331F0A94E2F7922F9095482F492345
:1078800060E0812F0E943E3920E030E0C23611F4E2
:1078900021E030E080E090E0C23411F481E090E03B
:1078A000822B932B892B99F061E0812F0E9429393B
:1078B00021E030E002C0220F331F0A95E2F7922F39
:1078C0009095482F492361E0812F0E943E39CF9146
:1078D0001F910F9108950F931F93CF93182FC62FC9
:1078E000042F20E030E0613611F421E030E080E048
:1078F00090E0C13411F481E090E0822B932B892B2E
:1079000029F0412F64E1802F0E943E3920E030E0D1
:10791000C23611F421E030E080E090E0C23411F48E
:1079200081E090E0822B932B892B29F0412F65E198
:10793000802F0E943E39CF911F910F9108950F9390
:107940001F93CF93082FC62F142F50E020E030E074
:10795000613611F421E030E080E090E0C13411F4B0
:1079600081E090E0822B932B892B71F062E1812FD3
:107970000E94293921E030E0002E02C0220F331F7F
:107980000A94E2F7582F522B20E030E0C23611F46F
:1079900021E030E080E090E0C23411F481E090E03A
:1079A000822B932B892B69F063E1812F0E94293967
:1079B00021E030E002C0220F331F0A95E2F7582F72
:1079C000522B412F6C2F852F0E946B3CCF911F9122
:1079D0000F9108950F931F93CF93082FC62F142F45
:1079E00050E020E030E0613611F421E030E080E04A
:1079F00090E0C13411F481E090E0822B932B892B2D
:107A000081F062E1812F0E94293921E030E0002ECF
:107A100002C0220F331F0A94E2F7922F9095582F3D
:107A2000592320E030E0C23611F421E030E080E05C
:107A300090E0C23411F481E090E0822B932B892BEB
:107A400079F063E1812F0E94293921E030E002C002
:107A5000220F331F0A95E2F7922F9095582F592342
:107A6000412F6C2F852F0E946B3CCF911F910F915E
:107A700008951F93CF93C82F162F40E020E030E0E9
:107A8000813611F421E030E080E090E0C13411F45F
:107A900081E090E0822B932B892B29F062E1812FEA
:107AA0000E942939482F20E030E0C23611F421E04D
:107AB00030E080E090E0C23411F481E090E0822B6D
:107AC000932B892B29F063E1812F0E942939482FBC
:107AD000842F9927CF911F9108950F931F93CF93D0
:107AE000182FC62F042F40E020E030E0613611F45B
:107AF00021E030E080E090E0C13411F481E090E0DA
:107B0000822B932B892B29F062E1802F0E94293947
:107B1000482F20E030E0C23611F421E030E080E070
:107B200090E0C23411F481E090E0822B932B892BFA
:107B300029F063E1802F0E942939482F81E090E0ED
:107B400002C0880F991F1A95E2F784239927CF91D5
:107B50001F910F9108950E94361485E49AE0909346
:107B6000DC0A8093DB0A1092DD0A1092D40A10928C
:107B7000D50A84ED9AE00E943E148823D1F7109232
:107B8000D30A8DE49AE09093E80A8093E70A109272
:107B9000E90A1092E00A1092E10A80EE9AE00E944F
:107BA0003E148823D1F71092DF0A85E59AE090937E
:107BB000F40A8093F30A1092F50A1092EC0A1092DC
:107BC000ED0A8CEE9AE00E943E148823D1F71092C1
:107BD000EB0A8DE59AE09093000B8093FF0A1092D8
:107BE000010B1092F80A1092F90A88EF9AE00E94AD
:107BF0003E148823D1F71092F70A85EF99E090930D
:107C00006D0A80936C0A10926E0A1092650A82E0E7
:107C10008093660A85E69AE00E943E148823D1F795
:107C20008DEF99E09093780A8093770A1092790A01
:107C30001092700A82E08093710A80E79AE00E94B5
:107C40003E148823D1F785E09AE09093830A8093CD
:107C5000820A1092840A10927B0A82E080937C0A46
:107C60008BE79AE00E943E148823D1F78DE09AE0DA
:107C700090938E0A80938D0A10928F0A1092860A32
:107C800082E08093870A86E89AE00E943E14882367
:107C9000D1F785E19AE09093990A8093980A10921F
:107CA0009A0A1092910A82E08093920A81E99AE0FE
:107CB0000E943E148823D1F78DE19AE09093A40AA4
:107CC0008093A30A1092A50A10929C0A82E08093E6
:107CD0009D0A8CE99AE00E943E148823D1F785E240
:107CE0009AE09093AF0A8093AE0A1092B00A109275
:107CF000A70A82E08093A80A87EA9AE00E943E14CD
:107D00008823D1F78DE29AE09093BA0A8093B90A5A
:107D10001092BB0A1092B20A82E08093B30A82EBFF
:107D20009AE00E943E148823D1F785E39AE090936D
:107D3000C50A8093C40A1092C60A1092BD0A82E056
:107D40008093BE0A8DEB9AE00E943E148823D1F7FF
:107D50008DE39AE09093D00A8093CF0A1092D10AD3
:107D60001092C80A82E08093C90A88EC9AE00E94C7
:107D70003E148823D1F708958091D30A8823E1F037
:107D80008091D30A813059F483ED9AE001960E94E4
:107D90003E14882389F482E08093D30A0DC0809139
:107DA000D30A823049F483ED9AE001960E9450157F
:107DB000882311F48093D30A8091DF0A8823E1F0AD
:107DC0008091DF0A813059F48FED9AE001960E948C
:107DD0003E14882389F482E08093DF0A0DC08091ED
:107DE000DF0A823049F48FED9AE001960E94501527
:107DF000882311F48093DF0A8091EB0A8823E1F055
:107E00008091EB0A813059F48BEE9AE001960E9442
:107E10003E14882389F482E08093EB0A0DC08091A0
:107E2000EB0A823049F48BEE9AE001960E945015DD
:107E3000882311F48093EB0A8091F70A8823E1F0FC
:107E40008091F70A813059F487EF9AE001960E94F9
:107E50003E14882389F482E08093F70A0895809184
:107E6000F70A823049F487EF9AE001960E94501594
:107E7000882311F48093F70A0895CF93DF93EC01E0
:107E800085E69AE00E945015882309F046C080914B
:107E9000670A9091680AAA27BB2788839983AA83D7
:107EA000BB83E0916C0AF0916D0A80818D83E09133
:107EB0006C0AF0916D0A81818E83E0916C0AF091D9
:107EC0006D0A82818F83E0916C0AF0916D0A838143
:107ED0008887E0916C0AF0916D0A84818987E0912E
:107EE0006C0AF0916D0A85818A87E0916C0AF091A5
:107EF0006D0A86818B87E0916C0AF0916D0A87810B
:107F00008C8780916B0A8C8385E69AE00E943E14F0
:107F10008823D1F781E090E0BBC280E79AE00E941D
:107F20005015882309F046C08091720A9091730A17
:107F3000AA27BB2788839983AA83BB83E091770A0A
:107F4000F091780A80818D83E091770AF091780A28
:107F500081818E83E091770AF091780A82818F8304
:107F6000E091770AF091780A83818887E091770A17
:107F7000F091780A84818987E091770AF091780AF4
:107F800085818A87E091770AF091780A86818B87CC
:107F9000E091770AF091780A87818C878091760A40
:107FA0008C8380E79AE00E943E148823D1F781E019
:107FB00090E06EC28BE79AE00E945015882309F08A
:107FC00046C080917D0A90917E0AAA27BB278883AC
:107FD0009983AA83BB83E091820AF091830A80810E
:107FE0008D83E091820AF091830A81818E83E091F2
:107FF000820AF091830A82818F83E091820AF09154
:10800000830A83818887E091820AF091830A8481C0
:108010008987E091820AF091830A85818A87E091BD
:10802000820AF091830A86818B87E091820AF0911F
:10803000830A87818C878091810A8C838BE79AE001
:108040000E943E148823D1F781E090E021C286E8A7
:108050009AE00E945015882309F046C08091880A52
:108060009091890AAA27BB2788839983AA83BB8317
:10807000E0918D0AF0918E0A80818D83E0918D0AC6
:10808000F0918E0A81818E83E0918D0AF0918E0AA3
:1080900082818F83E0918D0AF0918E0A8381888797
:1080A000E0918D0AF0918E0A84818987E0918D0A92
:1080B000F0918E0A85818A87E0918D0AF0918E0A6F
:1080C00086818B87E0918D0AF0918E0A87818C875B
:1080D00080918C0A8C8386E89AE00E943E14882363
:1080E000D1F781E090E0D4C181E99AE00E94501577
:1080F000882309F046C08091930A9091940AAA2798
:10810000BB2788839983AA83BB83E091980AF09167
:10811000990A80818D83E091980AF091990A818172
:108120008E83E091980AF091990A82818F83E09181
:10813000980AF091990A83818887E091980AF091D2
:10814000990A84818987E091980AF091990A85813A
:108150008A87E091980AF091990A86818B87E0914D
:10816000980AF091990A87818C878091970A8C836D
:1081700081E99AE00E943E148823D1F781E090E0E3
:1081800087C18CE99AE00E945015882309F046C007
:1081900080919E0A90919F0AAA27BB278883998382
:1081A000AA83BB83E091A30AF091A40A80818D8306
:1081B000E091A30AF091A40A81818E83E091A30A41
:1081C000F091A40A82818F83E091A30AF091A40A1E
:1081D00083818887E091A30AF091A40A848189872A
:1081E000E091A30AF091A40A85818A87E091A30A0D
:1081F000F091A40A86818B87E091A30AF091A40AEA
:1082000087818C878091A20A8C838CE99AE00E94F6
:108210003E148823D1F781E090E03AC187EA9AE0E2
:108220000E945015882309F046C08091A90A9091B8
:10823000AA0AAA27BB2788839983AA83BB83E091D4
:10824000AE0AF091AF0A80818D83E091AE0AF09181
:10825000AF0A81818E83E091AE0AF091AF0A8281EC
:108260008F83E091AE0AF091AF0A83818887E09115
:10827000AE0AF091AF0A84818987E091AE0AF0914D
:10828000AF0A85818A87E091AE0AF091AF0A8681B4
:108290008B87E091AE0AF091AF0A87818C8780913D
:1082A000AD0A8C8387EA9AE00E943E148823D1F7B6
:1082B00081E090E0EDC082EB9AE00E9450158823A7
:1082C00009F046C08091B40A9091B50AAA27BB274D
:1082D00088839983AA83BB83E091B90AF091BA0A93
:1082E00080818D83E091B90AF091BA0A81818E83F1
:1082F000E091B90AF091BA0A82818F83E091B90ABC
:10830000F091BA0A83818887E091B90AF091BA0A9C
:1083100084818987E091B90AF091BA0A85818A87B8
:10832000E091B90AF091BA0A86818B87E091B90A87
:10833000F091BA0A87818C878091B80A8C8382EB8E
:108340009AE00E943E148823D1F781E090E0A0C01B
:108350008DEB9AE00E945015882309F046C0809169
:10836000BF0A9091C00AAA27BB2788839983AA8352
:10837000BB83E091C40AF091C50A80818D83E091AE
:10838000C40AF091C50A81818E83E091C40AF091FC
:10839000C50A82818F83E091C40AF091C50A838166
:1083A0008887E091C40AF091C50A84818987E091A9
:1083B000C40AF091C50A85818A87E091C40AF091C8
:1083C000C50A86818B87E091C40AF091C50A87812E
:1083D0008C878091C30A8C838DEB9AE00E943E14B7
:1083E0008823D1F781E090E053C088EC9AE00E94A6
:1083F0005015882309F046C08091CA0A9091CB0A93
:10840000AA27BB2788839983AA83BB83E091CF0ADD
:10841000F091D00A80818D83E091CF0AF091D00A4B
:1084200081818E83E091CF0AF091D00A82818F837F
:10843000E091CF0AF091D00A83818887E091CF0A3A
:10844000F091D00A84818987E091CF0AF091D00A17
:1084500085818A87E091CF0AF091D00A86818B8747
:10846000E091CF0AF091D00A87818C878091CE0A63
:108470008C8388EC9AE00E943E148823D1F781E037
:1084800090E006C0188219821A821B8280E090E078
:10849000DF91CF910895CF93DF93DC018091D30AD0
:1084A000882339F483ED9AE09093040B8093030BB7
:1084B00021C08091DF0A882339F48FED9AE09093F0
:1084C000040B8093030B16C08091EB0A882339F4C8
:1084D0008BEE9AE09093040B8093030B0BC080917A
:1084E000F70A882309F072C087EF9AE09093040B93
:1084F0008093030BE091030BF091040B0084F18552
:10850000E02DED018D818083E091030BF091040B50
:108510000084F185E02D8E818183E091030BF09141
:10852000040B0084F185E02D8F818283E091030BA1
:10853000F091040B0084F185E02D88858383E09120
:10854000030BF091040B0084F185E02D8985848371
:10855000E091030BF091040B0084F185E02D8A85F6
:108560008583E091030BF091040B0084F185E02DED
:108570008B858683E091030BF091040B0084F185D9
:10858000E02D8C858783E091030BF091040B8C81A7
:108590008783E091030BF091040B8D919C91948360
:1085A0008383E091030BF091040B1286E091030B9F
:1085B000F091040B1182E091030BF091040B1282F5
:1085C000E091030BF091040B81E08083DF91CF9168
:1085D000089588EE99E00E943D3F882361F188EE7E
:1085E00099E00E94DC1188EE99E00E943D3F8823CB
:1085F00011F188EE99E00E94DC1188EE99E00E946A
:108600003D3F8823C1F088EE99E00E94DC1188EE9E
:1086100099E00E943D3F882371F088EE99E00E9426
:10862000DC1188EE99E00E943D3F882321F088EE1E
:1086300099E00E94DC110895FF920F931F93CF934E
:10864000DF93CDB7DEB760970FB6F894DEBF0FBEED
:10865000CDBF20E0822F99278C010B5F144FF801CA
:1086600080818C7F8083F22EF394BE016F5F7F4FF9
:108670008F2D0E942E3588898170982F990F990F20
:10868000990FF80180818370892B80832F2D2B30E7
:1086900008F360960FB6F894DEBF0FBECDBFDF9132
:1086A000CF911F910F91FF900895FC0180818370FD
:1086B0009927009719F0019731F0089580818D7204
:1086C0008162808308959081892F807FA1F493FD3A
:1086D00005C0892F8E7F866080830895808182FF08
:1086E00003C08B7F808303C080818460808380810E
:1086F0008C7F826080830895FC018081837099273C
:1087000081309105BCF0833091051CF0039731F066
:10871000089580818F708362808308959081892F6E
:10872000807F41F4892F8C7F808393FD03C0892F44
:10873000887F808308959927853C910509F457C067
:10874000863C9105ACF4823C9105C9F1833C9105CE
:108750003CF4803C910519F1813C910541F17AC0CE
:10876000833C910509F45EC0843C9105C1F172C05F
:10877000813D910561F1823D910544F4863C91056E
:10878000F1F1873C910509F442C064C0823D910536
:1087900009F450C0833D910509F454C05BC0309B7F
:1087A00003C081E090E0089580E090E00895319961
:1087B00003C081E090E0089580E090E00895329950
:1087C00003C081E090E0089580E090E00895499929
:1087D00003C081E090E0089580E090E0089534992E
:1087E00003C081E090E0089580E090E0089535991D
:1087F00003C081E090E0089580E090E0089536990C
:1088000003C081E090E0089580E090E0089586B193
:10881000992787FD9095809590958827990F881FB7
:1088200099270895339903C081E090E0089580E08E
:1088300090E008954A9903C081E090E0089580E0B7
:1088400090E008954B9903C081E090E0089580E0A6
:1088500090E0089580E090E0089530E0832F99271C
:10886000FC01EB5FF44F2081822F807F41F0822F4B
:10887000807F982F9051822F8F70892B80833F5F4C
:108880003B3060F3E5E0FBE0309B04C0CF010E9489
:10889000554303C0CF010E947C43E6E0FBE03199E1
:1088A00004C0CF010E94554303C0CF010E947C4306
:1088B000E7E0FBE0329904C0CF010E94554303C0BA
:1088C000CF010E947C43E8E0FBE0499904C0CF015E
:1088D0000E94554303C0CF010E947C43E9E0FBE0C6
:1088E000349904C0CF010E94554303C0CF010E94B8
:1088F0007C43EAE0FBE0359904C0CF010E94554378
:1089000003C0CF010E947C43EBE0FBE0369904C03A
:10891000CF010E94554303C0CF010E947C43ECE08D
:10892000FBE0379904C0CF010E94554303C0CF013B
:108930000E947C43EDE0FBE0339904C0CF010E942C
:10894000554303C0CF010E947C43EEE0FBE04A990F
:1089500004C0CF010E94554303C0CF010E947C4355
:10896000EFE0FBE04B9904C0CF010E94554308950E
:10897000CF010E947C4308959927853C910509F415
:1089800051C0863C9105ACF4823C9105B1F1833C29
:1089900091053CF4803C910511F1813C910531F148
:1089A0006BC0833C910509F452C0843C910599F158
:1089B00063C0813D910541F1823D91053CF4863CC7
:1089C0009105B9F1873C9105D9F156C0823D9105D9
:1089D00009F444C0833D910509F447C04DC080911E
:1089E000050B869586958170992708958091060BD1
:1089F000869586958170992708958091070B8695B5
:108A000086958170992708958091080B86958695A3
:108A10008170992708958091090B869586958170BC
:108A20009927089580910A0B8695869581709927DC
:108A3000089580910B0B86958695817099270895EE
:108A400080910C0B86958695817099270895809169
:108A50000D0B8695869581709927089580910E0B50
:108A60008695869581709927089580910F0B86953C
:108A700086958170992708958EEF90E00895109261
:108A8000B60087E08093B0001092B2008EE480932D
:108A9000B30082E08093700008950E943F451092D9
:108AA000120B1092130B1092140B1092150B1092C4
:108AB0001A0B10921B0B0E941C430E94E4050E949B
:108AC000B5300895CF93C82F8091100B882311F0F3
:108AD0001092100BA8950E94E942C23011F00E943A
:108AE000BC3EC23009F471C08091110B882309F497
:108AF00046C08091110B81508093110B0E94241667
:108B00008091120B8F5F8093120B823040F0109295
:108B1000120B0E942D440E941B170E941E07809179
:108B2000130B8F5F8093130B843040F01092130B64
:108B30000E9499170E94DD560E94E8538091140B01
:108B40008F5F8093140B8A3030F01092140BC13079
:108B500011F00E94C4118091150B8F5F8093150B4B
:108B6000843168F01092150B80911A0B8F5F8093FF
:108B70001A0B0E9455390E94C1180E9479118091E8
:108B80001A0B8A3010F110921A0B8091160B9091EB
:108B9000170BA091180BB091190B0196A11DB11DD7
:108BA0008093160B9093170BA093180BB093190B8F
:108BB0000E94BD3180911B0B8F5F80931B0B8C3308
:108BC00020F010921B0B0E947C31CF910895809170
:108BD000160B9091170BA091180BB091190BBC01BB
:108BE000CD0108951F920F920FB60F9211248F930B
:108BF0001092B20081E08093100B8091110B8F5F77
:108C00008093110B8F910F900FBE0F901F901895AE
:108C10000E9487520E943A5460E076E980E090E03A
:108C20000E945554089504C00E94CD520E942053C2
:108C30000E94B7528823C1F70895FC0190E061506B
:108C40006F3F21F0819198276150E0F7892F992794
:108C500008950F931F938C01FC0181818150682F2F
:108C6000C80101960E941D46F801808381819927E1
:108C7000BC01C8010E94E8521F910F910895AF9264
:108C8000BF92CF92DF92EF92FF920F931F93CF93F9
:108C9000DF93CDB7DEB7C35ED0400FB6F894DEBF2A
:108CA0000FBECDBF6C01FC0181818150682FC601D0
:108CB00001960E941D46D6019C91981711F00C94C4
:108CC0001552F6018281882309F0F8C08381992723
:108CD0008135910509F449C0823591053CF4803312
:108CE000910589F08035910561F1E8C083359105E2
:108CF00009F48EC0833591050CF478C08435910554
:108D000009F4B2C0DBC08E01035D1F4F80E5D801BE
:108D10001D928A95E9F785E18EA71FA680E888ABAA
:108D2000F601848189AB992796012B5F3F4FAC01F7
:108D3000B901CE01C2960E94C365C8010E942946AE
:108D4000BDC08E01035D1F4F80E5D8011D928A953D
:108D5000E9F785E08EA71FA680EA88AB0E94432F23
:108D600089ABC8010E942946A9C0F601B4800F2E24
:108D7000FDE2EF2EFF24F02DEC0EFD1E80E5D70165
:108D80001D928A95E9F789E18EA71FA681EA88AB33
:108D90008E0103581F4FB8018B2D0E946D2FB9AA69
:108DA0008CE0FE01F296D8010D9001928A95E1F7D0
:108DB000F801848595859FAF8EAF8685FE01E05CC6
:108DC000FF4F8083F8018785FE01EF5BFF4F8083B3
:108DD0009927AC01BE0163577F4FCE018E5B9F4F39
:108DE0000E94C365C7010E94294668C00E94FB2EED
:108DF000FE01BD9680E5DF011D928A95E9F784E0CA
:108E00008EA71FA682EA88ABCF010E94294656C0D2
:108E1000F601458156818481FE01ED51FF4F80832B
:108E2000813108F04BC080E5FE01BD9611928A9514
:108E3000E9F787E18EA71FA683EA88AB5BAB4AAB55
:108E4000FE01ED51FF4F808189ABFE01F496992719
:108E5000DA01019724F00E94A7660192FACFCE01B1
:108E60008D960E9429462AC0F6014581568184814B
:108E7000FE01ED51FF4F8083813100F5F6013796F9
:108E80009927DA01019724F001900E94B466FACF85
:108E9000DE019D9680E5FD0111928A95E9F787E054
:108EA0008EA71FA684EA88AB5BAB4AABFE01ED51EF
:108EB000FF4F808189ABCD010E942946F601828156
:108EC000813011F00C941E5283819927AA27BB2769
:108ED000FC013197EB36F10510F00C940752E65B7C
:108EE000FF4FEE0FFF1F0590F491E02D09940E94B3
:108EF000532DF601B4808B2D8150823210F00C94EA
:108F00001E5220E0AE01475F5F4F822F9927DA01A2
:108F1000A80FB91FF601E80FF91F82858C932F5F08
:108F20002F3098F3F6018581898386818A83878132
:108F30008B83838D948D9E838D83858D8F83808598
:108F4000888781858C83818D888F828D898F6B2D19
:108F5000CE0101960E947A346B2DCE0101960E94BB
:108F6000BE201DA685E08EA711E01FA781E888AB73
:108F700019AACE018D960E942946812F0E94624532
:108F80000C941E52F601B4808B2D8150823208F071
:108F900047C06B2DCE0101960E94BF348EE18EA793
:108FA00081E08FA782E888ABB9AA89818AAB8A81E0
:108FB0008BAB8B818CAB8C818EAB8D819E81FE01C6
:108FC000E85BFF4F918380838F81FE01E65BFF4F5B
:108FD000808320E0BE016F5F7F4FAE01475F5F4F30
:108FE000822F9927DC01A60FB71FFA01E80FF91F9E
:108FF0008081FD0186AB2F5F2F3090F388858DAB8C
:10900000888DFE01EA5BFF4F8083898DFE01E95B5D
:10901000FF4F8083CE018D960E9429460C941E52EC
:10902000FFEFBF1611F00C941E52FE01ED51FF4FE1
:109030001082FE01ED51FF4F8081982F823210F097
:109040000C941E520F2EF3EEEF2EFF24F02DEC0E9B
:10905000FD1E6E010894C11CD11C8E01075F1F4FBD
:10906000892F8F5F682FCE0101960E94BF348EE159
:109070008EA781E08FA782E888ABD7018C918F5FA4
:1090800089AB89818AAB8A818BAB8B818CAB8C81DC
:109090008EAB8D819E81FE01E85BFF4F91838083C3
:1090A0008F81FE01E65BFF4F808320E0822F9927AE
:1090B000DC01AC0DBD1DF801E80FF91F8081FD0139
:1090C00086AB2F5F2F3090F388858DAB888DFE01A6
:1090D000EA5BFF4F8083898DFE01E95BFF4F808350
:1090E000CE018D960E94294681E00E946245D701FB
:1090F0008C918F5F8C93982F823208F4B1CF0C94AF
:109100001E520E94532DF601B480AE0143585F4FAA
:1091100096012B5F3F4F8FE0DA01F90101900D922C
:109120008A95E1F7F6018489FA018787BA018B2DC8
:109130000E94113581E08FA783E888ABB9AA85E04A
:109140008EA7CE018D960E9429460C941E52F601E0
:10915000B4808B2D81508A3010F581E08FA784E890
:1091600088ABB9AA8E0103581F4FB8018B2D0E94FE
:109170002E358FE0FE01F296D8010D9001928A956E
:10918000E1F7F8018785FE01EF5BFF4F808385E102
:109190008EA7CE018D960E9429460C941E52FFEF99
:1091A000BF1611F00C941E52FE01ED51FF4F1082BC
:1091B000FE01ED51FF4F8081982F8B3010F00C9401
:1091C0001E52BB24B3948E0103581F4F0F2EFFE095
:1091D000AF2EF02D0F2EF1E4EF2EFF24F02DEC0E2C
:1091E000FD1E0F2EF3EECF2EDD24F02DCC0EDD1E56
:1091F000BFA684E888AB892F8F5F89ABB8010E9436
:109200002E35FE01F296D8012A2D0D9001922A9555
:10921000E1F7F8018785D7018C9385E18EA7CE0110
:109220008D960E9429468B2D0E946245F601808111
:109230008F5F8083982F8B30D8F20C941E520E943F
:10924000532D0E94561BA8950E94641EA8950E944B
:10925000CC1FA8950E94DF10A8950E94A956A8953A
:109260000E943B06A8950E9422310E945D0F81E07A
:109270008FA786E888AB84E08EA7CE018D960E94EA
:1092800029460C941E5284E18EA781E08FA787E8BF
:1092900088AB8DE0A7E7B1E0FE01F1960D90019259
:1092A0008A95E1F70E94E7459B01AC01AA27BB27FD
:1092B0008EAFBB27A52F942F832F8FAFFE01E05CCD
:1092C000FF4F2083CE018D960E9429460C941E529A
:1092D0000C9400000C941E52C60104960E940833A0
:1092E00081E08FA789E888AB84E08EA7CE018D96B8
:1092F0000E9429460C941E5281E08FA78AE888AB11
:109300008CE08EA7CE01C1960E941833CE018D96B7
:109310000E9429460C941E52CE0187960E949F2AD5
:1093200081E08FA781EA88AB8FA189AB88A58AAB42
:1093300089A58BAB8AA58CAB8BA58DAB8CA58EAB91
:109340008AE08EA7CE018D960E9429460C941E526B
:10935000F601B480F1E2FB1500F1BE016E5D7F4FB6
:109360008B2D0E94912B81E08FA782EA88ABB9AA4E
:109370008BA18BAB8CA18EAB8AA18AAB8DA19EA158
:10938000892F99278CAB8DA18DAB8AE08EA7CE015A
:109390008D960E9429460C941E522FEFB21611F0A2
:1093A0000C941E52FE01ED51FF4F1082FE01ED5153
:1093B000FF4F8081982F823210F00C941E52FF24B0
:1093C000F3948F01BE016E5D7F4F892F8F5F0E94E6
:1093D000912BFFA682EA88ABD8018C918F5F89AB75
:1093E0008BA18BAB8CA18EAB8AA18AAB8DA19EA1E8
:1093F000892F99278CAB8DA18DAB8AE08EA7CE01EA
:109400008D960E9429468F2D0E946245F801808129
:109410008F5F8083982F8232A8F20C941E52CE0167
:109420004A960E945B2C8AE08EA781E08FA780EA93
:1094300088AB88A189AB8E8D8AAB8A8D9B8D892F55
:1094400099278BAB8A8D8CAB8D8D8DAB8C8D8EAB34
:10945000CE018D960E9429460C941E52F60164811D
:1094600080E00E947A2384E08EA781E08FA783EAC0
:1094700088ABCE018D960E942946E0C7DE01A3533A
:10948000BF4FF60184818C938581FD018183F601B4
:109490008681FD018283F6018781FD018383F601C8
:1094A0008085FD018483F6018185FD018583F601B8
:1094B0008285FD018683F6018385FD018783CD01C9
:1094C0000E94822384E08EA781E08FA784EA88AB84
:1094D000CE018D960E942946B1C7FE01E358FF4F89
:1094E000A0E0B0E080E190E021E08030920719F444
:1094F0000E94AF6603C0182E0E94AF66F6018481F9
:109500009581A681B781FE01EF57FF4F808391833C
:10951000A283B383DE01A358BF4FF6018085FD010E
:109520008087F6018185FD018187F6018285FD0135
:109530008287A0E0B0E080E190E021E080309207F7
:1095400019F40E94C06603C0182E0E94C06684E011
:109550008EA781E08FA780EC88ABCE018D960E940C
:1095600029466CC7FE01E358FF4FA0E0B0E080E160
:1095700090E021E08030920719F40E94AF6603C0AA
:10958000182E0E94AF668BE08EA781E08FA781EC3A
:1095900088ABFE01EF57FF4F80819181A281B3819B
:1095A00089AB9AABABABBCABFE01E358FF4F8085F8
:1095B0008DAB81858EAB82858FABCE018D960E945F
:1095C00029463CC78AE38EA781E08FA780ED88AB50
:1095D000FE01F196A8E8B0E082E190E021E0803061
:1095E000920719F40E94AF6603C0182E0E94AF665E
:1095F000FE01ED5BFF4FAAE9B0E082E190E021E0DF
:109600008030920719F40E94AF6603C0182E0E94A2
:10961000AF66FE01EB5AFF4FADEBB0E082E190E0A8
:1096200021E08030920719F40E94AF6603C0182E23
:109630000E94AF66CE018D960E942946FFC684E146
:109640008EA781E08FA78EED88ABFE01F196ACEA84
:10965000B0E080E190E021E08030920719F40E94B0
:10966000AF6603C0182E0E94AF66CE018D960E9491
:109670002946E4C60E94223184E08EA781E08FA7AC
:1096800081ED88ABCE018D960E942946D7C688E031
:109690008EA781E08FA78FED88AB0E94B4318BAB92
:1096A0000E94B8319AAB89ABFE01ED51FF4FACEB94
:1096B000B0E081E090E021E08030920719F40E9450
:1096C000AF6603C0182E0E94AF66FE01ED51FF4F3A
:1096D00080818CABCE018D960E942946AFC6FE01DB
:1096E000E358FF4F80E5DF011D928A95E9F7ACEB67
:1096F000B0E081E090E021E08030920719F40E9410
:10970000C06603C0182E0E94C066FE01E358FF4FDA
:10971000A5E8B0E081E090E021E08030920719F404
:109720000E94C06603C0182E0E94C066FE01E35866
:10973000FF4FA6E8B0E082E090E021E080309207A1
:1097400019F40E94C06603C0182E0E94C06684E00F
:109750008EA781E08FA780EE88ABCE018D960E9408
:1097600029466CC6F601858196819093660E80939A
:10977000650E878190859093680E8093670E818532
:10978000928590936A0E8093690E838580936B0E09
:10979000848580936C0E858580936D0E8785908976
:1097A0009093700E80936F0E868580936E0E8189E4
:1097B0008093710E82898093720E83898093730ED9
:1097C000E5E6FEE0A0E7B0E08FE090E021E0803049
:1097D000920719F40E94C06603C0182E0E94C0664A
:1097E00085E08EA791E09FA785EA88AB99ABCE0173
:1097F0008D960E94294622C684E18EA781E08FA71C
:1098000086EA88AB19AA8091E200863269F48091D9
:10981000E300843049F48091E400833129F484E644
:1098200090E09BAB8AAB46C08091E2008E3169F438
:109830008091E300843049F48091E400833129F47D
:109840008DE790E09BAB8AAB35C08091E2008E3013
:1098500069F48091E300843049F48091E40083311D
:1098600029F48AEF90E09BAB8AAB24C08091E200A0
:10987000863069F48091E300843049F48091E400FB
:10988000833129F484EF91E09BAB8AAB13C08091C4
:10989000E200823069F48091E300843049F48091E1
:1098A000E400833129F488EE93E09BAB8AAB02C0DD
:1098B0001BAA1AAA8091670E9091680E9DAB8CAB83
:1098C0008091690E90916A0E9FAB8EAB80916B0E6A
:1098D00088AF80916C0E89AF80916D0E8AAF8091B8
:1098E0006F0E9091700E9DAF8CAF80916E0E8BAF0E
:1098F0008091710E8EAF8091720E8FAF8091730E3A
:10990000FE01E05CFF4F8083CE018D960E942946C8
:1099100095C5DE01AB52BF4FF60184818C938581E2
:10992000FD018183D60116968CE0FE01E952FF4FBE
:109930000D9001928A95E1F7FE01ED51FF4F1082E3
:10994000FE01ED51FF4F8081982F8C30A0F49E01D5
:109950002B523F4FDF01F901E90FF11D828188236E
:1099600021F08F3F11F0815082838C918F5F8C9317
:10997000982F8C3080F3CE018B529F4F0E94BA32C9
:1099800084E08EA781E08FA787EA88ABCE018D9611
:109990000E94294653C58E010B521F4FC8010E94D9
:1099A000D83282E18EA781E08FA788EA88ABD80100
:1099B0008C9189ABF80181818AABFE01ED51FF4F9B
:1099C0001082FE01ED51FF4F8081982F8C3080F482
:1099D0009801DF01F901E90FF11D82818F3F11F03C
:1099E0008F5F82838C918F5F8C93982F8C3090F354
:1099F0008CE0DE01A952BF4FFE01F3960D9001925B
:109A00008A95E1F7CE018D960E94294617C5F60189
:109A10008481FE01E358FF4F8083D60115968EE0C6
:109A2000FE01E258FF4F0D9001928A95E1F7FE0189
:109A3000ED51FF4F1082FE01ED51FF4F8081982FB5
:109A40008E30A0F49E0123583F4FDF01F901E90F4A
:109A5000F11D8181882321F08F3F11F08150818396
:109A60008C918F5F8C93982F8E3080F3DE01A358FA
:109A7000BF4FF6018389FD018787F6018489FD01C7
:109A8000808BD60155968EE0FE01E257FF4F0D9078
:109A900001928A95E1F7FE01ED51FF4F1082FE0120
:109AA000ED51FF4F8081982F8E30A0F49E012358F6
:109AB0003F4FDF01F901E90FF11D8189882321F072
:109AC0008F3F11F08150818B8C918F5F8C93982FF9
:109AD0008E3080F3CE0183589F4F0E94E83284E09D
:109AE0008EA781E08FA789EA88ABCE018D960E9470
:109AF0002946A4C48E0103581F4FC8010E94F832A2
:109B000083E28EA781E08FA78AEA88ABD8018C9187
:109B100089ABFE01ED51FF4F1082FE01ED51FF4F69
:109B20008081982F8E3080F49801DF01F901E90FD0
:109B3000F11D81818F3F11F08F5F81838C918F5F49
:109B40008C93982F8E3090F38EE0DE01A258BF4F99
:109B5000FE01F2960D9001928A95E1F7DE01A3587D
:109B6000BF4FFD018785FE01E05CFF4F8083FD0153
:109B70008089FE01EF5BFF4F8083FE01ED51FF4FB7
:109B80001082FE01ED51FF4F8081982F8E3080F4BE
:109B90009D01DF01F901E90FF11D81898F3F11F06E
:109BA0008F5F818B8C918F5F8C93982F8E3090F389
:109BB0008EE0DE01A257BF4FFE01EE5BFF4F0D901E
:109BC00001928A95E1F7CE018D960E94294636C40E
:109BD000F601B48085819927982F88272681820FE6
:109BE000911DBC018B2D0E94D62C85E08EA781E0B3
:109BF0008FA782EC88ABB9AACE018D960E94294628
:109C00001DC4F601B4808CE08EA781E08FA783ECA1
:109C100088ABB9AA8B2D0E94942C8AAB8B2D0E9405
:109C2000B02C892F99278BAB8B2D0E94B02C8CAB3D
:109C30008B2D0E94FF2C892F99278DAB8B2D0E9495
:109C4000FF2C8EAB8B2D0E94172D892F99278FAB60
:109C50008B2D0E94172D88AFCE018D960E9429462C
:109C6000EDC320E0F601848181FD21E0F6018481CD
:109C700082FD2260F6018181863029F46581822F80
:109C80000E942F2DDBC360E0822F0E942F2DD6C3B0
:109C90000E94342D84E08EA781E08FA785EC88ABED
:109CA000CE018D960E942946C9C3F601B4809E015B
:109CB00023583F4F9581492F4170D9018C91887F5E
:109CC0009670842B892B8C9386819781F9019283DE
:109CD0008183F60180859185F90194838383F60160
:109CE0008685F9018187F6018785F9018287F6016A
:109CF00082859385F90196838583F6018485958510
:109D0000F90190878783F6018089F9018387F6013D
:109D10008189F9018487F6018289F9018587F60135
:109D20008389F9018687D60154968FE0FE01E457B6
:109D3000FF4F0D9001928A95E1F7F60183A1F90199
:109D4000868FF60184A1F901878FF60185A1F901BB
:109D500080A3F60186A1F90181A315E0D6019796AB
:109D6000FE01E156FF4F812F0D9001928A95E1F798
:109D7000F60184A595A5A6A5B7A5F90187A390A787
:109D8000A1A7B2A7F60180A9F90183A7B9018B2D7C
:109D90000E949A3381E08FA782ED88AB1EA7B9AAF3
:109DA000CE018D960E94294649C3F601B4808E01EA
:109DB00003581F4FB8018B2D0E94D23381E08FA72B
:109DC00083ED88AB81E38EA7B9AAD8019C91292F96
:109DD00021708AA9887F9670822B892B8AABF80123
:109DE000818192819CAB8BAB838194819EAB8DAB47
:109DF00081858BAF82858CAF8581968198AF8FAB43
:109E0000878190859AAF89AF83858DAF84858EAF2A
:109E100085858FAF8685FE01E05CFF4F80838FE0F4
:109E2000DE01A457BF4FFE01EF5BFF4F0D90019283
:109E30008A95E1F7F801868DFE01E05BFF4F808394
:109E4000F801878DFE01EF5AFF4F8083F80180A152
:109E5000FE01EE5AFF4F8083F80181A1FE01ED5A09
:109E6000FF4F808385E0DE01A156BF4FFE01EC5A13
:109E7000FF4F0D9001928A95E1F7F80187A190A517
:109E8000A1A5B2A5FE01E75AFF4F80839183A2836B
:109E9000B383F80183A5FE01E35AFF4F8083CE010F
:109EA0008D960E942946CAC2F601B480AE0143587D
:109EB0005F4F828DDA018C93838DFA018183F601E5
:109EC000848DFA018283F6018681FA018383F6018B
:109ED0008781FA018483F6018085FA018583F60182
:109EE0008185FA018683F6018285FA018783F6016E
:109EF000858DFA01878BC6010B962FE0FE01EB578B
:109F0000FF4FDC010D9001922A95E1F7BA018B2DEC
:109F10000E940A3481E08FA784ED88AB85E08EA78C
:109F2000B9AACE018D960E94294688C2F601B48056
:109F30008E0103581F4FB8018B2D0E94423481E0DF
:109F40008FA785ED88AB8FE18EA7B9AAD8018C9138
:109F5000FE01E95BFF4F8083F8018181FE01E85B30
:109F6000FF4F8083F8018281FE01E75BFF4F808312
:109F7000F80183818BAB84818CAB85818DAB86812D
:109F80008EAB87818FAB8789FE01E65BFF4F8083B5
:109F90008FE0DE01AB57BF4FFE01F8960D900192A6
:109FA0008A95E1F7CE018D960E94294647C2F601B7
:109FB0003496AAEEB8E082E090E021E0803092078B
:109FC00019F40E94C06603C0182E0E94C06681E08A
:109FD0008FA783EE88AB84E08EA7CE018D960E947A
:109FE00029462CC281E08FA784EE88AB84E18EA73E
:109FF000FE01F196AAEEB8E082E090E021E0803028
:10A00000920719F40E94AF6603C0182E0E94AF6633
:10A01000CE018D960E94294611C2F601B480C60178
:10A020000596BC018B2D0E94283381E08FA788ED17
:10A0300088AB85E08EA7B9AACE018D960E942946ED
:10A04000FDC1F601B48081E08FA789ED88AB8EE178
:10A050008EA7B9AABE016E5C7F4F8B2D0E94613323
:10A06000CE018D960E942946E9C1F6018481809334
:10A07000790E858180937A0E868180937B0E87810D
:10A0800080937C0E808580937D0E818580937E0EEB
:10A09000828580937F0E83858093800EE9E7FEE0C2
:10A0A000AEE6BFE088E090E021E08030920719F44E
:10A0B0000E94C06603C0182E0E94C06681E08FA770
:10A0C00085EE88AB84E08EA7CE018D960E9429464E
:10A0D000B5C181E08FA786EE88AB8CE08EA780911A
:10A0E000790E89AB80917A0E8AAB80917B0E8BAB17
:10A0F00080917C0E8CAB80917D0E8DAB80917E0E1D
:10A100008EAB80917F0E8FAB8091800E88AFCE0199
:10A110008D960E94294692C1F6013496AEE8BFE0C2
:10A120008CE490E021E08030920719F40E94C06630
:10A1300003C0182E0E94C066F60184818093830EAE
:10A140008581982F97708091840E887F892B8093CA
:10A15000840E87898093850E808D982F97708091CB
:10A16000860E887F892B8093860E82A58093870E2A
:10A1700083A5982F97708091880E887F892B809374
:10A18000880E85AD8093890E86AD982F977080914B
:10A190008A0E887F892B80938A0E81E08FA787EEB5
:10A1A00088AB84E08EA7CE018D960E94294646C1D9
:10A1B00081E08FA788EE88AB80E58EA7FE01F1963F
:10A1C000AEE8BFE08CE490E021E08030920719F423
:10A1D0000E94AF6603C0182E0E94AF66CE018D9616
:10A1E0000E9429462BC1F6013496AAEDBFE089E012
:10A1F00090E021E08030920719F40E94C06603C00D
:10A20000182E0E94C066F6013D96A3EEBFE089E0DD
:10A2100090E021E08030920719F40E94C06603C0EC
:10A22000182E0E94C06681E08FA789EE88AB84E07B
:10A230008EA7CE018D960E94294600C181E08FA78E
:10A240008AEE88AB87E18EA7FE01F196AAEDBFE00A
:10A2500089E090E021E08030920719F40E94AF6617
:10A2600003C0182E0E94AF66FE01FA96A3EEBFE06F
:10A2700089E090E021E08030920719F40E94AF66F7
:10A2800003C0182E0E94AF66CE018D960E9429460B
:10A29000D5C0C60105960E949C3581E08FA786ED4A
:10A2A00088AB85E08EA7CE018D960E942946C6C058
:10A2B00081E08FA787ED88AB8DE18EA7CE01C29696
:10A2C0000E94AC35CE018D960E942946B7C0F6019A
:10A2D000B480C60104960E94BC3581E08FA78AED48
:10A2E00088AB85E08EA7B9AACE018D960E9429463B
:10A2F000A5C0F601B48081E08FA78BED88AB8AE41E
:10A300008EA7BE016F5C7F4F8B2D0E94E935CE0179
:10A310008D960E94294692C0F601B4808B2D0E9432
:10A32000481181E08FA78CED88ABB9AA85E08EA794
:10A33000CE018D960E94294681C0F6014481558147
:10A3400081E08FA78DED88AB86E18EA75AAB49AB34
:10A35000FE01ED51FF4F1082FE01ED51FF4F808154
:10A36000982F8031C8F48E010F5F1F4FBF01892FD6
:10A3700099279C01200F311F840F951FAA27BB2707
:10A38000ABBFFC018791F90182ABDB018C918F5F40
:10A390008C93982F803158F3CE018D960E942946D8
:10A3A0004DC0F6013496AEE5BFE080E190E021E0DB
:10A3B0008030920719F40E94C06603C0182E0E94D4
:10A3C000C06681E08FA781EE88AB84E08EA7CE01C6
:10A3D0008D960E94294632C081E08FA782EE88AB1D
:10A3E00084E18EA7FE01F196AEE5BFE080E190E04A
:10A3F00021E08030920719F40E94AF6603C0182E46
:10A400000E94AF66CE018D960E94294617C081E05A
:10A410008FA780E888AB85E08EA7F601838189ABA2
:10A42000CE018D960E94294609C085E08EA71FA601
:10A4300081E088ABCE018D960E942946CD51DF4F39
:10A440000FB6F894DEBF0FBECDBFDF91CF911F9145
:10A450000F91FF90EF90DF90CF90BF90AF90089555
:10A46000CF93DF93CDB7DEB72A970FB6F894DEBF50
:10A470000FBECDBF81E08B8388E88C8384E08A8324
:10A48000CE0101960E9429462A960FB6F894DEBFA7
:10A490000FBECDBFDF91CF9108950F931F93CF9340
:10A4A000DF93CDB7DEB7C055D0400FB6F894DEBF0E
:10A4B0000FBECDBF8A0121E02B832DE52C839E8327
:10A4C0008D836F8320E0261780F4AE01485F5F4FD5
:10A4D000822F9927DA01A80FB91FF801E80FF91F99
:10A4E00080818C932F5F261798F38FE08A83CE01AB
:10A4F00001960E942946C05BDF4F0FB6F894DEBF7D
:10A500000FBECDBFDF91CF911F910F91089548EC01
:10A5100050E060E070E08DE19BE00E94D065109219
:10A52000E50B1092E60B10921C0B0895382F20912A
:10A53000E60B8DE19BE0FC01E20FF11D3083809181
:10A54000E60B8F5F8093E60B80911C0B8F5F8093EF
:10A550001C0B80911C0B883C18F00E9487520895B8
:10A560008091E60B883C10F01092E60B08959091D4
:10A57000E60B8091E50B981738F08091E60B9091EF
:10A58000E50B891B992708959091E60B8091E50BC7
:10A59000981B892F8853992708952091E50B8DE109
:10A5A0009BE0FC01E20FF11DE0818091E50B8F5FE4
:10A5B0008093E50B80911C0B815080931C0B809144
:10A5C000E50B883C10F01092E50B8E2F992708952B
:10A5D0000F931F93CF93DF93EC018B0180EC0E94CC
:10A5E0007B54015010408FEF0F3F180709F188810D
:10A5F0009927803C910521F08B3D910541F00EC0DB
:10A600008BED0E947B548CED0E947B540AC08BED35
:10A610000E947B548DED0E947B5403C088810E9470
:10A620007B542196015010408FEF0F3F1807F9F629
:10A6300080EC0E947B54DF91CF911F910F91089580
:10A640000F931F93382F8091E70B9927009719F0EC
:10A650000197C1F059C0303C09F056C01092E80B88
:10A660002091E80B8AEE9BE0FC01E20FF11D3083A4
:10A670002F5F2093E80B81E08093E70B84E68093C3
:10A68000E90B42C0303C99F58091E80B8230F0F044
:10A690008091E80B0AEE1BE0F801E80FF11D308312
:10A6A0008F5F8093E80B82E08093E70B1092E90BB9
:10A6B000A8016091E80BC8010E948F53C8010E9455
:10A6C0003F461092E70B1092E80B1EC01092E80B69
:10A6D0002091E80B8AEE9BE0FC01E20FF11D308334
:10A6E0002F5F2093E80B84E68093E90B0DC0209147
:10A6F000E80B8AEE9BE0FC01E20FF11D30838091B4
:10A70000E80B8F5F8093E80B8091E80B893620F08F
:10A710001092E70B1092E80B1F910F910895FC0126
:10A72000DA0161506F3FF1F02081822F9927803C40
:10A73000910521F08B3D910519F010C0319610C0A4
:10A7400031962081822F99278C3D910521F08D3DF6
:10A75000910519F003C020EC01C02BED2D9331962B
:10A76000615010F708958091E90B882389F080915A
:10A77000E90B81508093E90B9091E90B992341F407
:10A780008091E70B813021F49093E80B9093E70BD5
:10A79000089585B1807F85B984B1876084B981E5EA
:10A7A0008CBD81E08DBD08958EBD0DB407FEFDCF3B
:10A7B0008EB5992708950E9438549C9AA4988FE0EA
:10A7C0008093540CA4986A9862980895A498089568
:10A7D000CF93DF93CDB7DEB728970FB6F894DEBFDF
:10A7E0000FBECDBFA49B18C0629914C08091530CBA
:10A7F000853050F0A4980E947B2182E28093110161
:10A8000010928B0E1092740E8091530C8F5F809378
:10A81000530C02C01092530CCE0101960E945B2C87
:10A8200029813A8181E590E0289FA001299F500D60
:10A83000389F500D1124CA01880F892F881F990B4A
:10A8400091950E9439548D81882319F48F81882332
:10A8500011F0A49A01C0A49828960FB6F894DEBF10
:10A860000FBECDBFDF91CF9108958093540C089512
:10A87000089508951092560C1092550C86E080931E
:10A88000C20088E98093C10060E875E280E090E052
:10A890000E94555481E08093F40E1092F50E0895B5
:10A8A0009093560C8093550C08959B01AC01DC01EC
:10A8B000CB01689412F8880F991FAA1FBB1F16942A
:10A8C000D1F780509C4DAB40BF4F689413F8220FD6
:10A8D000331F441F551F1694D1F7BC01CD010E94B0
:10A8E0003366DA01C9010197292F33272093C50068
:10A8F0008093C4000895982F8091C00085FFFCCFFD
:10A900009093C60008950F931F93CF93DF938C010C
:10A91000EB0121978FEFCF3FD80751F0F8018191DC
:10A920008F010E947B542197FFEFCF3FDF07B1F7E4
:10A9300081E090E0DF91CF911F910F9108951F92D8
:10A940000F920FB60F9211242F933F934F935F9363
:10A950006F937F938F939F93AF93BF93EF93FF93E7
:10A960008091C6000E949652FF91EF91BF91AF91E6
:10A970009F918F917F916F915F914F913F912F9117
:10A980000F900FBE0F901F901895DC01FB014150F6
:10A9900050408FEF4F3F580741F081918D934150C8
:10A9A00050408FEF4F3F5807C1F70895DC01FB017E
:10A9B000415050408FEF4F3F580769F091918D9172
:10A9C000891719F081E090E00895415050408FEFD1
:10A9D0004F3F580799F780E090E00895CF93DF93B9
:10A9E000DC01FB0160E0462F91E0562F8081803230
:10A9F00031F4692F9F5F319680818032D1F380815D
:10AA0000882379F08081803219F4442309F4492F96
:10AA10008081803209F040E09F5F319680818823F9
:10AA200089F7442331F48081882311F4492F01C030
:10AA3000462F262F3327E901C91BD109EC0FFD1F33
:10AA40003196842F9927821B930B019718161906AC
:10AA500024F4942F961B915001C090E091509F3F99
:10AA600029F081918D935F5F9150D8F71C925F5FC1
:10AA7000852F9927DF91CF910895FC0190E0819176
:10AA8000882331F09F5F8191882311F09F3FD1F798
:10AA9000892F99270895DC01FB018081882329F003
:10AAA00081918D9380818823D9F71C9208950F930B
:10AAB0001F93CF93DF93082F162FFA0141E0C0E1D7
:10AAC000D7E2C901BE010E9420666115710581F0BF
:10AAD0006C9FC0016D9F900D7C9F900D1124281BD1
:10AAE000390B862F805D8193440F01E015E00AC089
:10AAF000153040F0002319F080E3819302C080E21A
:10AB000081934F5FC8EED3E0C901BE010E94206669
:10AB10006115710581F06C9FC0016D9F900D7C9F48
:10AB2000900D1124281B390B862F805D81934F5F78
:10AB300001E014E00AC0143040F0002319F080E373
:10AB4000819302C080E281934F5FC4E6D0E0C901E7
:10AB5000BE010E9420666115710581F04F5F6C9FF8
:10AB6000C0016D9F900D7C9F900D1124281B390B07
:10AB7000862F805D819301E013E00AC0133040F01E
:10AB80004F5F002319F080E3819302C080E281933C
:10AB9000C9016AE070E00E9420666115710591F0BC
:10ABA0004F5FCB01880F991F880F991F880F991F3E
:10ABB000860F971F860F971F281B390B862F805DE6
:10ABC00081930AC0123040F04F5F002319F080E3F8
:10ABD000819302C080E28193822F805D81931082F5
:10ABE000842F9927DF91CF911F910F910895FC0138
:10ABF000262F862F82958F708A3038F06AE00E9467
:10AC00000066892F8F5B819309C0862F82958F7094
:10AC10006AE00E940066892F805D8193822F8F7089
:10AC20008A3038F06AE00E940066892F8F5B80834B
:10AC30000895822F8F706AE00E940066892F805DE0
:10AC400080830895EF92FF920F931F937C018B01F5
:10AC5000872F9927682FC7010E94F755C801907068
:10AC6000682FC7010E94F7551F910F91FF90EF9039
:10AC70000895CF92DF92EF92FF920F931F936C0192
:10AC80007A018B01CB01AA27BB27BC01C6010E9418
:10AC90002256D801C701A070B070BC01C6010E9445
:10ACA00022561F910F91FF90EF90DF90CF90089563
:10ACB0001F93CF93DF93CDB7DEB768970FB6F894A5
:10ACC000DEBF0FBECDBF10E0BE016F5F7F4F812F93
:10ACD0000E944234412F5527CA01880F991F880FBF
:10ACE000991F880F991F9C01241B350BF901E95A04
:10ACF000F34F898184838A8185838B8186838C81CC
:10AD000080838D8181838E818283F901E65AF34F9E
:10AD10008F81382F337088858370282F220F220F60
:10AD2000888D982F9295907F822F832B892B8083FB
:10AD3000FA01E35AF24F10821F5F143128F268962D
:10AD40000FB6F894DEBF0FBECDBFDF91CF911F913C
:10AD500008951F93CF93DF93CDB7DEB768970FB6F3
:10AD6000F894DEBF0FBECDBF10E0A89519821A82FD
:10AD70001B821C821D821E821F821886188E8FE005
:10AD8000189FC00111248858994FBC01CE01099623
:10AD90000E94AF65BE016F5F7F4F812F0E940A3412
:10ADA0001F5F143110F368960FB6F894DEBF0FBE24
:10ADB000CDBFDF91CF911F910895CF93C0E086E082
:10ADC000C89FC0011124FC01EB51F34FF093E40C38
:10ADD000E093E30C80819181009719F001979183B2
:10ADE0008083E091E30CF091E40C828193810097E1
:10ADF00019F0019793838283E091E30CF091E40CC6
:10AE000084819581009719F00197958384832C2F75
:10AE10003327C901880F991F880F991F880F991F21
:10AE2000821B930BFC01E95AF34F8081882319F4AC
:10AE30008181882321F08C2F8F5D0E942E58CF5F57
:10AE4000C43108F4BCCFCF9108959927873091057C
:10AE500009F466C088309105ACF48430910509F49A
:10AE60003EC08530910534F48230910511F103978D
:10AE700059F198C08530910509F43CC0069709F452
:10AE800044C090C08A30910509F46BC08B309105A5
:10AE900044F48830910509F44EC0099709F456C06E
:10AEA00081C08B30910509F467C00C9709F46FC01D
:10AEB00079C080EC0E94BC44882319F081E090E0C6
:10AEC000089580E090E0089581EC0E94BC448823BE
:10AED00019F081E090E0089580E090E0089582EC20
:10AEE0000E94BC44882319F081E090E0089580E03E
:10AEF00090E0089581ED0E94BC44882319F081E020
:10AF000090E0089580E090E0089584EC0E94BC44B5
:10AF1000882319F081E090E0089580E090E00895A2
:10AF200085EC0E94BC44882319F081E090E00895EC
:10AF300080E090E0089586EC0E94BC44882319F0DC
:10AF400081E090E0089580E090E0089587EC0E9411
:10AF5000BC44882319F081E090E0089580E090E0FF
:10AF6000089583EC0E94BC44882319F081E090E0AE
:10AF7000089580E090E0089582ED0E94BC4488230B
:10AF800019F081E090E0089580E090E0089583ED6D
:10AF90000E94BC44882319F081E090E0089580E08D
:10AFA00090E0089580E090E008950F93CF93DF93B1
:10AFB000CDB7DEB721970FB6F894DEBF0FBECDBF79
:10AFC00089838150843170F000E021E0AE014F5F51
:10AFD0005F4F69E071E08EE891E00E949D2F80E074
:10AFE00090E007C089819927FC01E45AF24F8081E3
:10AFF000992721960FB6F894DEBF0FBECDBFDF9123
:10B00000CF910F9108950F93CF93DF93CDB7DEB714
:10B0100021970FB6F894DEBF0FBECDBF8983843170
:10B0200060F000E021E0AE014F5F5F4F64E171E04E
:10B030008EE891E00E949D2F07C089812DE53DE0BB
:10B04000F901E80FF11D608321960FB6F894DEBF79
:10B050000FBECDBFDF91CF910F910895FF920F9357
:10B060001F93CF93DF93CDB7DEB721970FB6F89438
:10B07000DEBF0FBECDBF1982813209F46DC08232AE
:10B0800019F481E0898368C0833219F482E08983EE
:10B0900063C0843219F483E089835EC0853219F479
:10B0A00084E0898359C0863219F485E0898354C0CD
:10B0B000873219F486E089834FC0883219F487E01B
:10B0C00089834AC0893219F488E0898345C08A326D
:10B0D00019F489E0898340C08B3219F48AE08983AE
:10B0E0003BC08C3219F48BE0898336C08D3219F461
:10B0F0008CE0898331C08E3219F48DE089832CC0B5
:10B100008F3219F48EE0898327C0803319F48FE0E1
:10B11000898322C0813319F480E189831DC0823381
:10B1200019F481E1898318C0833319F482E189839A
:10B1300013C0843319F483E189830EC000E021E059
:10B14000AE014F5F5F4F69E471E08EE891E00E94CD
:10B150009D2F80E090E087C700E0102FF02E29811E
:10B1600086E0289FC00111248B51934F9093E40CEB
:10B170008093E30C3327C901880F991F880F991F0B
:10B18000880F991F821B930BFC01E95AF34F8081B2
:10B19000882309F49BC18981282F3327C901880F8F
:10B1A000991F880F991F880F991F821B930BFC0111
:10B1B000E95AF34F80818F3F11F411E087C18981F3
:10B1C000282F3327C901880F991F880F991F880FCF
:10B1D000991F821B930BFC01E95AF34FE0818E2FDC
:10B1E00082508B3008F04DC08E2F0E942557482F7B
:10B1F0008981282F3327C901880F991F880F991F2C
:10B20000880F991F821B930BFC01E65AF34F808134
:10B2100082958F7080FF02C081E04827442361F04F
:10B22000E091E30CF091E40C80819181892B11F481
:10B2300011E04CC110E04AC1A091E30CB091E40CC4
:10B240008981282F3327C901880F991F880F991FDB
:10B25000880F991F821B930BFC01E95AF34F9481CD
:10B2600085E0989FC00111248D939C93E091E30C9D
:10B27000F091E40C8081918101969183808310E0AC
:10B2800025C18981282F3327C901880F991F880F6D
:10B29000991F880F991F821B930BFC01E95AF34FEA
:10B2A000E0818E2F8D50803208F04DC08F5F0E945C
:10B2B0004B11482F8981282F3327C901880F991FE7
:10B2C000880F991F880F991F821B930BFC01E65A68
:10B2D000F34F808182958F7080FF02C081E0482704
:10B2E000442361F0E091E30CF091E40C80819181C2
:10B2F000892B11F411E0EAC010E0E8C0A091E30C42
:10B30000B091E40C8981282F3327C901880F991F38
:10B31000880F991F880F991F821B930BFC01E95A14
:10B32000F34F948185E0989FC00111248D939C93E5
:10B33000E091E30CF091E40C80819181019691837E
:10B34000808310E0C3C08981282F3327C901880F6B
:10B35000991F880F991F880F991F821B930BFC015F
:10B36000E95AF34FE0818E2F8D52823208F04DC0A2
:10B370008F5F0E94152C482F8981282F3327C90100
:10B38000880F991F880F991F880F991F821B930B95
:10B39000FC01E65AF34F808182958F7080FF02C0D6
:10B3A00081E04827442361F0E091E30CF091E40C44
:10B3B00080819181892B11F411E088C010E086C052
:10B3C000A091E30CB091E40C8981282F3327C901A7
:10B3D000880F991F880F991F880F991F821B930B45
:10B3E000FC01E95AF34F948185E0989FC001112434
:10B3F0008D939C93E091E30CF091E40C808191811A
:10B4000001969183808310E061C08981282F3327C2
:10B41000C901880F991F880F991F880F991F821BD8
:10B42000930BFC01E95AF34FE0818E2F8F548F303C
:10B4300008F04CC08F5F0E94D557482F8981282F74
:10B440003327C901880F991F880F991F880F991FEB
:10B45000821B930BFC01E65AF34F808182958F701B
:10B4600080FF02C081E04827442361F0E091E30CB3
:10B47000F091E40C80819181892B11F411E026C0B8
:10B4800010E024C0A091E30CB091E40C8981282F36
:10B490003327C901880F991F880F991F880F991F9B
:10B4A000821B930BFC01E95AF34F948185E0989F2E
:10B4B000C00111248D939C93E091E30CF091E40C76
:10B4C0008081918101969183808310E08981282F6A
:10B4D0003327C901880F991F880F991F880F991F5B
:10B4E000821B930BFC01E95AF34F8181882311F4ED
:10B4F000082F9FC18981282F3327C901880F991FE1
:10B50000880F991F880F991F821B930BFC01E95A22
:10B51000F34F81818F3F11F401E08BC18981282F86
:10B520003327C901880F991F880F991F880F991F0A
:10B53000821B930BFC01E95AF34F9181892F8250B2
:10B540008B3008F04EC0892F0E942557482F8981E3
:10B55000282F3327C901880F991F880F991F880F3B
:10B56000991F821B930BFC01E65AF34F8081829551
:10B570008F7081FF02C081E04827442361F0E09191
:10B58000E30CF091E40C82819381892B11F401E0AA
:10B5900050C100E04EC1A091E30CB091E40C898150
:10B5A000282F3327C901880F991F880F991F880FEB
:10B5B000991F821B930BFC01E95AF34F958185E09B
:10B5C000989FC0011124FD0193838283E091E30CD5
:10B5D000F091E40C8281938101969383828300E051
:10B5E00028C18981282F3327C901880F991F880F07
:10B5F000991F880F991F821B930BFC01E95AF34F87
:10B600009181892F8D50803208F04EC08F5F0E944B
:10B610004B11482F8981282F3327C901880F991F83
:10B62000880F991F880F991F821B930BFC01E65A04
:10B63000F34F808182958F7081FF02C081E048279F
:10B64000442361F0E091E30CF091E40C828193815A
:10B65000892B11F401E0EDC000E0EBC0A091E30CF8
:10B66000B091E40C8981282F3327C901880F991FD5
:10B67000880F991F880F991F821B930BFC01E95AB1
:10B68000F34F958185E0989FC0011124FD019383BC
:10B690008283E091E30CF091E40C82819381019626
:10B6A0009383828300E0C5C08981282F3327C90195
:10B6B000880F991F880F991F880F991F821B930B62
:10B6C000FC01E95AF34F9181892F8D52823208F0A3
:10B6D0004EC08F5F0E94152C482F8981282F332759
:10B6E000C901880F991F880F991F880F991F821B06
:10B6F000930BFC01E65AF34F808182958F7081FF96
:10B7000002C081E04827442361F0E091E30CF0910E
:10B71000E40C82819381892B11F401E08AC000E05E
:10B7200088C0A091E30CB091E40C8981282F3327C5
:10B73000C901880F991F880F991F880F991F821BB5
:10B74000930BFC01E95AF34F958185E0989FC00166
:10B750001124FD0193838283E091E30CF091E40CCA
:10B760008281938101969383828300E062C0898104
:10B77000282F3327C901880F991F880F991F880F19
:10B78000991F821B930BFC01E95AF34F9181892F7A
:10B790008F548F3008F04DC08F5F0E94D557482FCF
:10B7A0008981282F3327C901880F991F880F991F76
:10B7B000880F991F821B930BFC01E65AF34F80817F
:10B7C00082958F7081FF02C081E04827442361F099
:10B7D000E091E30CF091E40C82819381892B11F4C8
:10B7E00001E027C000E025C0A091E30CB091E40C7B
:10B7F0008981282F3327C901880F991F880F991F26
:10B80000880F991F821B930BFC01E95AF34F958116
:10B8100085E0989FC0011124FD0193838283E0910C
:10B82000E30CF091E40C82819381019693838283EF
:10B8300000E08981282F3327C901880F991F880FBD
:10B84000991F880F991F821B930BFC01E95AF34F34
:10B850008281882311F4F82EA4C18981282F3327EF
:10B86000C901880F991F880F991F880F991F821B84
:10B87000930BFC01E95AF34F82818F3F19F4FF24A7
:10B88000F3948FC18981282F3327C901880F991F0D
:10B89000880F991F880F991F821B930BFC01E95A8F
:10B8A000F34F9281892F82508B3008F04FC0892F3F
:10B8B0000E942557482F8981282F3327C901880FD7
:10B8C000991F880F991F880F991F821B930BFC01EA
:10B8D000E65AF34F808182958F7082FF02C081E02B
:10B8E0004827442369F0E091E30CF091E40C848153
:10B8F0009581892B19F4FF24F39453C1FF2451C17E
:10B90000A091E30CB091E40C8981282F3327C90161
:10B91000880F991F880F991F880F991F821B930BFF
:10B92000FC01E95AF34F968185E0989FC0011124EC
:10B93000FD0195838483E091E30CF091E40C848114
:10B940009581019695838483FF242BC18981282FBB
:10B950003327C901880F991F880F991F880F991FD6
:10B96000821B930BFC01E95AF34F9281892F8D5072
:10B97000803208F04FC08F5F0E944B11482F8981A1
:10B98000282F3327C901880F991F880F991F880F07
:10B99000991F821B930BFC01E65AF34F808182951D
:10B9A0008F7082FF02C081E04827442369F0E09154
:10B9B000E30CF091E40C84819581892B19F4FF2428
:10B9C000F394EFC0FF24EDC0A091E30CB091E40C20
:10B9D0008981282F3327C901880F991F880F991F44
:10B9E000880F991F821B930BFC01E95AF34F968134
:10B9F00085E0989FC0011124FD0195838483E09127
:10BA0000E30CF091E40C8481958101969583848305
:10BA1000FF24C7C08981282F3327C901880F991FA8
:10BA2000880F991F880F991F821B930BFC01E95AFD
:10BA3000F34F9281892F8D52823208F04FC08F5F71
:10BA40000E94152C482F8981282F3327C901880F80
:10BA5000991F880F991F880F991F821B930BFC0158
:10BA6000E65AF34F808182958F7082FF02C081E099
:10BA70004827442369F0E091E30CF091E40C8481C1
:10BA80009581892B19F4FF24F3948BC0FF2489C07E
:10BA9000A091E30CB091E40C8981282F3327C901D0
:10BAA000880F991F880F991F880F991F821B930B6E
:10BAB000FC01E95AF34F968185E0989FC00111245B
:10BAC000FD0195838483E091E30CF091E40C848183
:10BAD0009581019695838483FF2463C08981282FF3
:10BAE0003327C901880F991F880F991F880F991F45
:10BAF000821B930BFC01E95AF34F9281892F8F54DB
:10BB00008F3008F04EC08F5F0E94D557482F898133
:10BB1000282F3327C901880F991F880F991F880F75
:10BB2000991F821B930BFC01E65AF34F808182958B
:10BB30008F7082FF02C081E04827442369F0E091C2
:10BB4000E30CF091E40C84819581892B19F4FF2496
:10BB5000F39427C0FF2425C0A091E30CB091E40C1E
:10BB60008981282F3327C901880F991F880F991FB2
:10BB7000880F991F821B930BFC01E95AF34F9681A2
:10BB800085E0989FC0011124FD0195838483E09195
:10BB9000E30CF091E40C8481958101969583848374
:10BBA000FF242981822F9927AC01440F551F440F90
:10BBB000551F440F551F481B590BDA01A95AB34FA3
:10BBC0008C91882309F47FC1FD018181882309F4C8
:10BBD0007AC18281882309F476C1FA01E65AF34FCB
:10BBE000E0818E2F837009F084C0112309F43EC0D8
:10BBF0000023E1F18E2F86958695837061F46F2D79
:10BC0000822F0E940358FF2019F081E090E02BC2A0
:10BC100080E090E028C28981282F3327C901880F4E
:10BC2000991F880F991F880F991F821B930BFC0186
:10BC3000E65AF34F8081869586958370823079F439
:10BC400060E01F1509F461E089810E9403581F1507
:10BC500019F481E090E007C280E090E004C261E066
:10BC600089810E94035881E090E0FDC14981242F21
:10BC70003327C901880F991F880F991F880F991FB3
:10BC8000821B930BFC01E65AF34F808186958695C3
:10BC90008370823049F4FF2039F461E0842F0E94E0
:10BCA000035881E090E0DFC14981242F3327C90187
:10BCB000880F991F880F991F880F991F821B930B5C
:10BCC000FC01E65AF34F808186958695682F637054
:10BCD000613041F4FF2031F0842F0E94035881E04D
:10BCE00090E0C1C160E089810E94035880E090E04B
:10BCF000BAC14981242F3327C901880F991F880FA2
:10BD0000991F880F991F821B930BFC01E65AF34F72
:10BD1000E0818E2F8370823009F045C01017E1F565
:10BD20008E2F86958695837061F46F2D842F0E94E7
:10BD30000358FF2019F081E090E095C180E090E089
:10BD400092C18981282F3327C901880F991F880F35
:10BD5000991F880F991F821B930BFC01E65AF34F22
:10BD60008081869586958370823079F460E01F1516
:10BD700009F461E089810E9403581F1519F481E0DC
:10BD800090E071C180E090E06EC161E089810E9425
:10BD9000035881E090E067C160E089810E94035808
:10BDA00080E090E060C1112319F4002309F448C039
:10BDB0004981242F3327C901880F991F880F991FA4
:10BDC000880F991F821B930BFC01E65AF34F808169
:10BDD00086958695837061F46F2D842F0E94035899
:10BDE000FF2019F081E090E03EC180E090E03BC18F
:10BDF0004981242F3327C901880F991F880F991F64
:10BE0000880F991F821B930BFC01E65AF34F808128
:10BE1000869586958370823061F46F2D842F0E9401
:10BE20000358FF2019F081E090E01DC180E090E010
:10BE30001AC161E089810E94035881E090E013C13A
:10BE40004981242F3327C901880F991F880F991F13
:10BE5000880F991F821B930BFC01E65AF34F8081D8
:10BE600086958695682F6370613041F4FF2021F13B
:10BE7000842F0E94035881E090E0F5C04981242F6F
:10BE80003327C901880F991F880F991F880F991FA1
:10BE9000821B930BFC01E65AF34F808186958695B1
:10BEA0008370823049F4FF2039F461E0842F0E94CE
:10BEB000035881E090E0D7C060E089810E94035878
:10BEC00080E090E0D0C02981822F9927AC01440FF7
:10BED000551F440F551F440F551F481B590BDA01BE
:10BEE000A95AB34F8C91882309F452C0FD01818176
:10BEF000882309F44DC0FA01E65AF34F808183701C
:10BF000091F4112349F0002339F061E0822F0E945F
:10BF1000035881E090E0A7C060E089810E94035847
:10BF200080E090E0A0C04981242F3327C901880F09
:10BF3000991F880F991F880F991F821B930BFC0173
:10BF4000E65AF34F80818370823081F4101739F400
:10BF500061E0842F0E94035881E090E084C060E09B
:10BF600089810E94035880E090E07DC0112311F484
:10BF7000002339F061E089810E94035881E090E05C
:10BF800072C060E089810E94035880E090E06BC03D
:10BF90002981822F9927AC01440F551F440F551F4B
:10BFA000440F551F481B590BDA01A95AB34FFD0125
:10BFB0008181882309F455C08281882309F451C006
:10BFC000FA01E65AF34F808186958695837091F445
:10BFD000112349F0002339F061E0822F0E940358B9
:10BFE00081E090E040C060E089810E94035880E0D9
:10BFF00090E039C04981242F3327C901880F991F48
:10C00000880F991F880F991F821B930BFC01E65A1A
:10C01000F34F8081869586958370823081F4101766
:10C0200039F461E0842F0E94035881E090E01BC046
:10C0300060E089810E94035880E090E014C01123E1
:10C0400011F4002339F061E089810E94035881E0F6
:10C0500090E009C060E089810E94035880E090E090
:10C0600002C080E090E021960FB6F894DEBF0FBECC
:10C07000CDBFDF91CF911F910F91FF900895CF9386
:10C08000DF93CDB7DEB721970FB6F894DEBF0FBEB2
:10C09000CDBF282F04B603FE28C0FE013196ACEBBD
:10C0A000B0E081E090E031E08030930719F40E9425
:10C0B000AF6603C0182E0E94AF668981843190F468
:10C0C0008F5F8983FE013196ACEBB0E081E090E0B8
:10C0D00031E08030930719F40E94C06603C0182E27
:10C0E0000E94C06684B7877F84BF809160008861AA
:10C0F000809360002093600080916000886080934E
:10C10000600021960FB6F894DEBF0FBECDBFDF9161
:10C11000CF910895EF92FF920F931F937B018C01B3
:10C1200020E030E040E05FE40E94EE6288239CF073
:10C1300020E030E040E05FECC801B7010E94D86128
:10C14000DC01CB01BC01CD010E94886360507040CE
:10C150008040904804C0C801B7010E9488631F91C5
:10C160000F91FF90EF900895A0E0B0E0EAEBF0E6C9
:10C170000C9470668C017B015A01DC018C91823039
:10C1800058F0FB019081923010F4A7010BC184306C
:10C1900029F4943009F4A6C0A80104C19430A9F38D
:10C1A000923009F4A9C0823081F3F801C280D380B3
:10C1B000FB0162817381F8012481358146815781B9
:10C1C000F7016480758086809780C601861B970B77
:10C1D00097FDD8C080970CF46CC06C157D050CF0F1
:10C1E000ADC0662477244301F8016181F7018181A4
:10C1F000681709F499C0662309F491C0621A730A9A
:10C20000840A950AA401930157FDC0C0F50111826B
:10C21000B60119012A0179018A0139014A010894FC
:10C220006108710881089108FFEF6F16FFEF7F0624
:10C23000FFEF8F06FFE39F06F0F4A8019701220F9E
:10C24000331F441F551F19012A01B6016150704068
:10C250006B0179018A0139014A010894610871086A
:10C26000810891088FEF68168FEF78068FEF8806A8
:10C270008FE3980610F383E0D5018C9357FC64C0DC
:10C28000F501248335834683578373836283A50135
:10C2900089C06F5F7F4FD401C30181709070A0701F
:10C2A000B0709694879477946794682A792A8A2A3A
:10C2B0009B2A6C157D056CF311C00894C11CD11C20
:10C2C000DA01C90181709070A070B07056954795E1
:10C2D00037952795282B392B4A2B5B2BC616D7066B
:10C2E00064F382CFF8019181FB018181981709F4F1
:10C2F00053CF41EA51E056C0823009F04DCF88E07B
:10C30000DA01F80101900D928A95E1F7F801818137
:10C31000FB0191818923FA018183A50143C026197C
:10C3200037094809590970CFF5016183B601260D17
:10C33000371D481D591D19012A019DCF6B0120E0B1
:10C3400030E040E050E050CFD201C101B695A79552
:10C350009795879521E030E040E050E0222233229B
:10C3600044225522282A392A4A2A5B2AF5012482A6
:10C370003582468257820894C11CD11CD382C28266
:10C38000A50110C0909581959F4F24CF81E0F501C4
:10C390008183B60150954095309521953F4F4F4F81
:10C3A0005F4F37CFCA01E2E1CDB7DEB70C948C66A0
:10C3B000A0E2B0E0EEEDF1E60C947E66DC01CB018C
:10C3C000898F9A8FAB8FBC8F2D8F3E8F4F8F58A345
:10C3D000BE016F5F7F4FCE0149960E94C2648E01FD
:10C3E000075F1F4FB801CE014D960E94C264AE0197
:10C3F0004F5E5F4FB801CE0101960E94B4600E946B
:10C40000DA63DC01CB01BC01CD01E4E0A0960C9421
:10C410009A66A0E2B0E0EFE0F2E60C947E66DC0102
:10C42000CB01898F9A8FAB8FBC8F2D8F3E8F4F8F13
:10C4300058A3BE016F5F7F4FCE0149960E94C26430
:10C440008E01075F1F4FB801CE014D960E94C26456
:10C450008A8591E089278A87AE014F5E5F4FB801D8
:10C46000CE0101960E94B4600E94DA63DC01CB0128
:10C47000BC01CD01E4E0A0960C949A66A8E1B0E07E
:10C48000E4E4F2E60C947866DC01CB01898B9A8BAC
:10C49000AB8BBC8B2D8B3E8B4F8B588FBE016F5F50
:10C4A0007F4FCE0141960E94C2648E01075F1F4FED
:10C4B000B801CE0145960E94C264FE0131962981E1
:10C4C000223008F45FC03985323010F4B8017BC0E7
:10C4D00081819A8589278183243009F455C02230CF
:10C4E00009F452C0343009F454C0323009F458C051
:10C4F0006B817C818B859C85681B790B2D813E81AE
:10C500004F815885ED84FE840F8518892E153F05CF
:10C510004007510730F4220F331F441F551F61504D
:10C5200070407C836B8380E090E0A0E0B0E4AA24BC
:10C53000BB2465012E153F054007510740F0A82A8E
:10C54000B92ACA2ADB2A2E193F09400B510BB6958E
:10C55000A79597958795220F331F441F551F009766
:10C56000A105B10539F7D601C5018F779070A0708C
:10C57000B07080349105A105B105A9F0A482B582FF
:10C58000C682D782BF011FC02317E1F761EA71E0BD
:10C590001AC01D821E821F8218861C821B82F2CF47
:10C5A00084E08983EFCFA7FC05C021153105410543
:10C5B000510521F380E490E0A0E0B0E0A80EB91EA0
:10C5C000CA1EDB1EDBCFCB010E94DA63DC01CB018C
:10C5D000BC01CD01EAE068960C949466A8E1B0E055
:10C5E000E4EFF2E60C947E66DC01CB01898B9A8B3A
:10C5F000AB8BBC8B2D8B3E8B4F8B588FBE016F5FEF
:10C600007F4FCE0141960E94C2648E01075F1F4F8B
:10C61000B801CE0145960E94C2648981823018F02B
:10C620008985823018F42FEF3FEF09C0B801CE01A1
:10C6300001960E943C65282F332727FD3095C901BC
:10C64000E4E068960C949A66A8E0B0E0EAE2F3E6CB
:10C650000C947C669B01AC017B018C01EE2417FDE0
:10C66000E394FF2400271127EA82211531054105B3
:10C67000510539F482E08983CE0101960E94DA6384
:10C6800043C083E089836EE170E0CB01EE2031F599
:10C6900079018A01A80197012030E0E03E07E0E03F
:10C6A0004E07E0E45E0798F479018A01EE0CFF1C66
:10C6B000001F111F0197BC01A8019701E0E0EE16D1
:10C6C000E0E0FE06E0E00E07E0E41E0768F3ED821E
:10C6D000FE820F8318877C836B83CECF2030E0E00F
:10C6E0003E07E0E04E07E0E85E0741F0EE24FF245D
:10C6F0008701E21AF30A040B150BCCCF7C836B8302
:10C7000060E070E080E09FECE6E028960C9498668C
:10C71000ACE0B0E0EEE8F3E60C948066DC01CB011F
:10C7200089879A87AB87BC87BE016F5F7F4FCE0139
:10C7300009960E94C2648981823011F0823028F407
:10C7400060E070E080E090E031C0843039F02B810F
:10C750003C8137FDF5CF2F3131056CF08A8188237C
:10C7600029F060E070E080E090E820C06FEF7FEF9C
:10C770008FEF9FE71BC08EE190E0821B930B2D8112
:10C780003E814F81588504C056954795379527952A
:10C790008A95D2F78A81882339F050954095309553
:10C7A00021953F4F4F4F5F4FCA01B901E2E02C96F0
:10C7B0000C949C66A0E0B0E0E0EEF3E60C947666A4
:10C7C000882499245401DC01FC01248135814681AF
:10C7D00057818181082F112760E070E08C918230B1
:10C7E00020F46FEF70E04061A4C0843009F464C0AD
:10C7F000823009F463C0211531054105510509F462
:10C8000098C0FD0182819381FFEF82389F070CF071
:10C8100050C0A2E8EA2EAFEFFA2EE81AF90A8AE130
:10C82000E816F1040CF06BC06B0181E090E0A0E031
:10C83000B0E00E2C04C0880F991FAA1FBB1F0A94DA
:10C84000D2F70197A109B10982239323A423B52329
:10C850000097A105B10519F0F1E0CF2ED12C04C04D
:10C860005695479537952795EA94D2F7C601AA279A
:10C8700097FDA095BA2F282B392B4A2B5B2BDA0179
:10C88000C9018F779070A070B07080349105A105B8
:10C89000B105D1F1215C3F4F4F4F5F4F2030E0E0B9
:10C8A0003E07E0E04E07E0E45E0708F161E070E07B
:10C8B0001EC0803891053CF06FEF70E020E030E062
:10C8C00040E050E036C0BC0161587F4FDA01C90139
:10C8D0008F779070A070B07080349105A105B1057C
:10C8E000D1F0215C3F4F4F4F5F4F57FD1BC097E08A
:10C8F00056954795379527959A95D1F71AC020E018
:10C9000030E040E050E0BBCF27FFC8CF205C3F4F76
:10C910004F4F5F4FC3CF27FFE8CF205C3F4F4F4FB4
:10C920005F4FE3CF56954795379527956F5F7F4FBC
:10C93000DECF822E932E942F9F778A2D8078A82E7B
:10C94000A92A962F9795992797958A2D8F77A82EA4
:10C95000A92A76956795962F9F778B2D8078B82E8C
:10C96000B92A902F9795992797958B2D8F77B82E69
:10C97000B92AD501C401BC01CD01ECE0CDB7DEB7C9
:10C980000C949266CF93DF93FC01DB0140815181CF
:10C990002281622F6F7770E0221F2227221F93814E
:10C9A000892F880F822B282F3327991F9927991FAA
:10C9B000ED0199832115310541F4411551056105BA
:10C9C0007105E1F482E08C9354C02F3F310509F4E6
:10C9D00041C02F573040FD013383228383E08C9385
:10C9E00087E0440F551F661F771F8A95D1F7706443
:10C9F000ED014C835D836E837F833BC022E83FEF74
:10CA0000F901C7E0440F551F661F771FCA95D1F77C
:10CA100083E08C93403080E0580780E0680780E432
:10CA2000780778F4440F551F661F771F2150304058
:10CA3000F9014030C0E05C07C0E06C07C0E47C074F
:10CA400088F3ED01FB83EA83FD014483558366830C
:10CA500077830FC0411551056105710519F484E014
:10CA60008C9307C064FF03C081E08C93C1CF1C92FC
:10CA7000BFCFDF91CF9108950F931F93CF93DF9393
:10CA8000FC01DB018081823018F09C91923018F417
:10CA900061E070E05EC08430C1F0843001F1943018
:10CAA00009F447C0823009F44BC0823009F44EC00B
:10CAB0009230A9F04181ED0189814817B9F04423F2
:10CAC00089F08FEF9FEFBC0144C0943031F7EB0148
:10CAD0008981682F77278181681B71093AC081811C
:10CAE000882379F781E090E0BC0133C02281338153
:10CAF000ED018A819B81821793070CF32817390770
:10CB00009CF00481158126813781FD016481758146
:10CB100086819781601771078207930780F2061755
:10CB200017072807390778F4442359F281E090E089
:10CB3000DBCFFD018181882321F281E090E0D4CF19
:10CB4000923009F0B2CF60E070E003C0ED0189815E
:10CB5000F2CFCB01DF91CF911F910F910895FB018F
:10CB6000DC0105900D920020E1F70895FB01DC0146
:10CB700004C08D910190801921F441505040C8F7B4
:10CB8000881B990B0895FB01DC0140FF05C002C022
:10CB900001900D9201900D9242505040C8F70895B7
:10CBA000DC0140FF03C001C06D936D9342505040C3
:10CBB000D8F70895FB01DC0101900D920020E1F708
:10CBC0000895629FD001739FF001829FE00DF11DD7
:10CBD000649FE00DF11D929FF00D839FF00D749FF7
:10CBE000F00D659FF00D9927729FB00DE11DF91FA3
:10CBF000639FB00DE11DF91FBD01CF011124089500
:10CC0000991B79E004C0991F961708F0961B881F9E
:10CC10007A95C9F780950895AA1BBB1B51E107C0FF
:10CC2000AA1FBB1FA617B70710F0A61BB70B881FBC
:10CC3000991F5A95A9F780959095BC01CD0108954B
:10CC400097FB092E07260AD077FD04D0E5DF06D032
:10CC500000201AF4709561957F4F0895F6F790952E
:10CC600081959F4F0895A1E21A2EAA1BBB1BFD01BF
:10CC70000DC0AA1FBB1FEE1FFF1FA217B307E407BB
:10CC8000F50720F0A21BB30BE40BF50B661F771F13
:10CC9000881F991F1A9469F76095709580959095F3
:10CCA0009B01AC01BD01CF01089597FB092E05261C
:10CCB0000ED057FD04D0D7DF0AD0001C38F45095B1
:10CCC0004095309521953F4F4F4F5F4F0895F6F7B0
:10CCD00090958095709561957F4F8F4F9F4F0895E8
:10CCE0002F923F924F925F926F927F928F929F927C
:10CCF000AF92BF92CF92DF92EF92FF920F931F936A
:10CD0000CF93DF93CDB7DEB7CA1BDB0B0FB6F8941A
:10CD1000DEBF0FBECDBF09942A88398848885F845A
:10CD20006E847D848C849B84AA84B984C884DF80CB
:10CD3000EE80FD800C811B81AA81B981CE0FD11DAF
:10CD40000FB6F894DEBF0FBECDBFED010895F9997F
:10CD5000FECFB2BDA1BDF89A119600B40895F7DFD9
:10CD600001921A94E1F70895F999FECFB2BDA1BDE1
:10CD700000BC11960FB6F894FA9AF99A0FBE08956E
:0ACD80000190F2DF1A94E1F7089524
:10CD8A00012E2E2F63616E5F696E7075742E6300BB
:10CD9A006E222E2E2F6368616E6E656C732E630091
:10CDAA0053657175656E636520233100536571752E
:10CDBA00656E63652023320053657175656E636520
:10CDCA002023330053657175656E63652023340033
:10CDDA00455233002E2E2F656570726F6D63686140
:10CDEA006E6E656C732E630050434D3000455233AE
:10CDFA00004C4F4730340050434D2076657220393D
:10CE0A002E3139004F425220383434300B002E2E46
:10CE1A002F7669727475656C5F696E7075742E63AE
:0ACE2A0000000000000000000000FE
:00000001FF
